:100000000C94A80E0C94D90E0C94D90E0C94D90E05
:100010000C94D90E0C94D90E0C94D90E0C94D90EC4
:100020000C94D90E0C94D90E0C94D90E0C94D90EB4
:100030000C94D90E0C94D90E0C94D90E0C94356EE8
:100040000C94D90E0C94D90E0C94D90E0C94D90E94
:100050000C94D90E0C94D90E0C94D90E0C9410510A
:100060000C94D90E0C9441A10C9417A10C94D90EA8
:100070000C94D90E0C94D90E0C94D90E0C94D90E64
:100080000C94D90E0C94D90E0C94D90E0C94D90E54
:100090000C9407A20C9477A10C94BEA10C94BA9175
:1000A0000C94D90E0C94D90E0C94D90E0C94D90E34
:1000B0000C94D90E0C94D90E0C94D90E0C94D90E24
:1000C0000C94D90E0C94D90E0C94D90E0C94E1A07A
:1000D0000C94B7A00C94D90E0C94D90E0C94D90E94
:1000E0000C94D90E80127312D812D812D812D812CA
:1000F000D812D812D812D812D812040FAE11B111DA
:10010000BD11D311FD11CC11D812D812D812D812AA
:10011000D812A012B212CD12D318C718C718D3180C
:10012000D318AE18BB18BB18D318D318621D621DA4
:100130004A204A204A20BE1D991D991D991D7A1DED
:100140007A1DFA203321BF203721372192206220E7
:100150003721FA20FA207A32D6321A3377338C33A9
:10016000AD32263326332633A1328D32A9334037C0
:1001700040374F37283728372F37483748374837E1
:10018000283728376C376C378537673767377837C4
:1001900071377137713767376737003C033C1B3C59
:1001A000323C7C3C8F3CAF3CFE3FED3FF03FF83FA4
:1001B000F83FF03FED3FF83FF83FF83FED3FED3FB0
:1001C000ED3FF83FF83FF83FF83FF83FF83FF83F82
:1001D000F83FF83FF83FFE3F974C9A4C894C8D4CC6
:1001E000934CD14C9E4CA24CA84CAC4CB04CB64C51
:1001F000BA4CBE4CD14CC44CC84CCC4C664D6B4D2B
:10020000704D7A4D844DFD4D8E4D964D9E4DA84DB1
:10021000B24DBC4DCB4DD54DFD4DDF4DE94DF34DB0
:10022000BB5CE15C145D1D5D205D145DF15C145DE3
:100230002B5D2E5D025D3A5D3D5D3B62A0636F62AA
:100240008B62A063AD62A063E162FD621F635663CF
:100250007263286439642B642B6439642E643964B6
:10026000316431643164316431642B649C66A96605
:10027000AD66AD66C866C866B766B166BE660C791F
:10028000807880781B79B879B6790C7925792579C9
:1002900025790C790C79D578C878AA7893789078F4
:1002A000C878DA78FC78FC78B578B57842797179D5
:1002B0008579717971793579617961796179477970
:1002C0005379DA79147ADA79C979C979DA79DA7904
:1002D0005F7C5F7CDA79DA7956AC56AC56AC56ACBA
:1002E00053AC53AC5AAC5AAC5AAC5AAC5AAC5AACEC
:1002F0005AAC5AAC53AC53AC5AAC5AAC5AAC5AACDC
:100300005AAC58AC56AC07634236B79BD8A71A39DB
:10031000685618AEBAAB558C1D3CB7CC5763BD6D53
:10032000EDFD753EF6177231BF000000803F0800FA
:100330000000BE922449123EABAAAA2ABECDCCCC64
:100340004C3E00000080BEABAAAAAA3E00000000FE
:10035000BF000000803F0000000000084178D3BBD0
:100360004387D1133D190E3CC3BD4282AD2B3E687D
:10037000EC8276BED98FE1A93E4C80EFFFBE01C46E
:10038000FF7F3F00000000000C9448370C947A4C2B
:100390000C948B8A0C949F710C94F03F0C943A7FD0
:1003A0000C9480780C94964D0C94D69E0C94323C10
:1003B0000C941A330C94695B0C947A4D0C9442792A
:1003C0000C940A310C941B3C0C94B2120C949220A5
:1003D0000C9462830C94B73A0C946B460C94FD62B7
:1003E0000C94867E0C949A9F0C94991D0C94D812B0
:1003F0000C9471390C94F1520C945E8A0C948579AA
:100400000C943F8A0C948D4C0C94556C0C94C358EE
:100410000C94BA510C94AA510C94FC780C94828AD6
:100420000C94D6320C94BF200C94B5780C94477978
:100430000C94E94D0C941E7E0C948F7D0C949A4C78
:100440000C949C370C94C78E0C9488B10C94BF39D3
:100450000C94423B0C94576C0C94A9660C946179F3
:100460000C9481890C94AD320C94C0580C949C7DF2
:100470000C948A8A0C94DD8C0C94025D0C94F67DAD
:100480000C94A1320C94A84C0C943A5D0C94B76671
:100490000C94A0630C943A5A0C9467370C94DA7954
:1004A0000C94AE180C948B2B0C94323A0C94BA4CDE
:1004B0000C94704D0C94BC4D0C94B9510C940C7967
:1004C0000C94C8660C94468B0C94DA510C942E5DF7
:1004D0000C940D530C94622C0C94AD620C94EA2C89
:1004E0000C94C83A0C9493780C94B6790C94093E09
:1004F0000C94368F0C942E5B0C94892B0C94907872
:100500000C94C44C0C9456630C940B530C94AC5840
:100510000C94AE110C94621D0C940E310C94263385
:100520000C94ABAD0C94356C0C9477330C94205D2B
:100530000C947E830C94AEAD0C94974C0C941CA040
:100540000C94758D0C94033C0C94844D0C9439647C
:100550000C94CB5B0C94AF3C0C9431640C94CAB3F8
:100560000C94399E0C947A320C94FE3F0C94BB5C34
:100570000C9453AC0C9438860C94FD110C94C46C00
:100580000C94AC4C0C947A9F0C94CC4C0C94D97D6C
:100590000C949E4D0C9462200C946D830C948D7D74
:1005A0000C94664D0C9473120C94E66C0C9472636C
:1005B0000C94A68F0C943D5D0C9433210C948537DC
:1005C0000C94C7180C94ED3F0C94368E0C94803923
:1005D0000C94B1590C946F620C94639E0C941D5D45
:1005E0000C9471370C94B1110C946E8A0C94B68FE4
:1005F0000C94638E0C94729E0C94A9330C945379D2
:100600000C94D3110C94C8780C9452840C942A8CBA
:100610000C945AAC0C945F840C94716D0C94A7519B
:100620000C944F370C948E4D0C94BD8D0C94393A2C
:100630000C94B24D0C94B8790C94003C0C94357920
:100640000C940F310C9480830C94F15C0C94F53A6B
:100650000C94BB180C94652A0C94E53A0C9458AC95
:100660000C9482830C94A24C0C945A8A0C94744679
:100670000C94778A0C948B620C94F34D0C94147A3E
:100680000C94D18A0C94692A0C9469460C94948D2C
:100690000C94AA6C0C944A200C94D5780C942B5D85
:1006A0000C94662A0C94CD390C9428640C948846DA
:1006B0000C947D830C94255B0C94BE660C948C3357
:1006C0000C94BD110C94A78F0C94B1660C94FD4D45
:1006D0000C941B790C94934C0C94D5510C94DF4DD5
:1006E0000C9425790C94239F0C9440370C944B6CFC
:1006F0000C94787F0C94D14C0C94C4B30C948F3C24
:100700000C9456AC0C9471790C9470830C946E2AF2
:100710000C94AA780C946C830C94A58F0C94BE4C0A
:100720000C946C370C94B04C0C94CC110C94E1628A
:100730000C94949E0C94F83F0C942E640C943721E6
:100740000C94C9790C942B640C94408A0C94E15C51
:100750000C94DA780C94D28F0C94562A0C94A01234
:100760000C94F8390C94CD120C94145D0C949C6686
:100770000C94B64C0C94CB4D0C94836C0C94168654
:100780000C94894C0C94A66C0C94AD660C94D54DCD
:100790000C940A3A0C94CA8F0C946B4D0C94D31899
:1007A0000C947A1D0C943B620C94A82C0C94783712
:1007B0000C9414550C94EB510C94FA200C94A84D05
:1007C0000C942F370C94869E0C948D320C949D398A
:1007D0000C947C3C0C94A07D0C94040F0C94388CED
:1007E0000C9420530C94FF8F0C941F630C94BE1D2B
:1007F0000C945F7C0C94005C0C9480120C94568AD0
:100800000C949E4C0C94C84C0C9428376364696E0D
:100810006F70737578585B00476F74204950206182
:100820006464726573733A00276970205B69705B5A
:100830002C646E735B2C67775B2C7375626E6574CA
:100840005D5D5D5D27202D20736574207374617478
:1008500069632049500A004661696C656420746FC1
:1008600020636F6E6669677572652045746865728E
:100870006E6574207573696E6720444843502E205E
:10088000596F752063616E20736574206970206DE7
:10089000616E75616C6C7921000A75736573204413
:1008A0004843500A00204D41534B3A002047573AE5
:1008B0000020444E533A004C6F61646564206672B8
:1008C0006F6D20666C6173682049503A0053746103
:1008D0007274696E67206C616E00246E6F6465735C
:1008E0000024666F726D61740024646174617479B0
:1008F000706500302D31303000696E746567657247
:100900000068737600636F6C6F72004F4E2C4F4619
:10091000462C48414C542C524553542C584F4E2C85
:10092000584F46462C544F47474C4500656E756DF1
:1009300000666C6F617400332E302E310024686FB6
:100940006D696500757074696D652C6672656568A2
:1009500065617000303437346330615F323032317A
:100960002D30342D3032004C696768744875622030
:1009700000246E616D650072656164790020747297
:100980007920616761696E20696E20352073656327
:100990006F6E6473006661696C65642C2072633DE0
:1009A000004177616974696E6720666F72207265B5
:1009B0007461696E656420746F7069637300636F3E
:1009C0006E6E65637465642061732000202E2E2E88
:1009D0000020757365723A003A000A417474656DBF
:1009E0007074696E67204D51545420636F6E6E654C
:1009F0006374696F6E20746F200024737461746572
:100A000000646973636F6E6E65637465640055732B
:100A1000696E67204D5154542070617373776F7203
:100A2000642066726F6D20636F6E666967004E3A70
:100A300000446576696365204E616D653A005265D4
:100A400062696E6420737563636573732E20495009
:100A500020616464726573733A004572726F723A12
:100A600020726562696E64206661696C0052656E11
:100A70006577656420737563636573732E204950D1
:100A800020616464726573733A004572726F723AE2
:100A90002072656E65776564206661696C000A4E38
:100AA0006F206C696E6B00416363657074696E677B
:100AB00020636F6D6D616E64732E2E2E0A0044529A
:100AC000590046414E5F4F4E4C5900584F4E00481A
:100AD000414C54002054533A0020543A003D0050F9
:100AE000696E3A00447269766572205265733A0005
:100AF000416C72656164792048616C7465640A00B8
:100B0000416C726561647920496E616374697665D0
:100B10000A00416C7265616479204163746976658D
:100B20000A005475726E696E6720584F4E0A00585D
:100B30004F464620736B69707065642E2050726555
:100B40007620636D643A005475726E6564206F663A
:100B5000662066726F6D3A00526573746F726564D9
:100B60002066726F6D3A004E6F2073746F72656409
:100B70002076616C756573202D2064656661756CE7
:100B8000743A200049676E6F7265642C2063686157
:100B90006E6E656C20636D643D004F75744F664DDD
:100BA000656D6F7279210A003B200020436D643D22
:100BB00000205375623D00204974656D3D0052412F
:100BC0004D3D005265747279696E672064696D6D80
:100BD000657220434D440A004D6F64627573207046
:100BE0006F6C6C696E67206572726F723D00205683
:100BF000616C3A20004D423A20004E6F74207375AC
:100C000070706F72746564207265672074797065A6
:100C10000A00496C6C6567616C20617267756D656F
:100C20006E74730A005265747279696E6720564358
:100C300020434D440A004D6F6462757320706F6CE1
:100C40006C696E67206572726F723D002D002050D6
:100C5000492056616C203A004D6F646275732070B4
:100C60006F6C6C696E67206572726F723D002D004B
:100C700020464D2056616C203A00526574727969A5
:100C80006E672056432074656D7020434D440A0002
:100C900050574D2D4F757420496E69740050574D53
:100CA0002D4F75742073746F700052474220505757
:100CB0004D002050574D00524742572050574D008D
:100CC0003D0050696E3A00312D7769726520636F7F
:100CD000756E743A200020416464723A006465764F
:100CE000230020616C69766500204E6F64653A00D0
:100CF000536561726368696E6700312D776972654B
:100D00002073686F72746564005B305D3A20002068
:100D10002D202D202D20EFBBBF003E003E31202D89
:100D2000200020002D3E00436F6E76657274696E60
:100D300067200053617665643A0020537566663A11
:100D4000002041543A00206973200044656C6574AA
:100D5000696E6720636F6E662E2052414D20776169
:100D6000733A0053746F707065640053746F7070E1
:100D7000696E67206368616E6E656C73202E2E2E1F
:100D800000556E6C6F636B696E6720636F6E66698A
:100D900067202E2E2E00536B697070696E672E2EA1
:100DA000004F75744F664D656D6F727921005D203F
:100DB000000A5B003A004D41433A0055445020532D
:100DC00079736C6F6720696E697469616C697A65A3
:100DD000642E0A005379736C6F6720706172616DC5
:100DE000733A0020616374697665200020696E6142
:100DF000637469766520002076616C75652069737F
:100E0000200020756E6B6E6F776E0A00204772703F
:100E10003A0020696E76616C6964004D6F6462759A
:100E200073206F70206661696C65640A003D00562E
:100E300043230020636D643D003D0056435F6865B9
:100E4000617423005374617475732064656666650C
:100E50007265640A002D3E005075623A2000636D91
:100E60006400434F4F4C0048454154004155544F96
:100E7000002D3E005075623A2000736574002D3ECF
:100E8000005075623A20002D3E005075623A2000F5
:100E9000556E6B6E6F776E20636D64200A004F464F
:100EA00046004F4E0043757272656E74204C414E81
:100EB00020636F6E6669672869702C646E732C6797
:100EC000772C7375626E6574293A000A5573652034
:100ED000746865736520636F6D6D616E64733A202D
:100EE0002768656C7027202D2074686973207465ED
:100EF00078740A276D61632064653A61643A6265BB
:100F00003A65663A66653A30302720736574206129
:100F10006E642073746F7265204D41432D6164646B
:100F20007265737320696E20454550524F4D0A27F4
:100F30006970205B69705B2C646E735B2C67775BF8
:100F40002C7375626E65745D5D5D5D27202D207369
:100F50006574207374617469632049500A27736152
:100F6000766527202D207361766520636F6E666934
:100F70006720696E204E5652414D0A2767657427D7
:100F8000205B636F6E66696720616464725D272011
:100F90002D2067657420636F6E6669672066726FC7
:100FA0006D207072652D636F6E666967757265641A
:100FB0002055524C20616E642073746F72652061FD
:100FC0006464720A276C6F616427202D206C6F6146
:100FD0006420636F6E6669672066726F6D204E567F
:100FE00052414D0A2770776427202D206465666979
:100FF0006E65204D5154542070617373776F726425
:101000000A276B696C6C27202D2074657374207718
:1010100061746368646F670A27636C656172272077
:101020002D20636C65617220454550524F4D0A2753
:101030007265626F6F7427202D207265626F6F7406
:1010400020636F6E74726F6C6C657200536F6674A0
:10105000207265626F6F74696E672E2E2E00444D8C
:1010600058696E2042756666657220616C6C6F63AC
:101070002065727200496E697420696E2063683A57
:1010800000444D584F75742E20467265653A00092C
:10109000445332343832206572726F7200095265DF
:1010A00073657420646F6E650009436865636B69DE
:1010B0006E6720666F7220312D57697265206465F6
:1010C00076696365732E2E2E004453323438322DE8
:1010D0003130302070726573656E74004572726FC6
:1010E0007220312D7720696E697420233220467278
:1010F00065653A0077737461742E20467265653AAF
:10110000005465726D2E20467265653A0045727214
:101110006F7220312D7720696E697420233100466B
:101120007265653A004453323438325F3130305F93
:101130004932435F544F5F31575F425249444745FC
:1011400020696E69740020416464723A00646576B7
:10115000230052414D3D000A312D77697265200010
:101160000A6D71747420000A6D6F64627573207665
:1011700032000A6D6F6462757320763120282B2946
:10118000000A696E7075747320000A6974656D7366
:1011900020000A436F6E666967757265643A003BAA
:1011A000003D0050696E3A003B003D4C4F570054E3
:1011B0006865726D6F3A004F6E65207769726520C1
:1011C00052656164790A00467265653A00444D587B
:1011D000206F757420737461727465642E20436887
:1011E000616E6E656C733A2000444D5820696E2024
:1011F000737461727465642E204368616E6E656CF1
:10120000733A003E3E3E004E6F204D414320636FD7
:101210006E666967757265643A20736574206669E5
:10122000726D776172652773204D41430A0000009B
:101230002200250028002B002E003100340002017E
:101240000000050108010B0100000A0B02090C0D4A
:101250000E08070304010000000000000000000069
:10126000000000000000000000000000000000007E
:10127000000000001211100000000000000000003B
:101280000000000000000000000000000000204FEF
:10129000464600204F4E00757074696D6500667299
:1012A0006565686561700024737461747300200063
:1012B00020000A52414D3D002045787069726564F6
:1012C0000A00202D746172676574207A6F6E652D37
:1012D0000020416C61726D20457870697265640A06
:1012E0000020636D643A00204375723A0020536514
:1012F000743A00444D582D4F757420496E6974003E
:10130000444D582D4F75742073746F700041737382
:1013100069676E65643A00444D58206374726C3A94
:10132000200044656661756C742073657269616C38
:10133000206D6F6465204E38312075736564003808
:101340004531002600384E31000600384532002E67
:1013500000384E32000E00384F31003600384F3220
:10136000003E00374531002400374E31000400377D
:101370004532002C00374E32000C00374F3100341C
:1013800000374F32003C00203D3E004D6F646275D7
:10139000732074656D706C617465206E6F74206667
:1013A0006F756E643A2000496E76616C69642074D2
:1013B000656D706C6174652E002C002C002C002C67
:1013C000004D4255533A20636F6E6669672066612F
:1013D000696C65643A004D6F6462757320636F6E6B
:1013E000666967206572726F72004D6F6462757313
:1013F00020636F6E666967206C6F616465642000AE
:101400004D4255533A204F7574206F66206D656DBF
:101410006F7279004D4255533A20506F6C6C696E73
:1014200067206572726F7220004E6F742073757042
:10143000706F727465642072656720747970650AD4
:1014400000656E64506F6C6C20002D2D2D00506F68
:101450006C6C2000556E6B6E6F776E2073756666D0
:1014600069782000556E6B6E6F776E20636D642017
:1014700000636C724374723A20002F00496E3A2068
:10148000002D3E002000230050656E6465642073CB
:1014900074617465207265747269657665643A007A
:1014A0003D004C454741435920494E3A003D0049D3
:1014B0004E3A00000020002300260029002C002FB7
:1014C0000032000001000003010601090169313604
:1014D0000001693332000275313600037533320082
:1014E00004693868000569386C00067538680007BB
:1014F00075386C000878313000094164642040532D
:101500003A20003A002066726F6D20004D4220673D
:101510006F74200000002100240027002A002D0005
:101520003000330001010000040107010A0101023B
:1015300010202008081020401020408002010201E5
:10154000080402010102040810204080804020109D
:1015500008040201800402018040201008040201F6
:10156000080402010102040810204080010204085E
:101570001020408005050505070508080808020237
:1015800002020A0A0808040404040101010101011D
:1015900001010303030303030303040707070C0C00
:1015A0000C0C0C0C0C0C02020202060606060606C7
:1015B00006060B0B0B0B0B0B0B0B005EBCE2613F2B
:1015C000DD83C29C7E20A3FD1F419DC3217FFCA221
:1015D000401E5F01E3BD3E6082DC237D9FC1421C53
:1015E000FEA0E1BF5D0380DE3C62BEE0025CDF8105
:1015F000633D7C22C09E1D43A1FF4618FAA42779B3
:101600009BC584DA3866E5BB5907DB856739BAE4E0
:1016100006581947A5FB7826C49A653BD987045A12
:10162000B8E6A7F91B45C6987A24F8A6441A99C7C4
:10163000257B3A6486D85B05E7B98CD2306EEDB372
:10164000510F4E10F2AC2F7193CD114FADF3702EA0
:10165000CC92D38D6F31B2EC0E50AFF1134DCE90D2
:10166000722C6D33D18F0C52B0EE326C8ED0530D84
:10167000EFB1F0AE4C1291CF2D73CA947628ABF532
:1016800017490856B4EA6937D58B5709EBB5366860
:101690008AD495CB2977F4AA4816E9B7550B88D692
:1016A000346A2B7597C94A14F6A8742AC896154B44
:1016B000A9F7B6E80A54D7896B35436F6E6E656338
:1016C0007465642E00436F6E6E2E2061626F7274BB
:1016D0006564000000000000000000004F4E0000A4
:1016E00000000000004F4646000000000000524588
:1016F00053540000000000544F47474C4500000081
:1017000048414C540000000000584F4E00000000BB
:101710000000584F46460000000000494E43524525
:1017200041534500444543524541534500484541D6
:10173000540000000000434F4F4C000000000041E7
:1017400055544F000000000046414E5F4F4E4C592B
:101750000044525900000000000053544F50000054
:101760000000004849474800000000004D4544493A
:10177000554D0000004C4F5700000000000054522F
:101780005545000000000046414C53450000000054
:10179000454E41424C4544000044495341424C456A
:1017A0004400524742000000000000485356000029
:1017B0000000000054787432436D643A004E6F7438
:1017C00020737570706F7274656420726567207421
:1017D0007970650A00293A0028543A003D3E002DF0
:1017E0003E0057726F6E672041737369676E6D6557
:1017F0006E742000524742783A200020764C65767D
:10180000656C3A0020436F6E76563A0020436F6E47
:1018100076533A0020486F743A00436F6C643A0084
:1018200020436F6E76657274656420563A00436F8C
:101830006E76657274656420533A002D3E005772CF
:101840006F6E672041737369676E6D656E742000FB
:101850002D3E0057726F6E672041737369676E6D1E
:10186000656E7420004C6F61646564006C6F616428
:10187000206661696C6564004E6F2073746F7265D9
:101880006420636F6E666967004C6F6164696E67A0
:1018900020436F6E6669672066726F6D2045455004
:1018A000524F4D000A72657175657374204D515425
:1018B0005420436F6E6669670053617665642074D7
:1018C0006F20454550524F4D00536176696E672039
:1018D000636F6E66696720746F20454550524F4DA7
:1018E0002E2E0053617665640A0053657420647976
:1018F0006E616D69632049500A00454550524F4D55
:1019000020636C65617265640A0050617373776F60
:10191000726420757064617465640A00636F756C2D
:1019200064206E6F742070617273653A2000557088
:1019300064617465640A002B002D00485454502FD4
:10194000312E312025690020485454502F312E313A
:101950000D0A486F73743A2025730D0A416363655D
:1019600070743A202A2F2A0D0A436F6E6E656374D5
:10197000696F6E3A20636C6F73650D0A0025730002
:1019800020000D0A00474554006661696C656420BB
:10199000746F20636F6E6E6563740A004552524F18
:1019A000523A205365727665722072657475726E54
:1019B00065642000446F6E652E0A004170706C797A
:1019C000696E672E0A00436F6E66696720706172E8
:1019D00073696E67206661696C65640A00676F747D
:1019E00020436F6E6669670A00436F6E6669672001
:1019F0005552493A20687474703A2F2F002044657C
:101A00006661756C7420636F6E66696720736572BA
:101A100076657220757365643A20006C617A796826
:101A20006F6D652E727500205361766564000A281B
:101A30002B295359534C4F47000A282B295049440E
:101A4000000A282D294D43503233303137000A28FF
:101A50002D294152544E4554000A282D294F5441F6
:101A6000000A282D29535049204C4544000A282DAE
:101A7000294D4F544F5220435452000A282D2941DA
:101A800043204841494552000A282D2943435338F1
:101A9000313120262048444331303830000A282D87
:101AA00029524553544152545F4C414E5F4F4E5F53
:101AB0004D5154545F4552524F5253000A282D291C
:101AC0004841524452455345542C207573696E6702
:101AD00020736F6674000A282D29434F554E5445D4
:101AE00052000A282D29444854000A282B294F5710
:101AF000495245000A282B294D4F44425553000AAC
:101B0000282B294144414652554954204C45440014
:101B10000A282B29444D58000A282B2957697A6E28
:101B2000657435313030000A282B2944533234385B
:101B3000322D313030000A282B29467265655261FA
:101B40006D207072696E74696E6700435553544F0F
:101B50004D5F4649524D574152455F4D4143000A42
:101B60004669726D77617265204D4143204164641E
:101B70007265737320006C617A79686F6D652E727F
:101B800075000A436F6E66696720736572766572C9
:101B90003A000A282B295741544348444F47003202
:101BA00030313130334C0020432B2B20766572735B
:101BB000696F6E3A00303437346330615F323032EF
:101BC000312D30342D3032000A4C617A79686F6DD6
:101BD000652E7275204C6967687448756220636F62
:101BE0006E74726F6C6C65722000556E6B6E6F77E1
:101BF0006E207375666669782000556E6B6E6F7720
:101C00006E20636D642000466F72636564206578A2
:101C100065637574696F6E00496E76616C696420E6
:101C200050494420706172616D2061727261792E39
:101C3000002C002C002C002C005049443A20636FEB
:101C40006E666967206661696C65643A0050494454
:101C500020636F6E666967206C6F61646564200045
:101C600050494420636F6E666967206572726F72B7
:101C7000005049443A204F7574206F66206D656DA1
:101C80006F727900556E6B6E6F776E207375666636
:101C900069782000556E6B6E6F776E20636D6420DF
:101CA00000536574706F696E743A00496E70757494
:101CB0002076616C75653A00696E00735F6F7574AC
:101CC000006D79686F6D6500202D3E2000202D3E4F
:101CD0002000202D3E20002C20002E003E3E200023
:101CE000496E76616C696420636F6D6D616E64002E
:101CF00076616C0074656D70007361740068756561
:101D00000066616E0052474200485356006D6F6492
:101D10006500536574436D643A00536574466C61A5
:101D2000673A00436C72466C61673A0053746F7295
:101D30006564204558543A00737566666978436F48
:101D400064653A003E003C00543A0000CAB3C4B394
:101D500011241FBECFEFD1E2DEBFCDBF00E00CBF2C
:101D600017E0A0E0B2E0ECEEFAE801E00BBF02C041
:101D700007900D92AC30B107D9F72EE0ACE0B7E098
:101D800001C01D92A032B207E1F71EE0C7EADEE013
:101D900000E006C021970109802FFE010E94DEBFEE
:101DA000C63AD10780E00807A9F70E9438B20C9420
:101DB00064C50C9400004F925F926F927F928F9255
:101DC0009F92AF92BF92CF92DF92EF92FF920F93CA
:101DD0001F93CF93DF93CDB7DEB7C25AD1400FB672
:101DE000F894DEBF0FBECDBF2091FC083091FD08F6
:101DF000F9013B96EA31F10508F0DAC38827EE587D
:101E0000FF4F8F4F0C94DEBF0EEB13E0CE56DE4F2C
:101E100019830883C259D140CC56DE4F18821982EB
:101E20001A821B82C459D140CE57DE4F19830883D2
:101E3000C258D140CC57DE4F188219821A821B82B9
:101E4000C458D140CE59DE4F19830883C256D140C1
:101E5000CC59DE4F188219821A821B82C456D14097
:101E6000CE5BDE4F19830883C254D140CC5BDE4F7A
:101E7000188219821A821B82C454D1406DEC78E01A
:101E800083E29BE00E945EA083E29BE00E94A3515C
:101E9000BE016E567E4F86E090E00E941D6B892B3E
:101EA00009F467C167EB78E083E29BE00E945EA0E3
:101EB0001A830983CC56DE4F88819981AA81BB8120
:101EC000C459D1408B839C83AD83BE83CE010196E0
:101ED0000E94129ABE016E577E4F8AE090E00E94E7
:101EE0001D6B892B09F42EC161EB78E083E29BE046
:101EF0000E945EA01A830983CC57DE4F88819981A6
:101F0000AA81BB81C458D1408B839C83AD83BE839F
:101F1000CE0101960E94129ABE016E597E4F8EE04C
:101F200090E00E941D6B892B09F4DFC06CEA78E019
:101F300083E29BE00E945EA01A830983CC59DE4FA6
:101F400088819981AA81BB81C456D1408B839C83AF
:101F5000AD83BE83CE0101960E94129ABE016E5BD4
:101F60007E4F82E190E00E941D6B892B09F477C0BF
:101F700065EA78E083E29BE00E945EA01A83098311
:101F8000CC5BDE4F88819981AA81BB81C454D1404A
:101F90008B839C83AD83BE83CE0101960E94129AEF
:101FA0001A830983CC5BDE4F88819981AA81BB812A
:101FB000C454D1408B839C83AD83BE83CF57DF4F06
:101FC00019830883C158D040CC59DE4F888199814C
:101FD000AA81BB81C456D140CD57DF4F88839983F6
:101FE000AA83BB83C358D040CE53DF4F19830883E5
:101FF000C25CD040CC57DE4F88819981AA81BB81D9
:10200000C458D140CC53DF4F88839983AA83BB83C4
:10201000C45CD040CE5FDE4F19830883C250D140EC
:10202000CC56DE4F88819981AA81BB81C459D140A9
:10203000CC5FDE4F88839983AA83BB83C450D14091
:102040009E012F5F3F4FAE014F575F4FBE016E5352
:102050007F4FCE018E5F9E4F0E94FD6985C01A831F
:102060000983CC59DE4F88819981AA81BB81C456EE
:10207000D1408B839C83AD83BE83CF57DF4F1983C1
:102080000883C158D040CC57DE4F88819981AA81FE
:10209000BB81C458D140CD57DF4F88839983AA8331
:1020A000BB83C358D040CE53DF4F19830883C25C33
:1020B000D040CC56DE4F88819981AA81BB81C4591A
:1020C000D140CC53DF4F88839983AA83BB83C45C00
:1020D000D040AE014F5F5F4FBE016F577F4FCE01C3
:1020E0008E539F4F0E94496A3FC01A830983CC5781
:1020F000DE4F88819981AA81BB81C458D1408B83EE
:102100009C83AD83BE83CF57DF4F19830883C158AB
:10211000D040CC56DE4F88819981AA81BB81C459B9
:10212000D140CD57DF4F88839983AA83BB83C3589F
:10213000D040BE016F5F7F4FCE018F579F4F0E94EF
:102140009B6A12C01A830983CC56DE4F888199811D
:10215000AA81BB81C459D1408B839C83AD83BE834C
:10216000CE0101960E94E66A83E29BE00E94A351A1
:10217000F5C069E978E083E29BE00E945EA00FB6BB
:10218000F894A89580916000886180936000109217
:1021900060000FBE80916B07811107C080E597E05A
:1021A0000E942C8B81E080936B078DE097E09093E9
:1021B000CE098093CD090E946D69CE0101960E94DF
:1021C00093A789819A810E94E36C46E050E06AEC13
:1021D0007CE089E090E00E94F63E8EEB93E09A83EB
:1021E00089831B821C821D821E82CE0103960E945F
:1021F000CD6C0E94E26C8091CD099091CE09DC01FA
:1022000092961D921D921D921C929597FC0116A20A
:1022100017A210A611A69A961D921D921D921C92AD
:102220009D9740EE5EE260E070E046AB57AB60AF7A
:1022300071AF40EA5FE060E070E0DA964D935D9345
:102240006D937C93DD973E9624E1DF011D922A95E4
:10225000E9F726E0EAECFCE0DC01189601900D922B
:102260002A95E1F7FC01EE5BFF4F10820E948B671D
:102270008C01019709F04AC0CE0101960E9493A7F4
:1022800089819A810E94E36C6091CD097091CE0999
:10229000625F7F4FCE0101960E94ABA0CE010396F4
:1022A0000E94CD6C6091CD097091CE096A5E7F4F1E
:1022B000CE0101960E94ABA0CE0103960E94DB6C7A
:1022C0006091CD097091CE096E5E7F4FCE0101966F
:1022D0000E94ABA0CE0103960E94D46C0E94E26CD7
:1022E0006091CD097091CE09625E7F4FCE0101965B
:1022F0000E94ABA08B819C81AD81BE818093C90976
:102300009093CA09A093CB09B093CC0999E288E1D4
:102310000FB6F894A895809360000FBE909360006C
:10232000A895012B69F467E578E08EE29BE00E94B6
:102330005EA068E278E08EE29BE00E945EA032C17F
:1023400068E178E083E29BE00E945EA0CE01019606
:102350000E94A8A7CE0101960E94129A82E090E006
:1023600023C180917707811105C00E94283181E047
:102370008093770783E090E017C180913A0D811137
:1023800023C780910C0781110BC060E070E080E0F2
:1023900090E00E943B8108C10E9466A8811108C19B
:1023A00084E090E001C1A895CE55DE4F1882C25A54
:1023B000D140FE01EE56FE4F119211928EE0DF01E8
:1023C0001D928A95E9F70E9466A8882319F085E096
:1023D00090E0EAC00091F3081091F408011511058E
:1023E00009F444C2C8010E9425AAE82EF12CB2E0EB
:1023F000EB16F1040CF03DC239C20E94844E9B01E1
:10240000AC0160917307709174078091750790918A
:102410007607AA24AA94BA2C650118E8E12E13E1E4
:10242000F12E00E010E00E940293882309F4C0C05E
:1024300020E030E043E050E061E4CE0101960E94EC
:10244000B89362EA74E0CE0101960E946FC40091D5
:10245000E3091091E409B801CE0101960E941BB86E
:1024600009960817190790F10E9466A8882371F150
:102470008091E9099091EA09019611F481E090E0D8
:102480009093EA098093E909E091E109F091E2096A
:102490008091EA098583E091E109F091E209809158
:1024A000E90986836091E1097091E20947E050E013
:1024B000CE0101960E949DA8AC0145505109609142
:1024C000E1097091E20982EA0E94BDA886E090E0ED
:1024D0009093FD088093FC0867EA7AE083E29BE032
:1024E0000E945EA065C00E94844E60937307709343
:1024F0007407809375079093760785EF9FEF54C01C
:102500000E94844E9B01AC01609173077091740727
:102510008091750790917607AA24AA94BA2C650138
:1025200018E8E12E13E1F12E00E010E00E94029382
:10253000882309F43DC01092FD081092FC0838C0B1
:102540000E9466A881110E94689A0E94844E60933E
:1025500073077093740780937507909376078DE0E7
:1025600090E022C00E94844E9B01AC0160917307F1
:10257000709174078091750790917607AA24AA94A8
:10258000BA2C650110E1E12E17E2F12E00E010E017
:102590000E940293811104CF0BC00E94D280892B2C
:1025A00009F0FECE86EF9FEF9093FD088093FC0824
:1025B0000FB6F894A89580916000886180936000C0
:1025C000109260000FBE8091FC089091FD08029768
:1025D0000CF43DC10091CD091091CE0901151105F2
:1025E00009F435C10E94844E4B015C017801FEE381
:1025F000EF0EF11CF70180819181A281B381A501C9
:102600009401281B390B4A0B5B0BCA01B901683EC8
:1026100033E073078105910508F446C028EE33E0E6
:1026200040E050E00E9467BF861A970AA80AB90ADC
:10263000D7018D929D92AD92BC921397F80186A519
:1026400097A5A0A9B1A969017A01CC0CDD1CEE1CEB
:10265000FF1C8C159D05AE05BF0528F416A617A610
:1026600010AA11AA09C0821B930BA40BB50BF80189
:1026700086A797A7A0ABB1ABF80182A993A9A4A99B
:10268000B5A98C159D05AE05BF0528F412AA13AA9D
:1026900014AA15AA09C0821B930BA40BB50BF80151
:1026A00082AB93ABA4ABB5ABF80186A597A5A0A967
:1026B000B1A9892B8A2B8B2B69F4EE5BFF4F8081AC
:1026C000833041F484E08083C8010E948B670196C7
:1026D0007C0102C0E12CF12CF80182A993A9A4A9E4
:1026E000B5A9892B8A2B8B2BA1F4EE5BFF4F808140
:1026F000833011F081110DC01082F8013E9684E103
:10270000DF011D928A95E9F7C8010E948B67039645
:102710007C01B2E0EB16F10429F0E4E0EE16F104DE
:1027200009F04AC0CE0101960E9493A789819A813F
:102730000E94E36C6091CD097091CE09625F7F4F7A
:10274000CE0101960E94ABA0CE0103960E94CD6CF3
:102750006091CD097091CE096A5E7F4FCE010196DE
:102760000E94ABA0CE0103960E94DB6C6091CD0964
:102770007091CE096E5E7F4FCE0101960E94ABA094
:10278000CE0103960E94D46C0E94E26C6091CD0948
:102790007091CE09625E7F4FCE0101960E94ABA080
:1027A0008B819C81AD81BE818093C9099093CA09B8
:1027B000A093CB09B093CC09F3E0EF16F10461F1DB
:1027C0005CF431E0E316F104D1F042E0E416F104E8
:1027D000F1F56DE67AE02FC054E0E516F10449F119
:1027E00085E0E816F10499F56EE97AE08EE29BE067
:1027F0000E945EA08EE29BE00E94A35106C06AE8A0
:102800007AE08EE29BE00E945EA086EF9FEF9093BD
:10281000FD088093FC081BC06AE57AE08EE29BE02D
:102820000E945EA00E9466A8882379F30E94689A9D
:10283000ECCF6EE37AE083E29BE00E945EA0CE01E3
:1028400001960E94A8A7CE0101960E94129A99E2D1
:1028500088E10FB6F894A895809360000FBE90931E
:1028600060002091FC083091FD08AEC48EE090E03D
:102870009BCE60E070E0C8010E9412318C01909301
:10288000360D8093350D61E37AE083E29BE00E9490
:102890005EA0B80183E29BE00E94A9A083E29BE0D6
:1028A0000E94A3516EE27AE086ED9BE00E945EA05A
:1028B0004AE050E0B70186ED9BE00E9415A086ED4E
:1028C0009BE00E94A3510091F3081091F40861E08D
:1028D00070E0C8010E9412315C0192E0E916F10437
:1028E00091F062E0C8010E94A4A9FC01C184D284D5
:1028F000F3E0EF16F10459F063E070E0C8010E94C4
:1029000012318C0107C08BE5C82E87E0D82E8E01CE
:102910000E551E4F40E150E0BE016E567E4F86E3DD
:1029200090E00E948E80892B51F425E0E216F1049C
:102930000CF05FC3AE014E565E4F7A0104C0CE016B
:102940008E569E4F7C01B092FD09A092FC09D09258
:10295000FF09C092FE098CE997E39093F5098093F3
:10296000F40940E150E061E07AE0CE018E579E4FDD
:102970000E9408B820E030E041E050E060E2CE0183
:102980008E599E4F0E94B89340E250E06AEF79E082
:10299000CE018E599E4F0E94EAB76AED79E083E23C
:1029A0009BE00E945EA0B50183E29BE00E94A9A08B
:1029B00068ED79E083E29BE00E945EA04AE050E08F
:1029C000B60183E29BE00E9415A061ED79E083E20D
:1029D0009BE00E945EA0B80183E29BE00E94A9A058
:1029E0006CEC79E083E29BE00E945EA0D8018C91C0
:1029F000811104C0E12CF12C00E010E0A090350D15
:102A0000B090360D0E9466A881117DC18091DF09CA
:102A10009091E009DC01ED91FC910688F789E02DA9
:102A200019958823A1F081E090E09093EA098093C2
:102A3000E90987E0E2E1F2E0DE01119601900D92F2
:102A40008A95E1F7FE01319685E090E037C060910C
:102A5000FC097091FD098091DF099091E009409196
:102A6000FE095091FF09DC01ED91FC9161157105A2
:102A700021F00088F189E02D16C00684F785E02D4D
:102A80002EEB33E03A8329834090F8095090F909FE
:102A90006090FA097090FB094B825C826D827E82A5
:102AA000BE016F5F7F4F1995019709F4BCCF8EEF80
:102AB0009FEF9093030A8093020AAFC22191A091E5
:102AC000E109B091E209A80FB91F2C9301968C304F
:102AD0009105A1F70115110529F0E114F10421F088
:102AE00086EF03C086E301C086EBC090E109D09079
:102AF000E209F60184878091E60985878091E509DE
:102B000086878090E3099090E409B401C5010E9492
:102B10001BB841968816990608F4E9C04FE050E0CA
:102B2000B601C5010E949DA86C01A090E309B09078
:102B3000E409B501CE018E599E4F0E941BB88C0D41
:102B40009D1D0296A816B90608F4D1C06091E1094E
:102B50007091E209A601CE018E599E4F0E949DA858
:102B60006C01A090E309B090E409B501CE018E5745
:102B70009E4F0E941BB88C0D9D1D0296A816B9068B
:102B800008F4B5C06091E1097091E209A601CE0197
:102B90008E579E4F0E949DA86C0101151105B9F139
:102BA000A090E309B090E409B501C8010E941BB8E8
:102BB00096012E5F3F4F820F931FA816B90608F4A7
:102BC00096C06091E1097091E209A601C8010E94D6
:102BD0009DA86C01E114F104D1F00091E30910917A
:102BE000E409B801C7010E941BB896012E5F3F4F50
:102BF000820F931F0817190708F479C06091E10943
:102C00007091E209A601C7010E949DA86C01A6016E
:102C1000455051096091E1097091E20980E10E94FB
:102C2000BDA80E94844E6093EB097093EC098093D9
:102C3000ED099093EE096093EF097093F00980938A
:102C4000F1099093F2098091DF099091E009DC018C
:102C5000ED91FC910084F185E02D1995892B01F50A
:102C60000E94844E2091E7093091E809C090EF0955
:102C7000D090F009E090F109F090F2094B015C016D
:102C80008C189D08AE08BF08A8EEB3E00E94BBBF39
:102C900086169706A806B906B0F28CEF9FEF23C000
:102CA000CE018F579F4F0E942B976430710581058D
:102CB0009105E9F4E091E109F091E2098381811144
:102CC00011C00E94844E6093EF097093F0098093C5
:102CD000F1099093F2091092F3091092030A1092ED
:102CE000020A11C090E09093030A8093020A809137
:102CF000DF099091E009DC01ED91FC910488F589F0
:102D0000E02D19958AC10091350D1091360D6EEBAD
:102D100079E083E29BE00E945EA0B80183E29BE041
:102D20000E94A9A083E29BE00E94A35181E08093CE
:102D30000C0720E030E043E050E061E4CE018F5723
:102D40009F4F0E94B89362EA74E0CE018F579F4F65
:102D50000E946FC4CE018F579F4F0E94186920E0D8
:102D600030E042E050E061E4CE018F579F4F0E9477
:102D7000B89366EA74E0CE018F579F4F0E946FC4EC
:102D8000BE016F577F4F89E39BE00E94C077CE0161
:102D90008F579F4F0E94186920E030E041E050E0DB
:102DA00061E4CE018F579F4F0E94B89366EA74E0AA
:102DB000CE018F579F4F0E946FC4BE016F577F4F48
:102DC00089E39BE00E94C077CE018F579F4F0E94FE
:102DD0001869FE01EE5FFE4F119211921EE3DF01B2
:102DE000812E1D928A94E9F71A821982FE01339688
:102DF0008EE7DF011D928A95E9F720E030E041E09F
:102E000050E060E4CE018E5F9E4F0E94B89340E494
:102E100050E06AEF79E0CE018E5F9E4F0E94EAB7E4
:102E200040E850E067E779E0CE0101960E9408B8DB
:102E3000BE016F5F7F4FCE018E5F9E4F0E9488A9BB
:102E400020E030E041E050E060E4CE018E5F9E4F34
:102E50000E94B89340E450E061E779E0CE018E5FD4
:102E60009E4F0E94EAB740E850E067E679E0CE0165
:102E700001960E9408B840E850E064E579E0CE0190
:102E800001960E94EAB7BE016F5F7F4FCE018E5F51
:102E90009E4F0E9488A920E030E041E050E060E4CD
:102EA000CE018E5F9E4F0E94B89340E450E067EAE7
:102EB00072E1CE018E5F9E4F0E94EAB740E850E07B
:102EC00064E479E0CE0101960E9408B8BE016F5F0C
:102ED0007F4FCE018E5F9E4F0E9488A920E030E098
:102EE00041E050E060E4CE018E5F9E4F0E94B893B7
:102EF00040E450E06DE379E0CE018E5F9E4F0E948A
:102F0000EAB740E850E067E379E0CE0101960E941D
:102F100008B8BE016F5F7F4FCE018E5F9E4F0E944B
:102F200088A980913A0D8F5F80933A0DA091FE0899
:102F3000B091FF08109709F444C080911902909154
:102F40001A02AE014E5B5E4FFA01819391932EE11E
:102F500011922A95E9F79E012E533F4FF901819373
:102F6000919311921A95E9F716960D911C91179766
:102F7000E090FE08F090FF08E114F10479F00115EB
:102F8000110561F0D80118968C918F708530A1F7EA
:102F9000C8010E9425AA882379F367C020E030E0A9
:102FA00041E050E060E4CE018E5F9E4F0E94B893F6
:102FB00040E450E06AED78E0CE018E5F9E4F0E94C3
:102FC000EAB780913A0D815080933A0D85E090E008
:102FD0009093FD088093FC080E94844E60937307D1
:102FE00070937407809375079093760761EA79E090
:102FF00075CA64E070E08091F3089091F4080E9433
:1030000012317C016EE07AE083E29BE00E945EA0D8
:1030100083E29BE00E94A35196CC0091020A10919A
:10302000030A65E979E08EE29BE00E945EA04AE037
:1030300050E0B8018EE29BE00E9415A06DE779E0B8
:103040008EE29BE00E945EA08EE29BE00E94A35174
:103050000E94844E60937307709374078093750782
:10306000909376078CE090E09FCA60E0C8010E94D0
:10307000A4A9FC0181859285A385B4858A30910538
:1030800008F463C020E030E041E050E060E4CE01AD
:103090008E5F9E4F0E94B893F8016081718140E479
:1030A00050E0CE018E5F9E4F0E9495C468EA74E0A6
:1030B000CE018E5F9E4F0E946FC440E450E069EEE7
:1030C00078E0CE018E5F9E4F0E94EAB7BE016E5B34
:1030D0007E4FCE018E5F9E4F0E9488A9CE53DF4F58
:1030E0008881C25CD040882361F120E030E041E07B
:1030F00050E060E4CE018E5F9E4F0E94B893D801ED
:103100006D917C9140E450E0CE018E5F9E4F0E9415
:1031100095C468EA74E0CE018E5F9E4F0E946FC432
:1031200040E450E061EE78E0CE018E5F9E4F0E9459
:10313000EAB7BE016E537F4FCE018E5F9E4F0E9455
:1031400088A9F8010281138113CFFC0140E250E00D
:103150008827E457FF4F8F4F0C94DEBF61E379E07F
:10316000CE018E5B9E4F0E9408B8CE53DF4F18826F
:10317000C25CD04087CF6CE279E0CE018E5B9E4F7F
:103180000E9408B840E450E06BE079E017C065E0C9
:1031900079E0CE018E5B9E4F0E9408B840E450E07B
:1031A00061E079E00BC069EF78E0CE018E5B9E4F65
:1031B0000E9408B840E450E063EF78E0CE018E53FF
:1031C0009F4F0E9408B85ECFC901CE55DE4F0FB6A3
:1031D000F894DEBF0FBECDBFDF91CF911F910F914D
:1031E000FF90EF90DF90CF90BF90AF909F908F9027
:1031F0007F906F905F904F9008952F923F924F92E3
:103200005F926F927F928F929F92AF92BF92CF9276
:10321000DF92EF92FF920F931F93CF93DF93CDB77F
:10322000DEB7C55DD1090FB6F894DEBF0FBECDBFC6
:103230005C01C853DF4F0883C85CD040C753DF4FE1
:103240001883C95CD040822FC653DF4F2883CA5CE5
:10325000D040C553DF4F3883CB5CD040C453DF4FE1
:103260004883CC5CD040C353DF4F5883CD5CD04003
:10327000C253DF4F6883CE5CD040C153DF4F7883A9
:10328000CF5CD040C053DF4FF982E882C05DD040B0
:103290008F70C82ED12C2090FC083090FD08EE2DA8
:1032A000FF2D309719F08081811121C0D5011B9627
:1032B0008C91882341F0C5010B96C053DF4F998351
:1032C0008883C05DD040C114D10409F055C0C053FB
:1032D000DF4FE881F981C05DD040309761F4F5019E
:1032E000C588D688C114D10409F446C010C0C114E1
:1032F000D10409F041C08081882389F3CE01805335
:103300009F4F0E9425AE6C01892B49F335C0C653EF
:10331000DF4F8881CA5CD0408F7071F56C2DCE0173
:1033200088539F4F0E943435C854DF4F2883C85BB1
:10333000D040C754DF4F3883C95BD040C654DF4FFD
:103340004883CA5BD040C554DF4F5883CB5BD04025
:10335000C454DF4F6883CC5BD040C354DF4F7883C5
:10336000CD5BD040C254DF4F8883CE5BD040C15488
:10337000DF4F9883CF5BD0400E94A9942B013C0182
:103380008B01C053DF4FE880F980C05DD040D5018C
:10339000ED91FC91808091806EEB7BE086ED9BE06F
:1033A0000E945EA04AE050E0B20186ED9BE00E94E0
:1033B00015A067EB7BE086ED9BE00E945EA0B40168
:1033C00086ED9BE00E94A9A061EB7BE086ED9BE08F
:1033D0000E945EA0B70186ED9BE00E94A9A06BEA67
:1033E0007BE086ED9BE00E945EA068EA7BE086EDD4
:1033F0009BE00E945EA0043B11054CF46AE97BE06F
:103400008EE29BE00E945EA08EE29BE0AAC0CE010D
:1034100088539F4F0E94F233F50180819181892B5F
:1034200011F40C948323C5010E9459454C0191E08D
:1034300080E0181419040CF090E0692E782E5524C1
:103440005394161417040CF0512C86ED9BE00E9447
:10345000A351D50118968C91873009F486C0C053CA
:10346000DF4FE880F980C05DD040E114F10409F439
:103470005AC062EA7EE0C7010E94D1B7892BD9F118
:103480006EE97EE0C7010E94D1B7892BB9F16FECDC
:103490007AE0C7010E94D1B7892B99F16BEC7AE0F1
:1034A000C7010E94D1B7892B79F167E67EE0C70199
:1034B0000E94D1B7892B59F162E67EE0C7010E94D4
:1034C000D1B7892B39F16CE67EE0C7010E94D1B7F4
:1034D000892B19F162EC7AE0C7010E94D1B7892BE0
:1034E000F9F06EEB7AE0C7010E94D1B7892BD9F4CD
:1034F0000EE010E01AC001E010E017C002E010E09A
:1035000014C005E010E011C006E010E00EC00AE0B3
:1035100010E00BC00BE010E008C00CE010E005C0AC
:103520000DE010E002C000E010E0C5010E9437B0DD
:1035300090E0009709F03C0101151105B1F060160B
:10354000710699F064E87BE086ED9BE00E945EA046
:103550004AE050E0B30186ED9BE00E9415A086EDA5
:103560009BE00E94A3510C948323C054DF4F188228
:1035700019821A821B82C05CD040CC53DF4F188264
:1035800019821A821B82C45CD040CE53DF4F8881DF
:10359000C25CD0408F70CE53DF4F8883C25CD04076
:1035A000C054DF4F1882C05CD04040E0B501CE016E
:1035B00080549F4F0E949D34811182C067E67BE05A
:1035C00086ED9BE00E945EA0F501818592850097C3
:1035D00041F0DC01ED91FC91028CF38DE02D199509
:1035E00003C0F501808590E08D30910528F4FC0141
:1035F000EA53FC4F808101C080E08F70282F229514
:10360000207FCE53DF4F9881C25CD0409F70922BB9
:10361000CE53DF4F9883C25CD040843028F4823090
:10362000C8F4813069F133C0883039F0893079F5D8
:1036300080E090E0A6E9B2E404C080E090E0A0EA77
:10364000B1E4CC53DF4F88839983AA83BB83C45CE6
:10365000D04025C084E6CA53DF4F8883C65CD04083
:10366000C953DF4F8881C75CD0408E7FC953DF4F7D
:103670008883C75CD040CB53DF4F1882C55CD040F5
:103680008FEFCC53DF4F8883C45CD04008C0CC534D
:10369000DF4F188219821A821B82C45CD04040E03E
:1036A000B501CE0180549F4F0E944534CE01805415
:1036B0009F4F0E94F23360E07AE0C5010E94703FA4
:1036C000C853DF4F6881C85CD040643089F038F45B
:1036D000662309F457C3633009F49DC0BEC4673044
:1036E00009F41AC108F4B9C46A3008F475C1B5C444
:1036F000181419047CF562E0CE0180549F4F0E949B
:103700005C35C055DF4F2883C05BD040CF54DF4FBE
:103710003883C15BD040CE54DF4F4883C25BD0407A
:10372000CD54DF4F5883C35BD040CC54DF4F688308
:10373000C45BD040CB54DF4F7883C55BD040CA54C4
:10374000DF4F8883C65BD040C954DF4F9883C75B87
:10375000D0402EC061E0CE0180549F4F0E945C3566
:10376000C855DF4F2883C85AD040C755DF4F38832C
:10377000C95AD040C655DF4F4883CA5AD040C555B4
:10378000DF4F5883CB5AD040C455DF4F6883CC5AA3
:10379000D040C355DF4F7883CD5AD040C255DF4F5C
:1037A0008883CE5AD040C155DF4F9883CF5AD0403E
:1037B000C054DF4F6881C05CD040CE0188539F4F1A
:1037C0000E945C35C056DF4F2883C05AD040CF5589
:1037D000DF4F3883C15AD040CE55DF4F4883C25A9D
:1037E000D040CD55DF4F5883C35AD040CC55DF4F22
:1037F0006883C45AD040CB55DF4F7883C55AD04038
:10380000CA55DF4F8883C65AD040C955DF4F9883C9
:10381000C75AD0403DC4D50118968C91873009F421
:1038200039C4C5010E9437B0082F10E0853009F077
:103830006CC768E57BE086ED9BE00E945EA04AE0F5
:1038400050E0B80186ED9BE00E9415A086ED9BE05C
:103850000E94A351F5018085853079F56CE0CE0199
:1038600080549F4F0E945C35C856DF4F2883C8594B
:10387000D040C756DF4F3883C959D040C656DF4FB6
:103880004883CA59D040C556DF4F5883CB59D040E2
:10389000C456DF4F6883CC59D040C356DF4F78837E
:1038A000CD59D040C256DF4F8883CE59D040C15643
:1038B000DF4F9883CF59D040EBC361E0CE018054F5
:1038C0009F4F0E945C35C057DF4F2883C059D040BE
:1038D000CF56DF4F3883C159D040CE56DF4F488393
:1038E000C259D040CD56DF4F5883C359D040CC5633
:1038F000DF4F6883C459D040CB56DF4F7883C5591A
:10390000D040CA56DF4F8883C659D040C956DF4FD2
:103910009883C759D040BCC3D50118968C91873085
:1039200009F4B8C3C5010E9437B0082F10E08630F3
:1039300009F040C067E47BE086ED9BE00E945EA05A
:103940004AE050E0B80186ED9BE00E9415A086EDAC
:103950009BE00E94A35162E0CE0180549F4F0E94E1
:103960005C35C857DF4F2883C858D040C757DF4F52
:103970003883C958D040C657DF4F4883CA58D04013
:10398000C557DF4F5883CB58D040C457DF4F6883AB
:10399000CC58D040C357DF4F7883CD58D040C25762
:1039A000DF4F8883CE58D040C157DF4F9883CF5820
:1039B000D0406EC36FE27BE086ED9BE00E945EA08C
:1039C0004AE050E0B80186ED9BE00E9415A086ED2C
:1039D0009BE00E94A35199C660E0CE0180549F4FA6
:1039E0000E945C35C058DF4F2883C058D040CF5765
:1039F000DF4F3883C158D040CE57DF4F4883C2587D
:103A0000D040CD57DF4F5883C358D040CC57DF4FFD
:103A10006883C458D040CB57DF4F7883C558D04017
:103A2000CA57DF4F8883C658D040C957DF4F9883A5
:103A3000C758D040C653DF4F8881CA5CD040807FD2
:103A400041F0CE0188539F4F0E9453378B01672B63
:103A500011F405E010E0C853DF4F8881C85CD04006
:103A6000893019F4119501951109B2E0CB16D104F2
:103A700099F03CF4C114D10409F00CC355245394BB
:103A80000BC0F9E0CF16D10409F49EC02AE0C2169B
:103A9000D10409F413C1FEC2CE53DF4F8881C25C4A
:103AA000D040E82FE295EF708E2F90E0FC01319727
:103AB000EB30F10508F0EEC28827EA56FF4F8F4F32
:103AC0000C94DEBFCC53DF4F8881C45CD040080F1C
:103AD000111D0F3F110509F02CF417FF05C000E080
:103AE00010E002C00FEF10E0CC53DF4F0883C45C3E
:103AF000D040A6C2CC53DF4F68817981C45CD040EE
:103B0000060F171F053611052CF417FF05C000E03E
:103B100010E002C004E610E0012E000C220B330B73
:103B2000CC53DF4F088319832A833B83C45CD04086
:103B300087C2CC53DF4F688179818A819B81C45CC5
:103B4000D0400E94F4C0600F711F653671052CF4DF
:103B500077FF05C060E070E002C064E670E0072E09
:103B6000000C880B990B0E942CC1CC53DF4F68834B
:103B700079838A839B83C45CD04062C2CC53DF4F7D
:103B800088819981C45CD0404AE0409F9001419F68
:103B9000300D1124820F931F893EA3E09A072CF465
:103BA00097FF05C080E090E002C088EE93E0092E08
:103BB000000CAA0BBB0BCC53DF4F88839983AA83DD
:103BC000BB83C45CD0403CC2CE0188539F4F0E944F
:103BD0008B37882301F162E0CE0180549F4F0E9411
:103BE000C935E9962FAFE997EA963FAFEA97EB968A
:103BF0004FAFEB97EC965FAFEC97ED966FAFED970D
:103C0000EE967FAFEE97EF968FAFEF97C158DF4FED
:103C10009883CF57D040CE53DF4F8881C25CD040CD
:103C200082958F70823009F035C2CA53DF4F6881A8
:103C3000C65CD040C953DF4F8881C75CD040782F25
:103C40007170060F171F0E36B1E01B072CF417FF1B
:103C500005C00DE611E002C000E010E0CA53DF4FDE
:103C60000883C65CD040C953DF4F8881C75CD04011
:103C700010FB80F9C953DF4F8883C75CD04062E0F6
:103C8000CE0180549F4F0E943435E1962FAFE197CB
:103C9000E2963FAFE297E3964FAFE397E4965FAFCC
:103CA000E497E5966FAFE597E6967FAFE697E796E0
:103CB0008FAFE797E8969FAFE897C2C1CE018853D0
:103CC0009F4F0E948B378823F1F062E0CE01805431
:103CD0009F4F0E94C935A9962FAFA997AA963FAFCB
:103CE000AA97AB964FAFAB97AC965FAFAC97AD963C
:103CF0006FAFAD97AE967FAFAE97AF968FAFAF97E2
:103D0000E0969FAFE097CE53DF4F8881C25CD040F2
:103D100082958F70823009F0BDC1CB53DF4F88810F
:103D2000C55CD040080F111D053611052CF417FF96
:103D300005C000E010E002C004E610E0CB53DF4F06
:103D40000883C55CD04062E0CE0180549F4F0E9442
:103D50003435A1962FAFA197A2963FAFA297A39615
:103D60004FAFA397A4965FAFA497A5966FAFA59703
:103D7000A6967FAFA697A7968FAFA797A8969FAF57
:103D8000A8975EC1C653DF4F8881CA5CD040807F50
:103D900009F480C1E9E0CE16D10409F424C14CF441
:103DA000C114D104F1F022E0C216D10409F45FC0BD
:103DB00071C18BE0C816D10409F437C10CF4D0C02E
:103DC000BCE0CB16D10409F065C188E0FE01E853E0
:103DD000FF4FDE01A054BF4F01900D928A95E1F78D
:103DE00059C1181419043CF5CE0188539F4F0E9405
:103DF0005337672B682B692B59F562E0CE0180544D
:103E00009F4F0E945C3569962FAF69976A963FAFC6
:103E10006A976B964FAF6B976C965FAF6C976D968A
:103E20006FAF6D976E967FAF6E976F968FAF6F97F0
:103E3000A0969FAFA0971814190454F0CE01885390
:103E40009F4F0E945337672B682B692B09F063C47F
:103E5000C054DF4F6881C05CD040C5010E940CB0E7
:103E600060E079E0C5010E94703F55245394CE5321
:103E7000DF4F8881C25CD040982F92959F70945FED
:103E80009F70923050F4C653DF4F9881CA5CD04087
:103E900092959F70923009F45DC4F501108517303A
:103EA00039F4CE0188539F4F0E948B3781115AC439
:103EB000D50119968D919C911A97009741F0DC01DC
:103EC000ED91FC91028CF38DE02D199502C0812FAC
:103ED00090E07C01C853DF4F0881C85CD040C753D5
:103EE000DF4F1881C95CD040C653DF4F2881CA5CC0
:103EF000D040C553DF4F3881CB5CD040C453DF4F37
:103F00004881CC5CD040C353DF4F5881CD5CD0405A
:103F1000C253DF4F6881CE5CD040C153DF4F788100
:103F2000CF5CD040CE0180549F4F0E942C782996C0
:103F30002FAF29972A963FAF2A972B964FAF2B97F3
:103F40002C965FAF2C972D966FAF2D972E967FAF47
:103F50002E972F968FAF2F9760969FAF609770C068
:103F6000C353DF4F9881CD5CD040CE53DF4F888163
:103F7000C25CD040282F22952F7019F0223041F0DA
:103F800089C08F708062CE53DF4F8883C25CD0407F
:103F9000892F90E08536910514F084E690E0CB53AC
:103FA000DF4F8883C55CD04062E0CE0180549F4FD4
:103FB0000E94343521962FAF219722963FAF22974A
:103FC00023964FAF239724965FAF249725966FAF24
:103FD000259726967FAF269727968FAF2797289607
:103FE0009FAF28972DC0C253DF4F6881CE5CD04071
:103FF000C153DF4F7881CF5CD0407170CE018054C7
:104000009F4F0E942672882309F444C062E0CE01CB
:1040100080549F4F0E94343528AF39AF4AAF5BAF11
:104020006CAF7DAF8EAF9FAF0BC0CE0188539F4F5B
:104030000E94D277BC01CE0180549F4F0E94F4773A
:1040400040E0B501CE0180549F4F0E94453460E0AE
:104050007AE0C5010E94703F1DC0CE0180549F4F81
:104060000E945C3528AB39AB4AAB5BAB6CAB7DAB2C
:104070008EAB9FAB6C2DCE0180549F4F0E94343588
:1040800028A739A74AA75BA76CA77DA78EA79FA7DC
:1040900055245394F501618472846114710409F408
:1040A0003CC1C853DF4F8881C85CD04090E08A3063
:1040B000910508F0DCC0FC018827EF55FF4F8F4FBA
:1040C0000C94DEBF1814190454F162E27BE086ED13
:1040D0009BE00E945EA0D5011996ED91FC911A9784
:1040E0000190F081E02D84889588C053DF4FE880EF
:1040F000F980C05DD04061E0CE0180549F4F0E94A6
:104100005C35CC24C39489019A01AB01BC01F50153
:1041100081859285F40119958C0166E05BC062E1AE
:104120007BE063C0181419043CF5D301ED91FC91B8
:1041300084889588C053DF4FE880F980C05DD04007
:1041400062E0CE0180549F4F0E945C35CC24C39422
:1041500089019A01AB01BC01F50181859285F401C9
:1041600019958C0165E0C5010E940CB060E071E01A
:10417000C5010E94703FCFC060E07BE036C0C50142
:104180000E9437B0853079F1D301ED91FC9184889C
:104190009588C053DF4FE880F980C05DD04062E071
:1041A000CE0180549F4F0E945C3529833A834B8314
:1041B0005C836D837E838F839887CC24C39489012D
:1041C0009A01AB01BC01F50181859285F401199535
:1041D0008C0162E0C5010E940CB060E071E0C50195
:1041E0000E94703F87C060EF7AE086ED9BE00E94FE
:1041F0005EA08BC2C053DF4FE880F980C05DD04025
:10420000D301ED91FC910488F589E02DC52CC054B3
:10421000DF4F0881C05CD040CF53DF4F1881C15CB5
:10422000D040CE53DF4F2881C25CD040CD53DF4F0A
:104230003881C35CD040CC53DF4F4881C45CD04050
:10424000CB53DF4F5881C55CD040CA53DF4F6881E4
:10425000C65CD040C953DF4F7881C75CD040C301F2
:1042600019958C0147C0181419040CF441C0C053AF
:10427000DF4FE880F980C05DD040D301ED91FC9123
:104280000488F589E02DCC24C394C054DF4F088105
:10429000C05CD040CF53DF4F1881C15CD040CE53BB
:1042A000DF4F2881C25CD040CD53DF4F3881C35CE3
:1042B000D040CC53DF4F4881C45CD040CB53DF4F5C
:1042C0005881C55CD040CA53DF4F6881C65CD0407E
:1042D000C953DF4F7881C75CD040C30119958C0169
:1042E000C054DF4F6881C05CD040662319F072CFA4
:1042F0000FEF1FEF64EE7AE086ED9BE00E945EA078
:104300004AE050E0B80186ED9BE00E9415A086EDE2
:104310009BE00E94A351C80132C2F501808586301E
:1043200009F475C038F4843009F447C1853009F4C4
:10433000D6C0CEC1883009F49EC120F0893009F47E
:104340006BC1C6C10280F381E02D80858F708530FE
:1043500009F0BEC1B5E02B16310409F4B9C1C6801D
:10436000D78080913A0D8F5F80933A0DC114D104AC
:1043700009F447C0F60180858F708430E1F56185CE
:104380007285CE0101960E94F2B0C053DF4FE880E3
:10439000F980C05DD040C853DF4F0881C85CD04071
:1043A000C753DF4F1881C95CD040C653DF4F288107
:1043B000CA5CD040C553DF4F3881CB5CD040C4537A
:1043C000DF4F4881CC5CD040C353DF4F5881CD5C78
:1043D000D040C253DF4F6881CE5CD040C153DF4F25
:1043E0007881CF5CD040CE0101960E94FD18CE01AD
:1043F00001960E9444B0D6011296CD90DC9013979E
:10440000B5CF80913A0D815080933A0D61C160E043
:1044100070E0C5010E9422AF8C01009709F458C1D9
:1044200097FF07C011950195110966246394712CBB
:1044300002C0612C712CC80101978634910508F0E7
:1044400047C1C054DF4FE880C05CD040F12CD02E73
:1044500061E0802F0E94014D672869F0B1E0EB1602
:10446000F10429F061E0E6E0EE16F10409F460E001
:10447000E62EF12C12C0F1E0EF16F10451F091E0BC
:1044800080E026E0E216F10409F090E0E92EF82E33
:1044900003C0EE24E394F12C6E2D8D2D0E94D24C9E
:1044A0006FED7AE086ED9BE00E945EA04AE050E06E
:1044B000B80186ED9BE00E9415A06DED7AE086EDD7
:1044C0009BE00E945EA04AE050E0B70186ED9BE0D1
:1044D0000E9415A086ED9BE00E94A351F9C082E0E6
:1044E000C816D10409F461C0ACE0CA16D10409F0C1
:1044F000EFC0C5010E9407AF6B017C01EF2849F4B2
:10450000D501ED91FC91608171818AEA94E00E946D
:104510000A72CE0180549F4F0E94153720E030E090
:1045200048EC52E40E94E1C10E94F4C0CE52DF4F39
:10453000688379838A839B83C25DD040CE52DF4FEC
:10454000C880D980C25DD04088E00E94EC922B01E7
:104550003C017B0169ED7AE086ED9BE00E945EA064
:104560004AE050E0CE52DF4F68817981C25DD04091
:1045700086ED9BE00E9415A064ED7AE086ED9BE05D
:104580000E945EA0B301A201662777272AE086ED8C
:104590009BE00E945A5186ED9BE00E94A351B70117
:1045A000A601C5010E94A9AE93C040E0B501CE01AD
:1045B00080549F4F0E9445348BC0552009F488C019
:1045C000C054DF4F0881C05CD040CF53DF4F18810B
:1045D000C15CD040CE53DF4F2881C25CD040CD5368
:1045E000DF4F3881C35CD040CC53DF4F4881C45C7F
:1045F000D040CB53DF4F5881C55CD040CA53DF4F0A
:104600006881C65CD040C953DF4F7881C75CD04019
:10461000C5010E9474435CC0552009F459C0C054C0
:10462000DF4F0881C05CD040CF53DF4F1881C15CA1
:10463000D040CE53DF4F2881C25CD040CD53DF4FF6
:104640003881C35CD040CC53DF4F4881C45CD0403C
:10465000CB53DF4F5881C55CD040CA53DF4F6881D0
:10466000C65CD040C953DF4F7881C75CD040C501DC
:104670000E94A4422DC0552059F1C054DF4F08813B
:10468000C05CD040CF53DF4F1881C15CD040CE53C7
:10469000DF4F2881C25CD040CD53DF4F3881C35CEF
:1046A000D040CC53DF4F4881C45CD040CB53DF4F68
:1046B0005881C55CD040CA53DF4F6881C65CD0408A
:1046C000C953DF4F7881C75CD040C5010E94424486
:1046D000C054DF4F6881C05CD0406623C9F0C85326
:1046E000DF4F8881C85CD040853021F4181419044C
:1046F0007CF465E0C5010E940CB060E071E0C5018A
:104700000E94703F05C08FEF01C08DEF9FEF37C053
:1047100081E090E034C061E0CE0180549F4F0E9460
:104720005C3561962FAF619762963FAF6297639653
:104730004FAF639764965FAF649765966FAF659769
:1047400066967FAF669767968FAF679768969FAFBD
:1047500068977ECB8F708062CE53DF4F8883C25CB8
:10476000D0409BCBCE53DF4F9881C25CD0409F702E
:104770009062CE53DF4F9883C25CD04099CBCB522E
:10478000DF4F0FB6F894DEBF0FBECDBFDF91CF91E4
:104790001F910F91FF90EF90DF90CF90BF90AF905F
:1047A0009F908F907F906F905F904F903F902F9051
:1047B00008958F929F92AF92BF92CF92DF92EF9225
:1047C000FF920F931F93CF93DF9300D000D0CDB70C
:1047D000DEB780907807909079078114910409F4EE
:1047E000B8C080913A0D8F5F80933A0D0E94844E3D
:1047F0009B01AC01609180077091810780918207D5
:1048000090918307AA24AA94BA2C65011FE0E12E97
:10481000F12C00E010E00E940293882309F456C0B6
:10482000F401068117810115110509F441C0F80151
:1048300080858F708630C1F569EB74E0C8010E94F5
:10484000EC5E0097F9F0FC0120852F702530D1F443
:10485000E680F780E114F10439F1FA82E982B801C7
:10486000CE0101960E94A45D8D819E81892B31F03D
:1048700062E070E0CE0101960E944460F701E280A0
:10488000F380E8CF1A83098360E070E0CE010196DF
:104890000E94A45D8D819E81892B31F062E070E0E1
:1048A000CE0101960E944460F80102811381BBCFC2
:1048B0000E94844E609380077093810780938207E3
:1048C0009093830710921D0C10921E0C0E94844E30
:1048D0009B01AC0160917C0770917D0780917E0700
:1048E00090917F07AA24AA94BA2C650118E8E12EBA
:1048F00013E1F12E00E010E00E940293882321F1E1
:10490000E0917807F091790706811781011511056B
:1049100089F0F80180858F70863041F41A8309830D
:1049200060E070E0CE0101960E94A45DF801028172
:104930001381ECCF0E94844E60937C0770937D07B7
:1049400080937E0790937F0780913A0D81508093EA
:104950003A0D26960FB6F894DEBF0FBECDBFDF919D
:10496000CF911F910F91FF90EF90DF90CF90BF906C
:10497000AF909F908F9008952F923F924F925F92A9
:104980006F927F929F92AF92BF92CF92DF92EF92FF
:10499000FF920F931F93CF93DF93CDB7DEB7CE5522
:1049A000D1090FB6F894DEBF0FBECDBF80913A0D8E
:1049B0008F5F80933A0DE091FE08F091FF083097E9
:1049C000B9F006811781E090FE08F090FF08E1142D
:1049D000F10471F00115110559F0F80180858F700F
:1049E0008530A9F7C8010E9425AA823080F3E7C16B
:1049F00080913A0D815080933A0D8091FC089091FE
:104A0000FD08059709F439C50E94844E9B01AC014D
:104A10006091840770918507809186079091870740
:104A2000AA24AA94BA2C650118EEE12E13E0F12E07
:104A300000E010E00E940293882309F41EC510E0F4
:104A4000CC24C394D12C54E0252E312CE0917A074C
:104A5000F0917B07309709F410C511110EC58085C0
:104A60008F70853009F090C1F9AFE8AF23961FAE83
:104A70001EAE2397CE01C8960E9453B021968FADEB
:104A80002197883009F434C1893009F440C084305A
:104A900009F069C180910F0990911009892B09F0E3
:104AA00022C160E074E0CE01C8960E94F5AF892B68
:104AB00009F46AC019821A821B821C821D821E821E
:104AC0001F8218868B818F708B83198241E0BE0113
:104AD000685C7F4FCE0101960E949D3463EC7BE0C1
:104AE00086ED9BE00E945EA060E074E0CE01C89677
:104AF0000E9483AF09811A812B813C814D815E81A7
:104B00006F817885CE01C8960E947443ECC0809175
:104B10000F0990911009892B09F0E5C060E074E05D
:104B2000CE01C8960E94F5AF892B09F4F3C1198212
:104B30001A821B821C821D821E821F8218868B8114
:104B40008F708B83198241E0BE01685C7F4FCE017C
:104B500001960E949D3465E27CE086ED9BE00E9418
:104B60005EA060E074E0CE01C8960E9483AF098128
:104B70001A812B813C814D815E816F817885CE01C8
:104B8000C8960E94A442AFC0EAACFBACF701808596
:104B90008F70853009F02FC1C7010E9425AAA82E69
:104BA000B12CF2E0AF16B1040CF425C1D09210097B
:104BB000C0920F0960E070E0CE01C8960E9422AF5B
:104BC0003C0161E070E0CE01C8960E9422AF8C01EA
:104BD000F5E0AF16B1040CF47CC164E0C7010E949B
:104BE000A4A9FC01E184F28426E240E855E260E0F9
:104BF00070E08EE199E00E9446AD6092060A8EE177
:104C000099E09093050A8093040A1092110B109278
:104C1000130B1092120BF1E0EF16F10409F40CC122
:104C20000CF4F0C092E0E916F10409F0F7C010931B
:104C3000080A0093070AD0920A0AC092090A83E080
:104C40000E948FAA982E911028C1E0900B0AF09034
:104C50000C0AC7010F2C000CAA0BBB0B89839A838B
:104C6000AB83BC8380E190E09E838D83E8ADF9AD9A
:104C7000A080B18065EF7BE086ED9BE00E945EA0A6
:104C8000B50186ED9BE00E94A9A06EEE7BE086ED6B
:104C90009BE00E945EA0BE016F5F7F4F86ED9BE0B0
:104CA0000E9478B10E94A351B701CE01C8960E941C
:104CB000C941A0907A07B0907B07F501828193816A
:104CC0009A8389831B861A86CE0101960E9453B06F
:104CD000AB2809F0C2C0CE0101960E9444B01092E8
:104CE000100910920F09CE01C8960E94AB41B9C3BA
:104CF00080910F0990911009892BA9F760E074E069
:104D0000CE01C8960E94F5AF892B69F319821A82E9
:104D10001B821C821D821E821F8218868B818F70CF
:104D20008B83198241E0BE01685C7F4FCE01019602
:104D30000E949D346AE77CE086ED9BE00E945EA0C5
:104D400060E074E0CE01C8960E9483AF09811A81A9
:104D50002B813C814D815E816F817885CE01C89623
:104D60000E944244C0CFCE01C8960E94AB4161E090
:104D700070E0CE01C8960E940A76892B09F071C3B3
:104D8000CE01C8960E9444B0E0917A07F0917B076B
:104D9000309709F472C38281938190937B0780934B
:104DA0007A07892B09F052CEE091FE08F091FF08B6
:104DB0008681978190937B0780937A075EC31A83DD
:104DC00009831B861A86CE0101960E9453B0CE013C
:104DD00001960E945BAE882331F062E070E0CE0164
:104DE00001960E940A76F80102811381CE01019694
:104DF0000E9444B0E8CD62E17CE086ED9BE00E9439
:104E00005EA071CFEF2811F51093080A0093070AEE
:104E1000D0920A0AC092090A81E012CFE3E0EE16AE
:104E2000F104A1F41093080A0093070AD0920A0A29
:104E3000C092090A84E004CF1093080A0093070A7D
:104E4000F0920A0AE092090A82E0FACE6AEF7BE069
:104E500086ED9BE00E945EA0F6CECE0101960E94F8
:104E60005BAE882309F437CF8985843009F033CFCE
:104E700060E070E0CE0101960E9422AF68167906CC
:104E800009F029CF61E070E0CE0101960E9422AFC7
:104E90000817190709F01FCF20C0892D90E0A0E066
:104EA000B0E089839A83AB83BC8380E190E09E83EA
:104EB0008D8368ED7BE086ED9BE00E945EA0BE01E5
:104EC0006F5F7F4F86ED9BE00E9478B10E94A351F7
:104ED00006CF82E0E82EF12C87CEB701CE010196F5
:104EE0000E94C941E0917A07F0917B07828193810A
:104EF00090937B0780937A07892B09F0ECCEE091A1
:104F0000FE08F091FF088681978190937B0780933C
:104F10007A07E1CED0921009C0920F090E94D63DC7
:104F20005C01892B29F0F5018085807F8660808770
:104F300020E030E043E050E060E2CE0101960E94C4
:104F4000B893E8ADF9AD608171814FE150E0CE01D9
:104F500001960E9495C46DEB74E0CE0101960E940B
:104F60006FC426E040E855E260E070E08EE199E031
:104F70000E9446AD60E070E0CE01C8960E9422AF6C
:104F80008093060A8EE199E09093050A8093040AC3
:104F90001092110B1092130B1092120B84E398E0F5
:104FA0009093080A8093070AEAE0F0E0F0930A0A77
:104FB000E093090A83E00E948FAA8111F1C060E7A3
:104FC0007CE086ED9BE00E945EA02BE0622E2AE052
:104FD000722E0FE11AE030E1E32EF12CF301819102
:104FE00091913F01092E000CAA0BBB0B89A39AA338
:104FF000ABA3BCA3FEA2EDA2BE016F5D7F4F86ED09
:105000009BE00E9478B16EE67CE00E945EA00615EF
:10501000170521F786ED9BE00E94A35160910F0ACE
:105020007091100A80E090E00E942CC120E030E0F6
:1050300048EC52E40E9482C09B01AC0163EC74E036
:10504000C5010E9495768091130A9091140A2C0153
:10505000612C712CA301920165EC74E0C5010E94E2
:1050600050AA6091150A7091160A80E090E00E94A3
:105070002CC120E030E048EC52E40E9482C09B0149
:10508000AC0169EC74E0C5010E9495766091170A45
:105090007091180A80E090E00E942CC120E030E07E
:1050A00040E251E40E9482C09B01AC0167EC74E0D5
:1050B000C5010E94957620910B0A30910C0A40E0C0
:1050C00050E06BEC74E0C5010E9450AA45284628C8
:1050D000472809F47FC0EAADFBAD90859F709530FD
:1050E00009F078C061E0CF010E94A4A9009709F4FB
:1050F00071C0FC0120852F70243009F06BC06185E0
:105100007285CE0181960E94F2B0CE0181960E94F6
:105110005BAE882309F43FC063961CAE1DAE1EAE85
:105120001FAE639767961CAE1DAE1EAE1FAE67978F
:1051300062968FAD62978F7062968FAF629760961E
:105140001FAE609764E670E0CE01815B9F4F0E94C6
:10515000803568962FAF689769963FAF69976A96D2
:105160004FAF6A976B965FAF6B976C966FAF6C970C
:105170006D967FAF6D976E968FAF6E976F969FAF60
:105180006F97E12CF12C89019A01AB01BC01CE0192
:1051900081960E94FD18CE0181960E9444B01AC0EB
:1051A00090E0A0E0B0E089A39AA3ABA3BCA380E108
:1051B00090E09EA38DA368E57CE086ED9BE00E94D5
:1051C0005EA0BE016F5D7F4F86ED9BE00E9478B1CF
:1051D0000E94A35180910B0A83FF2EC08EE398E0BA
:1051E0009093080A8093070AD0920A0AC092090A8B
:1051F00083E00E948FAA81110BC020910B0A30918D
:105200000C0A40E050E06EEC74E0C5010E9450AA28
:105210001092100910920F09CE01C8960E945945AC
:105220001816190624F4CE01C8960E943376D0923F
:105230001009C0920F0908C020E030E0A9016EEC0F
:1052400074E0C5010E9450AA62E370E080E090E043
:105250000E944A4E83E190E09093080A8093070AE7
:1052600030920A0A2092090A83E00E948FAA8111D3
:10527000A0C06EE47CE086ED9BE00E945EA09BE017
:10528000E92E9AE0F92E03E11AE0F701619171919C
:105290007F014AE050E086ED9BE00E9415A06CE49F
:1052A0007CE086ED9BE00E945EA00E151F0569F76D
:1052B00086ED9BE00E94A35100910B0A10910C0A0D
:1052C00001151105D1F0B801012E000C880B990BC6
:1052D0000E942CC12DEE3EE94CE35EE30E94E1C149
:1052E00022E538EB42E152E40E9410C09B01AC0180
:1052F00062ED74E0C5010E94957660910D0A70918F
:105300000E0A072E000C880B990B0E942CC12DEE63
:105310003EE94CE35EE30E94E1C122E538EB42E165
:1053200052E40E9410C02B013C019B01AC0161ECD6
:1053300074E0C5010E9495766091110A7091120A7D
:1053400016161706A4F4072E000C880B990B0E9462
:105350002CC120E030E040E251E40E9482C09B0179
:10536000AC0166ED74E0C5010E94957608C020E0AE
:1053700030E0A90166ED74E0C5010E9450AA20E06A
:1053800030E040E252E4C301B2010E94DCC11816D1
:1053900044F5012B31F10E9466A8882329F0809101
:1053A000390D882309F44EC0CE01C8960E94337689
:1053B00018C090E0A0E0B0E089A39AA3ABA3BCA37F
:1053C00080E190E09EA38DA366E37CE086ED9BE008
:1053D0000E945EA0BE016F5D7F4F86ED9BE00E9444
:1053E00078B180E091E00E94E7B58C01892BD9F07B
:1053F0001CA21BA21EA21DA28FEF9FEF98A78FA336
:105400008DE392E09AA389A31AA619A61CA70BA75D
:1054100080E091E098AB8FA71EA61DA6B501CE0136
:1054200081960E94D63B0E9466A8882321F0809135
:10543000390D882381F0C8010E947FB6C5010E9402
:1054400063764DCCE8ADF9AD608171818AED94E071
:105450000E940A72A9CFB801CE0101960E940A7279
:10546000EACF0E94844E60938407709385078093EF
:1054700086079093870711E083CCC25ADF4F0FB69F
:10548000F894DEBF0FBECDBFDF91CF911F910F917A
:10549000FF90EF90DF90CF90BF90AF909F907F9064
:1054A0006F905F904F903F902F900895DC0116967B
:1054B0008D919C911797009739F0DC01ED91FC914B
:1054C0000680F781E02D19940895089580E090E01A
:1054D0000895809191079091920708954F925F925D
:1054E0006F927F92BF92CF92DF92EF92FF920F93D3
:1054F0001F93CF93DF9300D000D0CDB7DEB77C01F0
:10550000B62E80919007882309F475C08091EB072F
:105510009091EC072AE062135DC0FC01E556F84F5C
:105520001082D70118960D911C911997011511053C
:1055300009F44BC0F801618572856115710589F424
:1055400045805680678070848091BD099091BE0926
:10555000A091BF09B091C009481659066A067B069A
:10556000A1F1D8011B964D915C911C9741155105F5
:1055700061F1F701C480D580D80153968C9190E0F9
:1055800096012770332702C0959587952A95E2F7F3
:1055900080FF1BC0C601887F9370892B39F4F80106
:1055A00081899289887F9370C82AD92AD8018D91E0
:1055B0009C91DC01ED91FC916115710569F1068802
:1055C000F789E02D19950197E9F11092EC071092F7
:1055D000EB0711C08F34910574F4BDE06B1759F0DF
:1055E0009C012F5F3F4F3093EC072093EB07FC01AA
:1055F000E556F84F6083F70186819781009749F05F
:10560000DC01ED91FC910190F081E02D6B2D19955D
:105610006CC081E090E069C00488F589E02D2EEB34
:1056200033E03A832983D80115964D905D906D90B3
:105630007C9018974B825C826D827E82BE016F5F88
:105640007F4FC0CF6CE3F801808191810E94C69F9B
:10565000A60160E070E02AE0D8018D919C910E9443
:105660005A51F801228180819181211103C06CE19E
:105670007DE002C06AE17DE00E945EA0D8011D9637
:105680006D917C911E978D919C910E94A9A060E2E2
:10569000F801808191810E94C69FD8011F966D916B
:1056A0007C9150978D919C910E94A9A0F801228134
:1056B00080819181211103C06FE07DE002C069E02B
:1056C0007DE00E945EA06BE977E0D8018D919C910E
:1056D0000E94A9A0F80180819181DC01ED91FC91EB
:1056E000008CF18DE02D199570CF26960FB6F894A9
:1056F000DEBF0FBECDBFDF91CF911F910F91FF9005
:10570000EF90DF90CF90BF907F906F905F904F9021
:1057100008950C947FB6AF92BF92CF92DF92EF9232
:10572000FF920F931F93CF93DF93CDB7DEB76897A8
:105730000FB6F894DEBF0FBECDBFFC01098B1A8BEC
:105740002B8B3C8B4D8B5E8B6F8B788F8281938103
:10575000009709F4A0C0248135812115310509F491
:105760009FC0CC2009F497C06F0160E070E00E94F8
:1057700022AF192FD601ED91FC91028CF38DE02D13
:10578000C60119955C0182309105D1F183309105F4
:1057900021F0019799F585E034C0612F661F6627D7
:1057A000661FCE0141960E9452365C01BC01D601B3
:1057B00014968C910E943D4DF601C480D58062EC18
:1057C0007CE086ED9BE00E945EA04AE050E0B601DE
:1057D00086ED9BE00E9415A060EC7CE086ED9BE0EE
:1057E0000E945EA04AE050E0B50186ED9BE00E9479
:1057F00015A086ED9BE00E94A35150C081E001C03E
:1058000084E019861A861B861C861D861E861F86C6
:10581000188A8295807F9B859F70892B8B8719863C
:10582000EE24EA94FE2C09891A892B893C894D893A
:105830005E896F89788DCE0109960E942C78F1E0FF
:10584000AF16B10429F082E0A816B10451F026C0C9
:1058500063E070E0C6010E94D75E688970E00E9434
:105860003D4D6F8570E0D60114968C910E943D4DA0
:1058700061E070E0C6010E94D75E6E8570E00E9414
:105880003D4D62E070E0C6010E94D75E6D8570E01C
:105890000E943D4D03C020E030E002C021E030E036
:1058A000C90168960FB6F894DEBF0FBECDBFDF9179
:1058B000CF911F910F91FF90EF90DF90CF90BF900D
:1058C000AF900895CF93DF93DC011296ED91FC9198
:1058D00013973097C1F1EC018E819F818330910540
:1058E00079F00497D1F467EB7CE086ED9BE00E94B1
:1058F0005EA086ED9BE00E94A35181E090E025C070
:105900006AEA7CE086ED9BE00E945EA086ED9BE06B
:105910000E94A35182E090E018C04AE050E0608508
:1059200086ED9BE00E94BF9F62EB7CE086ED9BE0F2
:105930000E945EA086ED9BE00E94A351EA81FB815C
:10594000808590E002C080E090E0DF91CF910895E3
:10595000CF93DF93EC016DE97CE086ED9BE00E9444
:105960005EA086ED9BE00E94A351E881F981028C44
:10597000F38DE02DCE0119958130910519F0029734
:1059800049F01BC063E070E0CE010E94D75E60E08A
:105990000E94014D60E08C810E94014D61E070E049
:1059A000CE010E94D75E60E00E94014D62E070E08F
:1059B000CE010E94D75E60E002C060E08C810E9450
:1059C000014D109292071092910781E090E0DF91D3
:1059D000CF910895CF93DF93EC010E94255B60E99E
:1059E0007CE086ED9BE00E945EA086ED9BE00E943D
:1059F000A3518A819B81892B09F44CC08C819D81A4
:105A0000892B09F047C0E881F981028CF38DE02DE4
:105A1000CE0119958130910519F0029749F01BC00C
:105A200063E070E0CE010E94D75E61E00E94014D0C
:105A300061E08C810E94014D61E070E0CE010E9426
:105A4000D75E61E00E94014D62E070E0CE010E94ED
:105A5000D75E61E002C061E08C810E94014D8091BF
:105A6000A100887F8093A10080919100887F80931E
:105A700091008091A10082608093A10080919100AB
:105A800082608093910081E090E0909392078093F0
:105A9000910702C080E090E0DF91CF9108952F92AE
:105AA0003F924F925F926F927F928F929F92AF92AE
:105AB000BF92CF92DF92EF92FF920F931F93CF93FB
:105AC000DF93CDB7DEB761970FB6F894DEBF0FBE98
:105AD000CDBF0E94844E9B01AC01609197077091ED
:105AE00098078091990790919A07AA24AA94BA2CB2
:105AF000650118E8E12E13E1F12E00E010E00E94AC
:105B00000293882309F46DC3E090FA08F090FB0833
:105B1000D70112968C91823089F46AEF7CE086ED91
:105B20009BE00E945EA086ED9BE00E94A3518091C5
:105B3000FA089091FB080E940A70E8C180919507CD
:105B400090919607892B09F067C083E190E00E944D
:105B5000E7B58C018FE39AE8F801928B818BF6828E
:105B6000E5821482108289E0818381E082838383CD
:105B700010939607009395070E94844E4B015C0199
:105B8000F0E18F0EF7E29F1EA11CB11CD801159603
:105B9000ED91FC9116978FEF83871486DF011396A2
:105BA0003B961D92EA17FB07E1F7F8011482DD240A
:105BB000D394BE01665F7F4FD80115968D919C915D
:105BC00016970E94DF70181644F40E94844E6815E0
:105BD00079058A059B0508F4A4C100E010E0E12CDA
:105BE000F12C20918E0730918F078091950790912D
:105BF0009607E216F30674F460918C0770918D0796
:105C0000600F711F0E94C4A6BFEFEB1AFB0A085F6A
:105C10001F4FE7CFFC011282809193079091940768
:105C200020918E0730918F07821793070CF46AC07A
:105C30000E94844E1B012C0160EF7CE089E39BE015
:105C40000E9482A0E091FA08F091FB08309751F091
:105C50008FEF83871486DF0113963B961D92AE1754
:105C6000BF07E1F7E0918807F091890780E090E0B5
:105C700020918E0730918F07821793073CF4208183
:105C800031812E7F219331930196F2CF6624639464
:105C9000712C8091FA089091FB08009709F482C258
:105CA00060918E0770918F0723E0660F771F2A950A
:105CB000E1F720918C0730918D07620F731F0E94CE
:105CC000DF7018160CF06EC280908E0790908F07D0
:105CD000F4E18F1691040CF065C20E94844E9B0182
:105CE000AC01AA24AA94BA2C650118E8E12E13E1AC
:105CF000F12E00E010E0C201B1010E940293811177
:105D000051C294C100918C0710918D079C0143E012
:105D1000220F331F4A95E1F7020F131FF80120816C
:105D2000283209F0EEC0AE014F5F5F4FB80180919D
:105D30009507909196070E949E70882369F12A81A9
:105D400030E0C901982F8827990F990F990F698121
:105D5000F8E06F9FB00111249C01262B372BD8014E
:105D60008C918031E1F4688570E08F81FB01E81B44
:105D7000F109CF019695982F8827979587950E94CE
:105D8000CABF60517109207F13E0220F331F1A959B
:105D9000E1F7620F731F04C060E874EE01C0B9013F
:105DA0006138F4EE7F077CF0072E000C880B990B0E
:105DB0000E942CC120E030E040E05CE30E94E1C1A1
:105DC0009B01AC0104C020E030E04EEF52ECE091CA
:105DD0008A07F0918B07309789F080919307909113
:105DE0009407BC01A3E0660F771FAA95E1F7A09185
:105DF0008C07B0918D076A0F7B1F1995009193074F
:105E00001091940743E0000F111F4A95E1F780912C
:105E10008C0790918D07080F191FE0909507F0905F
:105E20009607D8018C91803149F0B801C7010E94D2
:105E3000B170D82E882309F460C002C03CE0D32E94
:105E4000F701858196810E940A70882309F455C064
:105E5000B801D70115968D919C9116970E94C06F3D
:105E6000F701408164E4858196810E949E6FD7018D
:105E700012968C91882309F440C0E7EFED0DE330D2
:105E800040F4F0E0EE0FFF1FE951FD4F40805180DC
:105E900004C09EEE492E92E0592E0115110539F1EC
:105EA000F7018381882319F18081811120C00E942C
:105EB000844E4B015C01052C000C66087708AE018E
:105EC0004F5F5F4FB801C7010E94487089818111FF
:105ED00014C00E94844EDC01CB0184199509A609E7
:105EE000B70988159905AA05BB0548F306C0B20194
:105EF000550C880B990B0E944A4E80919307909104
:105F00009407019690939407809393070E94844E80
:105F100060939707709398078093990790939A07D7
:105F200060C167E0CE010A960E944D6F998989137E
:105F300073C063EC74E089E39BE00E94A9A0F801C0
:105F40008081811138C0858196810E940A70BE01CE
:105F5000665F7F4FD80115968D919C9116970E9490
:105F6000C06F40E064EBF801858196810E949E6FCE
:105F7000D8011596ED90FC901697C7010E945A6FB4
:105F8000C7010E94319067E88FEC99E00E94FF8F73
:105F900060E88FEC99E00E94FF8FC7010E942E906D
:105FA000C7010E945A6FF82EF801858196810E94E0
:105FB0000A70F5FE38C0AE014F5F5F4FBE01665FED
:105FC0007F4FC8010E944870D8011196FC908A85C5
:105FD000803109F401C1BE01665F7F4FC8010E9494
:105FE000B1708F1518F4F80181810BC08A8580315A
:105FF00011F48CE006C0BE01665F7F4FC8010E94AD
:10600000B170D80111968C93119714968C911497B6
:106010008F5F14968C93CDCD69EC74E089E39BE09F
:106020000E94A9A0C6CDD801DC92C5CFA0908C0754
:10603000B0908D07740183E0EE0CFF1C8A95E1F7A8
:10604000EA0CFB1C67E0C7010E944D6FF7019781C6
:1060500089131FCE00E010E008151905CCF548E0C3
:1060600050E0B701C5010E943DC428E0A20EB11C5A
:10607000892B59F5000F111FE0918807F0918907CE
:10608000E00FF11F8081918181609183808369EEAF
:106090007CE086ED9BE00E945EA080918E0790914F
:1060A0008F07A3E0880F991FAA95E1F720918C072D
:1060B00030918D07820F931F0E9446A762EE7CE00D
:1060C00086ED9BE00E9482A0E4CD0F5F1F4FC4CFFE
:1060D0008091950790919607892B09F4DACDE0918C
:1060E0008E07F0918F07EE0FFF1F80918807909128
:1060F0008907E80FF91F7182608200918E07109165
:106100008F076DED7CE086ED9BE00E945EA04AE08B
:1061100050E0B80186ED9BE00E9415A066ED7CE0A2
:1061200086ED9BE00E945EA080918E0790918F0784
:1061300063E0880F991F6A95E1F720918C073091F1
:106140008D07820F931F0E9446A786ED9BE00E9459
:10615000A35160918E0770918F07E3E0660F771F60
:10616000EA95E1F780918C0790918D07680F791F70
:10617000DB018C91883261F48091950790919607AC
:106180000E94C4A68091FA089091FB080E94769123
:1061900080918E0790918F07019690938F0780933F
:1061A0008E0777CD00918E0710918F0767EC7CE00A
:1061B00086ED9BE00E945EA04AE050E0B80186EDCB
:1061C0009BE00E9415A086ED9BE00E94A3511092D7
:1061D0009407109293079ACEFCE0FF1508F403CFC2
:1061E00008CF61960FB6F894DEBF0FBECDBFDF912A
:1061F000CF911F910F91FF90EF90DF90CF90BF90C4
:10620000AF909F908F907F906F905F904F903F9056
:106210002F900895FC01848195810895089580E070
:1062200090E00895009789F0FC0120852F702530BB
:1062300061F40E94A4A9009741F0FC0120852F7011
:10624000243019F481859285089580E090E00895C6
:10625000CF92DF92EF92FF920F931F93CF93DF9332
:1062600000D000D0CDB7DEB7809190078111A0C0DB
:106270008091FC089091FD0802970CF499C08091E0
:10628000290D90912A0D892B09F492C062E072E0E9
:1062900085EF9BE00E94368E69EE74E08091290DB7
:1062A00090912A0D0E94EC5E7C01009709F480C059
:1062B0000E9425AA082F10E00115110509F478C0E5
:1062C00060E070E0C7010E9412316C0101301105DD
:1062D00009F46BC061E0C7010E94A4A9FC0101851B
:1062E0001285CE0101960E94A8A7CE0101960E94B8
:1062F000D5A764ED7DE083E29BE00E945EA0B6013D
:1063000083E29BE00E94A9A060EF74E083E29BE03F
:106310000E94A9A04AE050E0B80183E29BE00E94FD
:1063200015A060EF74E083E29BE00E94A9A064EFF7
:106330007DE083E29BE00E94A9A083E29BE00E94B3
:10634000A351D092EB0BC092EA0B1093ED0B00938C
:10635000EC0B84EF9DE09093EF0B8093EE0B80911C
:10636000F3089091F408009741F060E070E00E941B
:1063700012319093360D8093350D8091350D9091AB
:10638000360D009721F09093F10B8093F00B109253
:10639000F30B1092F20B81E0809390076BEB7DE0A2
:1063A00083E29BE00E945EA003C002E012E099CF6E
:1063B00026960FB6F894DEBF0FBECDBFDF91CF910A
:1063C0001F910F91FF90EF90DF90CF900895DF9293
:1063D000EF92FF920F931F93CF93DF9300D000D0E3
:1063E000CDB7DEB766EB7DE083E29BE00E945EA066
:1063F0000AEC1CE0D12C80E1E82EF12CF801808120
:10640000803130F462EF74E083E29BE00E94A9A047
:10641000F8018081F5E090E0A0E0B0E089839A8304
:10642000AB83BC83FE82ED82BE016F5F7F4F83E250
:106430009BE0DF1639F00E9478B164EB7DE00E94AA
:106440005EA004C00E9478B10E94A351D3940F5F54
:106450001F4F86E0D812D2CF26960FB6F894DEBF33
:106460000FBECDBFDF91CF911F910F91FF90EF90A5
:10647000DF9008954F925F926F927F928F929F92DA
:10648000AF92BF92CF92DF92EF92FF920F931F9342
:10649000CF93DF9300D000D0CDB7DEB75C017E8311
:1064A0006D837A0149016115710509F45AC14115DD
:1064B000510509F456C1FB011082FC01608166237D
:1064C00011F030FD54C1CD80DE8091FE4DC1F5014B
:1064D0008281E82FE295EF708E2F90E0FC013197DA
:1064E000EC30F10508F040C18827E555FF4F8F4F8C
:1064F0000C94DEBFF501248130E0D8010E94F5BF85
:106500002FEF30E040E050E00E9489BF5F934F934F
:106510003F932F9384EF94E00BC0F50187818F9315
:1065200086818F9385818F9384818F9387EF94E009
:106530009F938F93FF92EF92DF92CF920E94CDC4F0
:1065400002C1F50187818F9386818F9385818F9317
:1065500084818F938BEF94E0EBCFF501848095805D
:10656000A680B780C501B4012AE030E040E050E0E9
:106570000E9489BF97FF07C090958095709561959F
:106580007F4F8F4F9F4F9F938F937F936F93C50143
:10659000B4012AE030E040E050E00E9489BF5F9300
:1065A0004F933F932F938FEF94E0C5C0C5010E9496
:1065B000D277F501248185809680B78097FF18C037
:1065C00030E0D8010E94F5BF2FEF30E040E050E00E
:1065D0000E9489BF5F934F933F932F931F928F9297
:1065E000B0FABB24B0F8BF929F9289E095E0A3C0B7
:1065F0009F938F9330E0D8010E94F5BF2FEF30E0DA
:1066000040E050E00E9489BF5F934F933F932F93E8
:106610001F928F92B0FABB24B0F8BF929F9286E08F
:1066200095E09F938F93FF92EF92DF92CF920E941B
:10663000CDC489C0F50185811F928F939681878192
:1066400081708F939F938CE095E072CFF5018480E9
:106650009580A680B78020E030E0A901C501B40193
:106660000E947DC02401350187FF04C077FA709431
:1066700077F87094C301B2010E94F4C069837A83F1
:106680008B839C8329813A81B901330F880B990B45
:106690000E942CC19B01AC01C301B2010E9410C039
:1066A00020E030E048EC52E40E94E1C10E949EC22A
:1066B0000E94F4C0162F072F20E030E0A901C50189
:1066C000B4010E947DC087FF09C00F931F933A81D8
:1066D0003F9389818F9382E195E02ACF0F931F9397
:1066E000FA81FF9329812F9383E195E021CFF50172
:1066F00084811F928F9385811F928F9386811F9231
:106700008F9389E095E09F938F93FF92EF92DF92B2
:10671000CF920E94CDC417C0F50187811F928F933D
:1067200084811F928F9385811F928F9386811F9200
:106730008F9386E095E09F938F93FF92EF92DF9285
:10674000CF920E94CDC40FB6F894DEBF0FBECDBF6E
:106750000BC0F50164817581A701C6010E94B3C415
:1067600003C080E090E027C08D819E8124C0F9E0C5
:106770006F9FB00111246D52794E8D819E810E94D0
:1067800008B8A7016BE175E08D819E810E9495C4D8
:10679000ED81FE8101900020E9F731972D813E8146
:1067A000E21BF30B6901CE0EDF1EEE1AFF0A31E089
:1067B000E31AF1088ACE26960FB6F894DEBF0FBE14
:1067C000CDBFDF91CF911F910F91FF90EF90DF90A0
:1067D000CF90BF90AF909F908F907F906F905F9081
:1067E0004F900895EF92FF920F931F93CF93DF93F3
:1067F000CDB7DEB7A0970FB6F894DEBF0FBECDBF02
:106800007C010FEF10E020E033E040E250E0BE01F9
:106810006F5F7F4F0E943A32F7016281062F0F703F
:10682000162F12951F70BE016F5F7F4F86ED9BE0A4
:106830000E94A9A061E47DE086ED9BE00E945EA03D
:106840004AE050E0612F86ED9BE00E94BF9F6AE323
:106850007DE086ED9BE00E945EA04AE050E0602F64
:1068600086ED9BE00E94BF9F86ED9BE00E94A351B6
:10687000A0960FB6F894DEBF0FBECDBFDF91CF91CB
:106880001F910F91FF90EF900895EF92FF920F9359
:106890001F93CF93DF936115710551F0E42EEB0147
:1068A0008C01CB010E945BAEF82E811103C03DC06C
:1068B000F12C3BC0EC81FD813097B1F080858F7069
:1068C0008250823088F4D80114964D915D916D917B
:1068D0007C9117974187528763877487EC81FD818C
:1068E0008085807F82608087EC81FD81309769F0B0
:1068F0008085982F9F708EEF890F823030F4D801F9
:1069000012968C91807F892B8087EE2029F0F801E8
:106910006081CE010E940CB063E37DE086ED9BE0D8
:106920000E945EA0C8010E94F2338F2DDF91CF91AB
:106930001F910F91FF90EF900895AF92BF92CF9269
:10694000DF92EF92FF920F931F93CF93DF93611526
:10695000710551F0A42E7B01EC01CB010E945BAECE
:10696000B82E811103C074C0B12C72C0F701C4806D
:10697000D580F6010085C114D10409F441C0802FEF
:106980008F709EEF980F923038F4102F1595159553
:106990001595159589F434C0853091F560E0C601F0
:1069A0000E94A4A9009761F1FC0110851595159529
:1069B0001595159529F104C0823071F4F60107C0D0
:1069C00060E0C6010E94A4A9009731F0FC01818516
:1069D0009285A385B48503C080E090E0DC018C83C0
:1069E0009D83AE83BF831295107F8A818F70182B91
:1069F0001A83AA2069F1C7010E9437B0888328C092
:106A00000295007F0595059505950595023099F04D
:106A1000033009F0A9CFF6016185728583859485DD
:106A20000E942CC12A812F7020672A836C837D836A
:106A30008E839F830DC0F6014185528563857485E1
:106A40008A818F70806A8A834C835D836E837F83A3
:106A50008B2DDF91CF911F910F91FF90EF90DF90E1
:106A6000CF90BF90AF900895CF93DF93CDB7DEB7AF
:106A700028970FB6F894DEBF0FBECDBFFC016F7034
:106A80008281807F682B628388E0DE01119601900D
:106A90000D928A95E1F729813A814B815C816D8164
:106AA0007E818F81988528960FB6F894DEBF0FBE41
:106AB000CDBFDF91CF910895CF93DF93CDB7DEB7F0
:106AC00028970FB6F894DEBF0FBECDBFFC016083E0
:106AD00098E0DE01119601900D929A95E1F72981D7
:106AE0003A814B815C816D817E818F81988528966A
:106AF0000FB6F894DEBF0FBECDBFDF91CF910895E2
:106B00000F931F93CF93DF93CDB7DEB728970FB6C0
:106B1000F894DEBF0FBECDBF8C0177FD06C0653691
:106B200071052CF064E670E002C060E070E0F801EE
:106B30008281982F92959F709150923018F08F70AB
:106B4000806182832FEF30E0DB010E94F5BF24E6F5
:106B500030E040E050E00E9489BFF801248388E0E3
:106B6000DE01119601900D928A95E1F729813A8113
:106B70004B815C816D817E818F81988528960FB6CF
:106B8000F894DEBF0FBECDBFDF91CF911F910F9163
:106B90000895CF92DF92EF92FF920F931F93CF93BE
:106BA000DF93CDB7DEB760970FB6F894DEBF0FBEA8
:106BB000CDBFFC01028102950F70202F30E0862F9F
:106BC00090E02817390711F488E04FC0162F6F01A5
:106BD00067E27DE086ED9BE00E945EA04AE050E027
:106BE000602F86ED9BE00E94BF9F64E27DE086ED12
:106BF0009BE00E945EA04AE050E0612F86ED9BE0A2
:106C00000E94BF9F62E27DE086ED9BE00E945EA055
:106C1000F601008119861A861B861C861D861E8633
:106C20001F86188A1295107F6B856F70162B1B8735
:106C30000987EE24EA94FE2C11812281338144815C
:106C4000558166817781CE0109960E942C78F601E4
:106C50002083318342835383648375838683978340
:106C6000C6010E94F23388E0F601DE011196019020
:106C70000D928A95E1F729813A814B815C816D8182
:106C80007E818F81988560960FB6F894DEBF0FBE27
:106C9000CDBFDF91CF911F910F91FF90EF90DF90CB
:106CA000CF900895CF92DF92EF92FF92FC01362FA2
:106CB000928192959F70963009F47AC020F4915099
:106CC000923070F1A5C09730B9F19A50923008F027
:106CD0009FC084819581A681B781662399F0B7FD15
:106CE0009DC08F3F9105A105B10529F024F08FEFDC
:106CF00090E0A0E0B0E02FEF30E0A901481B590B75
:106D0000CA018EC0B7FD87C08F3F9105A105B105AF
:106D100009F00CF485C08FEF90E0A0E0B0E080C0F7
:106D20006481332331F02FEF30E0C901861B9109D4
:106D300077C0862F90E074C0C480D580E680F7804D
:106D40006623E9F020E030E0A901C701B6010E9406
:106D50007DC087FD63C020E030E04FE753E4C7010A
:106D6000B6010E94DCC118160CF455C0A7019601AB
:106D700060E070E08FE793E40E9410C015C020E04F
:106D800030E0A901C701B6010E947DC087FD43C064
:106D900020E030E04FE753E4C701B6010E94DCC1B8
:106DA0001816E4F1C701B6010E94F4C0CB0138C047
:106DB00064817581868197813323B1F0673F5FEFEE
:106DC00075078507950754F161152AE0720781055B
:106DD00091050CF526EF3FEF4FEF5FEF0E9489BF63
:106DE000C90181509F4F1CC0673F4FEF7407840754
:106DF00094078CF061155AE075078105910574F4CC
:106E00002AE030E040E050E00E9489BFC90108C09C
:106E10008FEF9FEF05C080E090E002C08FEF90E021
:106E2000FF90EF90DF90CF900895FC014281E42F16
:106E3000E295EF704E2F50E0FA013197EB30F105FB
:106E400070F5DC018827E954FF4F8F4F0C94DEBFAB
:106E500014966D917D918D919C9117970EC014960B
:106E60006D917D918D919C9117972AE030E040E0E3
:106E700050E00E9489BFCA01B9010E942CC1089547
:106E800014966C9170E080E090E00E942AC1089511
:106E900014966D917D918D919C911797089560E066
:106EA00070E0CB010895CF93DF93EC018A81E82F46
:106EB000E295EF708E2F90E0FC013197EB30F105F9
:106EC00020F58827EE53FF4F8F4F0C94DEBF6C8167
:106ED0007D818E819F811CC06C8170E080E090E09C
:106EE00017C06C817D818E819F810E94F4C010C08B
:106EF0006C817D818E819F812AE030E040E050E00E
:106F00000E9489BFCA01B90103C060E070E0CB01F3
:106F1000DF91CF910895FC019281892F807E80328C
:106F200041F0907F81E0903431F0903521F080E0A5
:106F3000089581E008950895AF92BF92CF92DF92B5
:106F4000EF92FF920F931F93CF93DF93CDB7DEB7EE
:106F5000C154D1090FB6F894DEBF0FBECDBF5C019E
:106F60006B018A0161EB7DE086ED9BE00E945EA0F3
:106F7000B50186ED9BE00E94A9A06EEA7DE086ED5A
:106F80009BE00E945EA0C114D10409F4A1C00C0DC5
:106F90001D1DF80110820E94A9946A3F71055CF4DE
:106FA00061EA7DE08EE29BE00E945EA08EE29BE0C3
:106FB0000E94A3518DC07601E016F10641F0F70161
:106FC00061917F0186ED9BE00E94C69FF5CF86ED23
:106FD0009BE00E94A3518091FC089091FD089E01C6
:106FE0002F5F3F4F790120E030E0059719F443E02F
:106FF00050E019C042E050E061E4C7010E94B8933C
:10700000F70101900020E9F731978F010E191F0950
:10701000A801B701C5010E94A5C40097A9F020E00E
:1070200030E041E050E061E4C7010E94B893F7010D
:1070300001900020E9F731978F010E191F09A8016F
:10704000B701C5010E94A5C4892B39F066E97DE02E
:1070500086ED9BE00E945EA03BC00A0D1B1D6DE10A
:1070600075E0C8010E9485C4892B69F4F60101907E
:107070000020E9F73197EC19FD09329720F0C6019D
:107080000E94D7A225C06FE270E0C8010E947AC4B6
:107090005C01009741F0FC01108281818432C1F0D3
:1070A000FFEFAF1ABF0AF8018081843289F0B8017E
:1070B000C7010E94F2B0C7010E945BAE882329F08D
:1070C000A501B601C7010E944772C7010E9444B0E2
:1070D000CF5BDF4F0FB6F894DEBF0FBECDBFDF91A1
:1070E000CF911F910F91FF90EF90DF90CF90BF90C5
:1070F000AF900895CF92DF92EF92FF920F931F937C
:10710000CF93DF93CDB7DEB767970FB6F894DEBFA6
:107110000FBECDBF8091290D90912A0D892B09F4C6
:10712000D1C061E87DE086ED9BE00E945EA086ED27
:107130009BE00E94A35180913A0D8823E9F00E94C0
:107140004CA380910209882341F08091000990911D
:107150000109892B11F00E944F2D0E94215E809120
:10716000FC089091FD08059711F00E94BC240E9434
:1071700057560E94D923DFCF6BE67DE086ED9BE07A
:107180000E945EA086ED9BE00E94A351E091FE0864
:10719000F091FF08068117818091FE089091FF0809
:1071A000892B71F10115110559F1D80118968C91AF
:1071B0008F70853009F5C8010E9425AA8823E1F067
:1071C000D8016D917C91CE0101960E94F2B0CE0162
:1071D00001960E945BAE882359F08A859B850097B3
:1071E00039F0DC01ED91FC910284F385E02D1995D5
:1071F000CE0101960E9444B0F80102811381CCCFE8
:1072000010927B0710927A0763E67DE086ED9BE0A3
:107210000E945EA086ED9BE00E94A3511092900711
:107220000E94A9946B017C016BE47DE086ED9BE0FC
:107230000E945EA02AE030E0B701A60186ED9BE047
:107240000E94B29F8091290D90912A0D0E94637631
:1072500010922A0D1092290D10927907109278073A
:107260001092FF081092FE081092380D1092370D00
:107270001092F4081092F3081092F2081092F1089C
:10728000109201091092000910920E0910920D0936
:107290000E94A9946B017C0166E47DE086ED9BE091
:1072A0000E945EA02AE030E0B701A60186ED9BE0D7
:1072B0000E94B29F86ED9BE00E94A3511092F008BD
:1072C00010920C0767960FB6F894DEBF0FBECDBFC5
:1072D000DF91CF911F910F91FF90EF90DF90CF90B2
:1072E0000895CF93DF93EC01E881F9810284F3855F
:1072F000E02DCE0119950196B9F7DF91CF91089550
:10730000FC01A285B3851097A9F086859785029721
:1073100088F0CD010196938782876C938685978547
:107320000197978786870284F385E02D108281E09C
:1073300090E0089580E090E00895FC0186819781B7
:107340008F3F2FEF920729F02FEF3FEF37832683F0
:107350000895A085B185109789F02485358521157C
:10736000310561F0CD010196918780878C91215084
:10737000310935872487082E000C990B0895FC01EC
:1073800086819781019639F481E024853585232B08
:1073900019F480E0089581E00895CF92DF92EF9292
:1073A000FF920F931F93CF93DF937C016A018B01B0
:1073B000C0E0D0E0CC15DD0589F0D701ED91FC915E
:1073C0000284F385E02DC70119958F3FBFEF9B071E
:1073D00029F0F80181938F012196ECCFCE01DF9146
:1073E000CF911F910F91FF90EF90DF90CF90089574
:1073F000CF93C62FDC01ED91FC910088F189E02D3F
:107400001995DC01ED91FC910190F081E02D6C2F3C
:10741000CF911994CF93DF93EC018E819F810196D8
:10742000D9F4288539858A859B85820F931F81151C
:107430009041A0F4E881F9810284F385E02DCE012A
:107440001995813291056CF3E881F9810684F785FD
:10745000E02D682FCE01199581E001C080E0DF9119
:10746000CF910895062E000C770BFC01778366837D
:107470000895CF93DF93EC018E819F81019611F5E2
:10748000E881F9810088F189E02DCE011995DC01B0
:10749000ED91FC910084F185E02D1995892BA1F0E7
:1074A000E881F9810284F385E02DCE0119958132BE
:1074B000910534F3E881F9810684F785E02D682F82
:1074C000CE01199581E001C080E0DF91CF91089550
:1074D0000F931F93CF93DF93EC018B0166E275E06E
:1074E0000E94A9A001151105B9F1F80161918F0160
:1074F000662391F1603220F0623211F06C3541F573
:107500006CE5CE010E94C69FF801319780818C30D6
:10751000D1F044F48930D9F08A30B9F0883029F7B5
:1075200062E616C0823259F024F48D30F1F662E73B
:107530000FC08F3231F08C35C1F66CE509C062E2C4
:1075400007C06FE205C066E603C06EE601C064E7EF
:10755000CE010E94C69FC9CF62E2CE010E94C69FA3
:1075600080E090E0DF91CF911F910F910895FC0191
:107570002085318582859385AC014F5F5F4F5387AE
:107580004287820F931F0E9449BF81E090E00895D7
:10759000FC01868197818F3F2FEF920729F02FEF13
:1075A0003FEF378326830895208531858285938533
:1075B000AC014F5F5F4F53874287820F931F0E943A
:1075C00041BF082E000C990B0895FC01868197811C
:1075D0008F3F2FEF920729F02FEF3FEF378326835E
:1075E0000895808591850C94DCB8CF92DF92EF925C
:1075F000FF92CF93DF93EC018E819F818F3F2FEF1E
:10760000920759F02FEF3FEF3F832E83DF91CF9109
:10761000FF90EF90DF90CF9008950E94844E6B0111
:107620007C01A4EFCA0EA1E0DA1EE11CF11CE88186
:10763000F9810088F189E02DCE011995DC01ED91E9
:10764000FC910084F185E02D1995892B39F40E9475
:10765000844E6C157D058E059F0548F3E881F98100
:107660000088F189E02DCE011995DC01ED91FC91A6
:107670000284F385E02DDF91CF91FF90EF90DF90B2
:10768000CF901994EF92FF920F931F93CF93DF93B4
:10769000009719F48FEF9FEF82C0FC01E484F5841A
:1076A000D7010D911C91D801ED91FC910688F789C5
:1076B000E02DC8011995882369F3D801ED91FC915B
:1076C0000084F185E02DC8011995D801ED91FC9158
:1076D000892B61F30284F385E02DC8011995EC0133
:1076E0000196C1F2F8018589882339F04AE050E01B
:1076F0006C2F89E39BE00E94BF9FD70112968C916B
:10770000882309F44BC0C532D10509F047C0D80120
:10771000ED91FC910084F185E02DC8011995029747
:107720005CF0D801ED91FC910688F789E02DC80145
:1077300019958111ECCFAECFD1E0C0E0D801ED9129
:10774000FC910284F385E02DC80119958F3FBFEFAE
:107750009B0709F49FCF9C01215431092A3131053F
:1077600030F09C01215631092A31310538F48D2F32
:107770008295807F829FC00D11240AC0C0978A30F5
:10778000910530F49D2F9295907F989FC00D112404
:10779000D150A0F68C2FCC0F990B01C0CE01DF91F8
:1077A000CF911F910F91FF90EF9008958F929F922C
:1077B000AF92BF92CF92DF92EF92FF920F931F93FF
:1077C000CF93DF936115710509F406C1FB010085B4
:1077D0000295007F0595059505950595002E000CF1
:1077E000110B220B330B0730110508F0F5C0DB013C
:1077F000EC01F8018827E353FF4F8F4F0C94DEBF55
:1078000068E275E006C019968C91882389F06DE2D4
:1078100075E0CE01DF91CF911F910F91FF90EF9016
:10782000DF90CF90BF90AF909F908F900C9494A0DA
:1078300062E375E0EECF19964D915D916D917C916B
:107840001C972AE030E0CE01DF91CF911F910F917C
:10785000FF90EF90DF90CF90BF90AF909F908F9070
:107860000C94CD9F1996CD90DD90ED90FC901C97D7
:1078700020E030E0A901C701B6010E947DC087FF6A
:1078800009C067EE74E0CE010E94A9A0F7FAF09457
:10789000F7F8F094C701B6010E94FBC04B015C01F0
:1078A0002AE030E0AB01BC01CE010E94B29F68E348
:1078B00075E0CE010E94A9A0C501B4010E942AC1B1
:1078C0009B01AC01C701B6010E9410C02DEC3CEC3D
:1078D0004CE45DE30E9411C020E030E040E251E45E
:1078E0000E94E1C10E94FBC0AB0160E070E02AE0B1
:1078F000CE010E945A5170C019966D917C911A97D1
:10790000CE01DF91CF911F910F91FF90EF90DF900B
:10791000CF90BF90AF909F908F900C94683A16963E
:107920000D911C9117976BE5CE010E94C69F0196A1
:1079300019F48FEF9FEF52C00115110571F0B801D6
:10794000CE010E94D63B0196A1F3F801028113817A
:107950000115110589F36CE2E7CF6DE52FC016968E
:107960000D911C9117976BE7CE010E94C69F01965F
:1079700001F30115110509F1F80160817181CE0152
:107980000E94683A0196A9F26AE3CE010E94C69F5E
:10799000019679F2B801CE010E94D63B019649F2D8
:1079A000F801028113810115110519F36CE2CE0172
:1079B0000E94C69F0196E9F6BCCF6DE7CE010E94FA
:1079C000C69F21E030E0019611F020E030E08827EA
:1079D0009927821B930B02C080E090E0DF91CF914A
:1079E0001F910F91FF90EF90DF90CF90BF90AF90DD
:1079F0009F908F900895CF93DF93EC01E881F981F8
:107A00000284F385E02DCE0119958F3F2FEF920769
:107A100071F0E881F9818132910594F30684F7854C
:107A2000E02D682FCE01199580E090E002C08FEF25
:107A30009FEFDF91CF910895EF92FF920F931F93E5
:107A4000CF93DF938C017B01DC01ED91FC910284EB
:107A5000F385E02D1995829709F07AC0F7018085AA
:107A6000807F8460808786E090E00E94E7B5EC012B
:107A7000892B09F46DC0EDEEF7E0F983E88380E02F
:107A800091E0DF019C011D9221503040E1F79B8382
:107A90008A831D821C82D801ED91FC910284F385BA
:107AA000E02DC80119958F3FBFEF9B0709F44DC02A
:107AB0008232910509F44FC0803291050CF44BC01D
:107AC0008C35910511F0BE013DC0D801ED91FC91BE
:107AD0000284F385E02DC80119958F3FBFEF9B0706
:107AE000A1F18236910531F15CF48F329105F9F004
:107AF0008C359105C9F0829771F6BE0182E222C0F1
:107B00008E369105D1F034F48636910521F6BE010A
:107B10008CE018C08237910599F08437910509F0FF
:107B2000BACFBE0189E00EC0BE018CE50BC0BE011C
:107B30008FE208C0BE0188E005C0BE018AE002C035
:107B4000BE018DE00E9493A3A6CFCE010E947FB616
:107B50008FEF9FEF24C08C819D81009749F0E881D1
:107B6000F9818E0F9F1FFC0131978081882321F0BE
:107B7000BE0180E00E9493A38C819D810E94E7B5A5
:107B80008C01009739F06DEE77E00E948EC4CE0133
:107B90000E947FB6F7011287018780E090E0DF91B5
:107BA000CF911F910F91FF90EF9008958DE090E09D
:107BB0000E94E7B5009729F02DE0FC0111922A956B
:107BC000E9F708950F931F93CF93DF930097E1F0A8
:107BD000EC010C851D850115110579F0D8018D91F9
:107BE0009C91009739F0DC01ED91FC910488F589B6
:107BF000E02D1995C8010E947FB6CE01DF91CF918B
:107C00001F910F910C947AB8DF91CF911F910F9132
:107C10000895AF92BF92CF92DF92EF92FF920F93AF
:107C20001F93CF93DF9300D01F92CDB7DEB76115BE
:107C3000710509F496C06B01182FDB011C96AD90FD
:107C4000BC901D97F501E080F180D701ED91FC918A
:107C50000688F789E02DC7011995811104C0C60176
:107C60000E94E23D7EC0F5019281911114C0D701BE
:107C7000ED91FC910190F081E02D612FC7011995E4
:107C8000F7018589882309F469C0612F89E39BE0A6
:107C90000E94C69F63C0812F8F7D81548A3138F343
:107CA00080ED810F8A3018F383ED810F8230F8F276
:107CB0001F35E9F21E37D9F21132B1F086EC810F8F
:107CC000823090F08AED810F873070F01D3361F0C3
:107CD000812F8F7E8F3241F08DED810F823020F029
:107CE0001B3511F01D3511F491FFC1CF19821A8295
:107CF0001B821C82812F012E000C990B9F931F93D6
:107D00008AE395E09F938F938E010F5F1F4F1F9320
:107D10000F930E940AC56E01F4E0CF0ED11C0F90A4
:107D20000F900F900F900F900F90D701ED91FC9155
:107D30000190F081E02DD8016C91C7011995F701F0
:107D40008589882331F0D8016C9189E39BE00E94FA
:107D5000C69F0F5F1F4F0C151D0539F780E090E09F
:107D600002C08FEF9FEF0F900F900F900F90DF9159
:107D7000CF911F910F91FF90EF90DF90CF90BF9028
:107D8000AF9008952C9A08952C980895CF92DF9281
:107D9000EF92FF920F931F93CF93DF93EC017A0141
:107DA0008B016C01C40ED51ECC15DD05A9F00E9417
:107DB000C43E8FE00E94F58A8D2F0E94F58A8C2F99
:107DC0000E94F58A219680E00E94F58AF80181934D
:107DD0008F010E94C23EE8CFC701DF91CF911F9172
:107DE0000F91FF90EF90DF90CF900895CF92DF92A8
:107DF000EF92FF920F931F93CF93DF93EC017A01E1
:107E00008B016C01C40ED51ECC15DD05A1F00E94BE
:107E1000C43E80EF0E94F58A8D2F0E94F58A8C2F38
:107E20000E94F58A2196F80181918F010E94F58ABE
:107E30000E94C23EE9CFC701DF91CF911F910F9100
:107E4000FF90EF90DF90CF9008951F93CF93DF9333
:107E5000D82F192FC62F0E94C43E80EF0E94F58AAA
:107E6000812F0E94F58A8D2F0E94F58A8C2F0E9407
:107E7000F58A0E94C23E81E0DF91CF911F91089563
:107E80001F93CF93DF93182F66E270E00E94878CD8
:107E9000C82FD0E067E270E0812F0E94878CDC2F32
:107EA000CC279E01282BC901DF91CF911F91089506
:107EB0001F93CF93DF93182F60E270E00E94878CAE
:107EC000C82FD0E061E270E0812F0E94878CDC2F08
:107ED000CC279E01282BC901DF91CF911F910895D6
:107EE000AF92BF92CF92DF92EF92FF920F931F93C8
:107EF000CF93DF93CDB7DEB7CC55D1090FB6F89449
:107F0000DEBF0FBECDBF6C017B015B01AA2488E000
:107F1000B82273FD0DC00E94A994663971058105D0
:107F2000910530F08091FC089091FD08059781F44F
:107F3000B70166277370C6010E94BDAF64E47EE09E
:107F400086ED9BE00E945EA0AA24AA94BA2CF0C100
:107F500069961CAE1DAE1EAE1FAE69976D961CAE27
:107F60001DAE1EAE1FAE6D9768968FAD68978F7071
:107F700068968FAF689766961FAE669741E0B60128
:107F8000CE018B5A9F4F0E949D3460E073E0C60182
:107F90000E94F5AFE82AF92A1AAA19AAFE01F39657
:107FA00082E1DF011D928A95E9F77A96119211928A
:107FB00086E0DF011D928A95E9F7F0FE21C0669602
:107FC0008FAD669790E08831910590F4FC01882789
:107FD000EC52FF4F8F4F0C94DEBF62EA7EE002C08E
:107FE0006EE97EE0CE01835B9F4F0E94DAB708C046
:107FF00060E97EE086ED9BE00E945EA0E894F0F8E8
:1080000068968FAD689782958F70813008F45FC055
:10801000833018F0883009F05AC00E9466A888237F
:1080200009F482C18091390D81117EC120E030E0D8
:1080300043E050E060E3CE0101960E94B893D60180
:10804000ED91FC91608171814FE250E0CE0101968B
:108050000E9495C404E610E020E032E044E150E0E4
:10806000BE016F5C7F4FCE018B5A9F4F0E943A3208
:10807000F1FE06C066968FAD6697823009F02FC17B
:10808000F0FE25C0BE01635B7F4FCE0101960E94CA
:1080900088A961E87EE086ED9BE00E945EA0BE01BB
:1080A0006F5F7F4F86ED9BE00E94A9A06EE77EE0A8
:1080B00086ED9BE00E945EA0BE01635B7F4F86ED74
:1080C0009BE00E94A9A086ED9BE00E94A351F1FED7
:1080D0008EC020E030E043E050E060E3CE01019646
:1080E0000E94B893D601ED91FC91608171814FE2BD
:1080F00050E0CE0101960E9495C468EA74E0CE017A
:1081000001960E946FC468968FAD689782958F70B4
:108110008450823018F567E1CE018B5A9F4F0E9440
:108120005C3526962FAF269727963FAF2797289640
:108130004FAF289729965FAF29972A966FAF2A9756
:108140002B967FAF2B972C968FAF2C972D969FAFAA
:108150002D970FEF10E020E033E004C00FEF10E0A8
:1081600020E032E044E150E0BE016F5C7F4FCE0181
:108170008B5A9F4F0E943A3240E350E06AE77EE01C
:10818000CE0101960E94EAB764E77EE086ED9BE0AF
:108190000E945EA0BE016F5F7F4F86ED9BE00E9454
:1081A000A9A061E77EE086ED9BE00E945EA0BE0193
:1081B0006F5C7F4F86ED9BE00E94A9A086ED9BE05F
:1081C0000E94A3510E9466A8882309F4ADC0809143
:1081D000390D8111A9C0BE016F5C7F4FCE010196A0
:1081E0000E9488A960E072E0C6010E9483AFF0FEA1
:1081F00097C066968FAD66978A3059F028F4813023
:1082000071F0863061F016C08B3031F08C3059F04F
:1082100011C067E67EE009C062E67EE006C0F601B6
:108220008085853039F46CE67EE0CE01835B9F4F1C
:108230000E94DAB720E030E043E050E060E3CE0196
:1082400001960E94B893D601ED91FC9160817181F5
:108250004FE250E0CE0101960E9495C468EA74E0B6
:10826000CE0101960E946FC440E350E06EE57EE0CF
:10827000CE0101960E94EAB768E57EE086ED9BE0BC
:108280000E945EA0BE016F5F7F4F86ED9BE00E9463
:10829000A9A065E57EE086ED9BE00E945EA0BE01A0
:1082A000635B7F4F86ED9BE00E94A9A086ED9BE07B
:1082B0000E94A3510E9466A88823B1F18091390DD4
:1082C000811132C0BE01635B7F4FCE0101960E94D7
:1082D00088A960E071E0C6010E9483AF21C08530AB
:1082E00009F4CECEBE016F5C7F4FCE0101960E9495
:1082F00088A96AE87EE086ED9BE00E945EA0BE0150
:108300006F5F7F4F86ED9BE00E94A9A067E87EE04B
:1083100086ED9BE00E945EA0BE016F5C7F4FCFCEDA
:10832000AA24A394B12C04C0B701C6010E94BDAF1A
:10833000C501C45ADF4F0FB6F894DEBF0FBECDBFE4
:10834000DF91CF911F910F91FF90EF90DF90CF9031
:10835000BF90AF900895CF93DF93EC0160E073E09E
:108360000E94F5AF009791F02091FC083091FD0834
:108370002630310559F4BC01CE010E94703F60E007
:1083800073E0CE01DF91CF910C9483AFDF91CF9159
:108390000895CF92DF92EF92FF920F931F93CF93A6
:1083A000DF93CDB7DEB728970FB6F894DEBF0FBEC8
:1083B000CDBF6C018B0162E070E00E9422AF7C01B6
:1083C00019821A821B821C821D821E821F821886BD
:1083D0008B818F708B831982F7FC92C040E0B601CD
:1083E000CE0101960E949D3463E070E0C6010E94B8
:1083F00022AFAC011816190614F04FE350E081E0EB
:10840000E816F10421F4012F110F110B04C082E0D2
:10841000E816F1040CF411272FEF30E0D8010E9488
:10842000F5BF9A01550F440B550B0E9489BF890176
:10843000C6010E9437B0E82EF12C60E0CE01019613
:108440000E9452360817190771F40115110509F435
:108450005AC082E0E816F10489F085E0E816F104DC
:1084600009F051C00BC001151105C1F186E0E816F5
:10847000F10441F081E0E816F10421F061E0C60169
:108480000E940CB017FD07C00F3F110531F02CF012
:108490000FEF10E002C000E010E08B81982F929562
:1084A0009F709150923018F08F7080618B830D8394
:1084B00040E0B601CE0101960E94453482E0E81604
:1084C000F10421F085E0E816F10429F460E071E0A0
:1084D000C6010E94703F60E072E00EC085E0E816C1
:1084E000F10489F082E0E816F10469F062E0C60167
:1084F0000E940CB060E071E0C6010E94703F03C0B2
:1085000080E090E002C081E090E028960FB6F894F9
:10851000DEBF0FBECDBFDF91CF911F910F91FF90B6
:10852000EF90DF90CF900895CF93DF93EC016BE154
:108530007EE086ED9BE00E945EA060E074E0CE01EC
:10854000DF91CF910C94BDAFBF92CF92DF92EF92AB
:10855000FF920F931F93CF93DF93CDB7DEB728978A
:108560000FB6F894DEBF0FBECDBF7C0109831A831E
:108570002B833C834D835E836F837887CE01019686
:108580000E94B1A96C01023011F0053011F4C12C28
:10859000D12C60E070E0C7010E9422AFB82E192FE5
:1085A0006FE27EE086ED9BE00E945EA04AE050E034
:1085B0006B2D712F86ED9BE00E9415A06DE27EE091
:1085C00086ED9BE00E945EA04AE050E0B60186ED99
:1085D0009BE00E9415A086ED9BE00E94A3510091B4
:1085E0000F09109110090115110561F041E0B70163
:1085F000CE0101960E944534C7010E94944200E0DA
:1086000010E061C081E090E09093100980930F0921
:1086100026E040E855E260E070E08EE199E00E94DB
:1086200046ADB092060A8EE199E09093050A8093D8
:10863000040A1092110B1092130B1092120B80ED82
:1086400097E090938C0A80938B0A10928E0A109276
:108650008D0AC114D10439F085E090E09093900A1E
:1086600080938F0A04C01092900A10928F0A86E0BD
:108670000E948FAA62E370E080E090E00E944A4E80
:1086800082ED97E090938C0A80938B0A10928E0A69
:1086900010928D0A24E62C9DC0012D9D900D112471
:1086A0009093900A80938F0A86E00E948FAA10927E
:1086B000100910920F09882321F0C7010E949442EB
:1086C00002C001E010E0C80128960FB6F894DEBFA2
:1086D0000FBECDBFDF91CF911F910F91FF90EF9013
:1086E000DF90CF90BF9008952F923F924F925F926C
:1086F0006F927F928F929F92AF92BF92CF92DF92B2
:10870000EF92FF920F931F93CF93DF93CDB7DEB716
:108710002E970FB6F894DEBF0FBECDBF5C01098364
:108720001A832B833C834D835E836F837887CE01CE
:1087300001960E94B1A94C01023011F0053011F4EC
:10874000812C912CF50102811381F80180858F70B5
:10875000853009F051C0C8010E9425AAE82EF12CED
:10876000F2E0EF16F1040CF447C060E0C8010E948B
:10877000A4A9FC01818592859C878B8761E0C80153
:108780000E94A4A9FC014184528463847484809172
:108790000F09909110099E878D8792E0E916F104E8
:1087A00009F44CC062E0C8010E94A4A9FC018185C3
:1087B00092859A878987F3E0EF16F10409F442C0A5
:1087C00063E0C8010E94A4A9FC0121843284F4E082
:1087D000EF16F104A1F064E0C8010E94A4A9FC0115
:1087E000C184D28421143104D1F08D859E85892BDA
:1087F00051F0C5010E94944280E090E02AC022E03E
:10880000C22ED12CEFCF9101D4010E94EDBF24E6FE
:1088100030E040E050E00E9489BF790105C0ED855D
:10882000FE85EF2B31F7740109851A859601A201A7
:108830006B857C85C5010E94B57C0BC0EFEFFFEF17
:10884000FA87E9878FE3282E312C92E0C92ED12CAC
:10885000CCCF2E960FB6F894DEBF0FBECDBFDF9102
:10886000CF911F910F91FF90EF90DF90CF90BF902D
:10887000AF909F908F907F906F905F904F903F90C0
:108880002F9008958F929F92AF92BF92CF92DF92D6
:10889000EF92FF920F931F93CF93DF93CDB7DEB785
:1088A0006F970FB6F894DEBF0FBECDBF7C01088F67
:1088B000198F2A8F3B8F4C8F5D8F6E8F7F8FCE01EC
:1088C00048960E94B1A96C01D7011296ED91FC91D6
:1088D000139780858F70843009F0C9C0B02E6185F0
:1088E0007285CE0101960E94F2B0CE0101960E94DF
:1088F0005BAE882309F449C08985893009F045C0F9
:1089000060E070E0CE0101960E9422AFA82E192FE0
:108910006BE37EE086ED9BE00E945EA04AE050E0C3
:108920006A2D712F86ED9BE00E9415A069E37EE021
:1089300086ED9BE00E945EA04AE050E0B60186ED25
:108940009BE00E9415A063E37EE086ED9BE00E9421
:108950005EA0602F70E04AE050E086ED9BE00E9450
:1089600015A086ED9BE00E94A35100910F09109184
:1089700010090115110561F041E0B701CE014896DB
:108980000E944534C7010E94944200E010E06AC092
:1089900081E090E09093100980930F0926E040E871
:1089A00055E260E070E08EE199E00E9446ADA09251
:1089B000060A8EE199E09093050A8093040A1092CA
:1089C000110B1092130B1092120BB2E0BB1609F4AC
:1089D00056C085E0B81609F452C0B601DD0C880B0C
:1089E000990B0E942CC122E538EB42E152E40E942F
:1089F00011C020E030E040E251E40E94E1C12DEEE0
:108A00003EE94CE35EE30E9482C04B015C0120E042
:108A100030E0A9010E94DCC120E030E040E05FE3EB
:108A200087FD28C0C501B4010E9411C00E94F4C096
:108A300083ED97E090938C0A80938B0A10928E0AB4
:108A400010928D0A7093900A60938F0A86E00E94BC
:108A50008FAA1092100910920F09882399F0C7016C
:108A60000E949442CE0101960E9444B00EC000E0E4
:108A700010E00BC0C501B4010E9410C0D7CF60E068
:108A800070E0D6CF01E010E0EDCFC8016F960FB6D1
:108A9000F894DEBF0FBECDBFDF91CF911F910F9134
:108AA000FF90EF90DF90CF90BF90AF909F908F900E
:108AB00008950F931F93CF93DF93CDB7DEB76F97D2
:108AC0000FB6F894DEBF0FBECDBF8C01188E198E85
:108AD0001A8E1B8E1C8E1D8E1E8E1F8E8A8D8F7081
:108AE0008A8F188ED801ED91FC916081718186ED9D
:108AF0009BE00E94A9A0C8010E945BAE81110DC03D
:108B000062E17EE086ED9BE00E945EA086ED9BE048
:108B10000E94A3518FEF9FEFD1C0C8010E9437B0D0
:108B2000F80190859730B1F0853009F491C030F4A8
:108B3000813049F0823009F48BC00CC0863019F0C6
:108B40008A50833038F463EE7DE086ED9BE00E942E
:108B50005EA0B2C0D80119968D919C911A9700978A
:108B6000C9F0DC01ED91FC910688F789E02D19959B
:108B700011E0009709F410E0892B19F063EE7DE015
:108B800002C06CEE7DE086ED9BE00E945EA0812F2E
:108B900090E094C040E0B801CE0148960E949D3418
:108BA000F8018085873079F038F4833009F45AC0B1
:108BB000843009F450C05CC0883009F453C0893057
:108BC00009F449C055C00280F381E02D80858F7083
:108BD000853009F056C06CE07EE086ED9BE00E9497
:108BE0005EA0D8011296ED91FC9113970681178132
:108BF0000115110569F1F80180858F70843011F538
:108C000061857285CE0101960E94F2B0CE01019677
:108C10000E945BAE882391F0CE0101960E945945D7
:108C2000181619065CF463EE7DE086ED9BE00E9469
:108C30005EA0CE0101960E9444B03EC0CE010196D6
:108C40000E9444B0D80112960D911C911397D0CF79
:108C50006CEE7DE00FC060E0CE0148960E94523677
:108C60008C0111C0CE0148960E9453378B010BC076
:108C700062E07EE086ED9BE00E945EA080E090E0F6
:108C80001DC000E010E067EF7DE086ED9BE00E94F4
:108C90005EA04AE050E0B80186ED9BE00E9415A07E
:108CA00086ED9BE00E94A35131E020E0012B09F406
:108CB00030E0832F922F02C081E090E06F960FB6D4
:108CC000F894DEBF0FBECDBFDF91CF911F910F9102
:108CD00008950C94D2806CE470E183E29BE00E94E2
:108CE0005EA0E0E0F0E01994CF93C1E068EE73E09D
:108CF00080E090E00E944A4E4AE050E06C2F83E210
:108D00009BE00E94BF9FCF5FC43181F7CF91089550
:108D10000F931F93CF93DF93CDB7DEB728970FB68E
:108D2000F894DEBF0FBECDBF0E94D87F65EA7EE01B
:108D300083E29BE00E945EA0CE0101960E94A8A75C
:108D4000CE0101960E94129A0EEB13E01A8309835A
:108D50001B821C821D821E82CE0107960E9493A751
:108D60008F8198850E94E36C44E050E0BE016D5F06
:108D70007F4F81E090E00E94C63E0E94E26CCE01EF
:108D800001960E94129A1A8309831B821C821D82FB
:108D90001E82CE0107960E9493A78F8198850E941C
:108DA000E36C44E050E0BE016D5F7F4F85E090E0F2
:108DB0000E94C63E0E94E26CCE0101960E94129A69
:108DC0006BEC7EE083E29BE00E945EA028960FB6EB
:108DD000F894DEBF0FBECDBFDF91CF911F910F91F1
:108DE00008954F925F926F927F928F929F92AF926F
:108DF000BF92CF92DF92EF92FF920F931F93CF9388
:108E0000DF93CDB7DEB76D970FB6F894DEBF0FBE18
:108E1000CDBF0091290D10912A0D0115110509F4FE
:108E200052C580913A0D8F5F80933A0D60E475E0F2
:108E3000C8010E94EC5E9093FF088093FE0866E4F0
:108E400075E0C8010E94EC5E9093380D8093370D59
:108E500065E575E0C8010E94EC5E90937907809308
:108E600078076DE475E0C8010E94EC5E9093F40809
:108E70008093F3080E94283162E575E08091290D06
:108E800090912A0D0E94EC5E9093F2088093F10875
:108E9000009709F4A9C00E9425AA082F10E0011527
:108EA000110509F4A1C0000F111F000F111F8091BF
:108EB000EE089091EF08892B09F085C0C8010E9447
:108EC000E7B59093EF088093EE081092B10D1092E1
:108ED000B00D1092F6081092F5081092AF0D109296
:108EE000B30D1092B20D7801013082E018071CF02A
:108EF000E12CA2E0FA2EC70101960E94E7B59093FB
:108F0000B50D8093B40D9093AE0D8093AD0D8E0D85
:108F10009F1D9093A80D8093A70D0E94844E60938F
:108F2000A90D7093AA0D8093AB0D9093AC0D80E0CA
:108F300090E0E091B40DF091B50DE80FF91F1082AB
:108F40000196E816F906ACF782E090E09093B10D37
:108F50008093B00D80E98093C9001092C8001092F0
:108F6000CD0083E08093CC008EE08093CA00F09225
:108F70000702E09206022091B40D3091B50D809168
:108F8000060290910702820F931F9093A80D809381
:108F9000A70D232B09F480C365E770E189E39BE00B
:108FA0000E945EA04AE050E0B80189E39BE00E9485
:108FB00015A089E39BE00E94A35181EB99E5909372
:108FC000A60D8093A50D69EE71E183E29BE00E94FE
:108FD0005EA04AE050E0B80183E29BE00E9415A049
:108FE00083E29BE00E94A35168E575E08091290D22
:108FF00090912A0D0E94EC5E8C01009709F442C00A
:109000000E9425AA81114FC33DC00E94A9944B0123
:109010005C0161E870E186ED9BE00E945EA02AE0C1
:1090200030E0B501A40186ED9BE00E94B29F86ED81
:109030009BE00E94A3516DEC71E183E29BE00E94F2
:109040005EA04AE050E0B60183E29BE00E9415A0DA
:1090500083E29BE00E94A3510E94A9946B017C01D2
:1090600067EC71E186ED9BE00E945EA02AE030E0B3
:10907000B701A60186ED9BE00E94B29F86ED9BE0C2
:109080000E94A3510091290D10912A0D6CE575E005
:10909000C8010E94EC5E90930E0980930D0963E66F
:1090A00075E0C8010E94EC5E90930109809300096D
:1090B000009709F4DAC1209102092111D6C1DC011F
:1090C0001696ED90FC9017978091FA089091FB0806
:1090D000892B09F004C165E271E186ED9BE00E94F5
:1090E0005EA086ED9BE00E94A3510E94A9944B01D3
:1090F0005C016FE171E186ED9BE00E945EA02AE0D9
:1091000030E0B501A40186ED9BE00E94B29F86EDA0
:109110009BE00E94A35181E190E00E94E7B58C01A1
:1091200088E1F801818312821082108A17861092DA
:10913000400D10923F0D1092060D1092280D0E94C6
:109140005490E5EAAE2EEFE8BE2EB0923C0DA09210
:109150003B0DF6EACF2EFFE8DF2ED0923E0DC092F7
:109160003D0D1093FB080093FA08012B39F46DE0D4
:1091700071E18EE29BE00E945EA05AC080EA90E01E
:109180000E94E7B590938D0780938C070E94A99465
:109190002B013C0161E071E186ED9BE00E945EA045
:1091A0002AE030E0B301A20186ED9BE00E94B29F6D
:1091B00086ED9BE00E94A35188E290E00E94E7B513
:1091C00090938907809388070E94A9942B013C0102
:1091D00064EF70E186ED9BE00E945EA02AE030E043
:1091E000B301A20186ED9BE00E94B29F86ED9BE059
:1091F0000E94A35180918C0790918D07892B31F0AB
:109200008091880790918907892BB9F40E94A994CD
:109210004B015C016CED70E18EE29BE00E945EA070
:109220002AE030E0B501A4018EE29BE00E94B29FEB
:109230008EE29BE00E94A3515BC088E891EB909383
:109240008B0780938A071092400D10923F0D109269
:10925000060D1092280D0E945490B0923C0DA092E1
:109260003B0DD0923E0DC0923D0D8091FA08909139
:10927000FB080E94319081E00E94D476811132C0B7
:1092800069EC70E186ED9BE00E9482A00091FA08F3
:109290001091FB08C8010E94319040E060EFC801C6
:1092A0000E949E6FC8010E942E90E091FA08F091F2
:1092B000FB0881E0808369EA70E186ED9BE00E9413
:1092C00082A08091FA089091FB080E940A7088237E
:1092D00031F06DE970E186ED9BE00E9482A081E0B3
:1092E00090E008C06FE870E186ED9BE00E9482A0EC
:1092F00080E090E0282F217020930209892B31F023
:1093000067EB71E183E29BE00E945EA010928F0701
:1093100010928E07CC24C394D12CE114F10409F4EB
:10932000A4C080910209882309F49FC0D701189630
:109330008C9118978F70863009F093C00D911C9115
:10934000FE0131965F014801F0E18F0E911C35015D
:10935000D8018C910E940795582EF80181810E94B6
:109360000795529460EF56228529D5018D935D01B2
:109370000E5F1F4F8016910659F780918E079091CE
:109380008F07843191050CF06CC0880F991FE09114
:109390008807F0918907E80FF91FD182C082A09158
:1093A0008E07B0918F0733E0AA0FBB1F3A95E1F704
:1093B00080918C0790918D07A80FB91F88E0F30169
:1093C00001900D928A95E1F700918E0710918F0719
:1093D0006DE471E186ED9BE00E945EA04AE050E002
:1093E000B80186ED9BE00E9415A066E471E186ED70
:1093F0009BE00E945EA080918E0790918F0743E0D2
:10940000880F991F4A95E1F720918C0730918D07BD
:10941000820F931F0E9446A786ED9BE00E94A351F6
:10942000E0918E07F0918F0753E0EE0FFF1F5A95E2
:10943000E1F780918C0790918D07E80FF91F8081EB
:10944000883231F48091FA089091FB080E9476915D
:1094500080918E0790918F07019690938F0780934C
:109460008E07F701E280F38058CF10927B071092AD
:109470007A07E091FE08F091FF083097F9F0C68076
:10948000D7800091FE081091FF080115110579F0B1
:10949000C114D10461F0D60118968C918F7085307B
:1094A000A1F7C6010E9425AA823078F32EC1F801E7
:1094B0008681978190937B0780937A0786ED9BE066
:1094C0000E94A351E0917807F0917907309709F451
:1094D00064C080913A0D8F5F80933A0D06811781A9
:1094E0000115110509F454C0D80118968C918F709C
:1094F000863009F049C0198F088F60E070E0CE0116
:1095000048960E94A45D8C8D9D8D892BE9F18091F8
:10951000290D90912A0D892BB9F1E88CF98CF7016E
:1095200080858F708630D1F469EB74E0C7010E94AA
:10953000EC5E009709F03CC1FA82E98260E070E0DD
:10954000CE0101960E94A45D8D819E81892B31F010
:1095500062E070E0CE0101960E944460EC8DFD8DCA
:1095600010821182128213828A8D843008F03FC1EA
:10957000823008F043C162E08B8D0E94014DEC8D7A
:10958000FD8D8181807F8183F80102811381A8CFC5
:1095900080913A0D815080933A0D62E971E183E246
:1095A0009BE00E945EA06AE871E183E29BE00E947A
:1095B0005EA081E02091FE083091FF08232B09F482
:1095C00080E00E94C78061E871E183E29BE00E9435
:1095D0005EA081E02091780730917907232B09F470
:1095E00080E00E94C78062E771E183E29BE00E9415
:1095F0005EA067E671E183E29BE00E945EA081E0ED
:1096000020910D0930910E09232B09F480E00E946E
:10961000C78060E671E183E29BE00E945EA081E08A
:109620002091F3083091F408232B09F480E00E9484
:10963000C78067E571E183E29BE00E945EA081E064
:109640002091000930910109232B09F480E00E9448
:10965000C78083E29BE00E94A3510E94A9946B0102
:109660007C0162E571E183E29BE00E945EA02AE05A
:1096700030E0B701A60183E29BE00E94B29F83E243
:109680009BE00E94A35181E08093F00880913A0D05
:10969000815080933A0D17C16EE570E189E39BE03C
:1096A0000E9482A08ACC6FEF680FC8010E94A4A913
:1096B000DC011996CD90DD90ED90FC901C97909177
:1096C000D10C992359F0809170008E7F80937000A7
:1096D0001092D10C109202021092010282E180934A
:1096E000000291110E94C36E5601C6010E94EB6EEA
:1096F00001E010E0A016B1060CF487CC60E0C801D0
:109700000E94216F0F5F1F4FF5CFDA82C9821B863F
:109710001A86CE0101960E9453B0CE0101960E9496
:109720005BAE8823D9F18A859B850097E1F0DC0147
:10973000ED91FC910484F585E02D1995892B49F074
:109740008A859B85DC01ED91FC910284F385E02DF7
:1097500019958A859B85DC01ED91FC910680F78146
:10976000E02D19951BC060E070E0CE0101960E94CB
:1097700022AF8C0197FFA4C0119501951109AA246D
:10978000A394B12CCE0101960E9437B0E82EF12CA3
:1097900089858530D1F1863009F45CC0D6011296F6
:1097A000CD90DC901397CE0101960E9444B069CE13
:1097B000FC0120852F70253009F0BECEC680D780F1
:1097C000C114D10409F4CACEDA82C982B701CE012C
:1097D00001960E94A45DED81FE81108211821282A9
:1097E0001382D6011296CD90DC901397E9CF803486
:1097F00039F0823409F0C8CE60E003C060E0BCCE2E
:1098000062E08B8D0E94014DBFCEEF2829F462E00B
:10981000CE0101960E940CB061E0802F0E94014DA4
:1098200060E0802F0E94D24C6FEA71E186ED9BE0F0
:109830000E945EA04AE050E0B80186ED9BE00E94E5
:1098400015A06AEA71E186ED9BE00E945EA068EADD
:1098500071E131C0902E61E0802F0E94014D61E0E6
:10986000AB2821F0EA94EF2829F403C0EA94EF280A
:1098700009F060E0E62EF12C892D0E94D24C63EABB
:1098800071E186ED9BE00E945EA04AE050E0B801E5
:1098900086ED9BE00E9415A061EA71E186ED9BE0F8
:1098A0000E945EA04AE050E0B70186ED9BE00E9476
:1098B00015A06FE971E186ED9BE00E945EA06ECF7E
:1098C000A12CB12C5FCF6D960FB6F894DEBF0FBE02
:1098D000CDBFDF91CF911F910F91FF90EF90DF905F
:1098E000CF90BF90AF909F908F907F906F905F9040
:1098F0004F9008950E9416C490E0FC013197E23128
:10990000F10508F04EC08827E451FF4F8F4F0C94AB
:10991000DEBF809180008F7703C0809180008F7DB3
:1099200080938000089580918000877FF9CF84B56F
:109930008F7702C084B58F7D84BD08958091B0007B
:109940008F7703C08091B0008F7D8093B000089521
:10995000809190008F7707C0809190008F7D03C029
:1099600080919000877F8093900008958091A0005F
:109970008F7707C08091A0008F7D03C08091A000E9
:10998000877F8093A0000895809120018F7707C082
:10999000809120018F7D03C080912001877F80937B
:1099A000200108951F93CF93DF93282F30E0F90112
:1099B000E85BFD4E8491F901E25DFA4ED491F90124
:1099C000EC58FA4EC491CC23C1F0162F81110E949D
:1099D0007C4CEC2FF0E0EE0FFF1FE25DFD4EA591F9
:1099E000B4919FB7F894111104C08C91D095D823ED
:1099F00002C0EC91DE2BDC939FBFDF91CF911F91D2
:109A00000895CF93DF9390E0FC01E25DFA4E24913C
:109A1000FC01EC58FA4E8491882361F190E0880FA4
:109A2000991FFC01EC5EFA4EC591D491FC01E25DF8
:109A3000FD4EA591B491611109C09FB7F89488813A
:109A4000209582238883EC912E230BC0623061F431
:109A50009FB7F8948881322F309583238883EC91C7
:109A60002E2B2C939FBF06C08FB7F894E8812E2B26
:109A700028838FBFDF91CF9108951F93CF93DF93FA
:109A8000182FEB0161E00E94014D209711F460E076
:109A900004C0CF3FD10539F461E0812FDF91CF9130
:109AA0001F910C94D24CE12FF0E0E85BFD4EE49165
:109AB0008E2F90E0FC013197E231F10508F09DC056
:109AC0008827E250FF4F8F4F0C94DEBF84B580682B
:109AD00084BDC7BD97C084B5806284BDC8BD92C037
:109AE00080918000806880938000D0938900C0932B
:109AF000880088C080918000806280938000D0932D
:109B00008B00C0938A007EC0809180008860809323
:109B10008000D0938D00C0938C0074C08091B00001
:109B200080688093B000C093B3006CC08091B00097
:109B300080628093B000C093B40064C080919000B4
:109B4000806880939000D0939900C09398005AC089
:109B500080919000806280939000D0939B00C0938E
:109B60009A0050C080919000886080939000D093BC
:109B70009D00C0939C0046C08091A00080688093A7
:109B8000A0008091A0008F7B8093A000D093A900BB
:109B9000C093A80037C08091A00080628093A0008D
:109BA000D093AB00C093AA002DC08091A000886024
:109BB0008093A000D093AD00C093AC0023C08091EF
:109BC0002001806880932001D0932901C09328014F
:109BD00019C080912001806280932001D0932B01D5
:109BE000C0932A010FC080912001886080932001DA
:109BF000D0932D01C0932C0105C0C038D1050CF0C5
:109C00004BCF45CFDF91CF911F910895863308F058
:109C1000865390917B00282F2870977F922B9093EA
:109C20007B008770806480937C0080917A008064E0
:109C300080937A0080917A0086FDFCCF8091780035
:109C40002091790090E0922B08953FB7F89480918D
:109C5000080990910909A0910A09B0910B0926B54C
:109C6000A89B05C02F3F19F00196A11DB11D3FBF54
:109C7000BA2FA92F982F8827820F911DA11DB11DE2
:109C8000BC01CD0142E0660F771F881F991F4A95DE
:109C9000D1F708958F929F92AF92BF92CF92DF92A9
:109CA000EF92FF926B017C010E94254E4B015C01FB
:109CB000C114D104E104F104F1F00E94254EDC014D
:109CC000CB0188199909AA09BB09883E9340A105CF
:109CD000B10570F321E0C21AD108E108F10888EE5D
:109CE000880E83E0981EA11CB11CC114D104E104AC
:109CF000F10419F7DDCFFF90EF90DF90CF90BF9088
:109D0000AF909F908F9008952FB7F89460910409B9
:109D10007091050980910609909107092FBF089558
:109D20004F925F926F927F928F929F92AF92BF926B
:109D3000CF92DF92EF92FF920F931F93CF93DF9317
:109D4000CDB7DEB763970FB6F894DEBF0FBECDBFB9
:109D50007C015B013A01FB0120E080E090E06AE0D9
:109D60003191332309F140ED430F4A3080F4689F6D
:109D7000A001699F500D1124CA01C097830F911D46
:109D800037FD9A958F3F910559F350F313C03E323A
:109D900089F4233079F0D301A20FB11D12968C9370
:109DA0002F5F80E090E0DCCF233021F4F301858346
:109DB00081E021C0F70142815381648175818091E6
:109DC000C3099091C409A091C509B091C60948176B
:109DD00059076A077B0709F499C10E94844E8701DD
:109DE000085F1F4F6F7077277C5FC8010E94368E17
:109DF000813019F080E090E0FCC18EEB93E09A8313
:109E00008983F70182819381A481B5818B839C83AF
:109E1000AD83BE8345E350E0BE016F5F7F4FC80155
:109E20000E94368F892B19F4C12CD12C6AC10E9453
:109E3000844EF701778366837627672776277A83B0
:109E4000698342E050E0BE016F5F7F4FC8010E940E
:109E50008B8A81E090E09E878D8742E050E0BE01D2
:109E6000635F7F4FC8010E948B8A80E091E09E87EC
:109E70008D8742E050E0BE01635F7F4FC8010E94C2
:109E80008B8A1E861D8642E050E0BE01635F7F4FD5
:109E9000C8010E948B8A42E050E0BE01635F7F4FA1
:109EA000C8010E948B8A42E050E0BE01635F7F4F91
:109EB000C8010E948B8A4501F5018081882301F148
:109EC00064015601F60181912F01882321F08E3221
:109ED00011F06201F6CFC818D9081C141D0474F4DF
:109EE000CF8641E050E0BE01615F7F4FC8010E9414
:109EF0008B8AA601B401C8010E948B8A4201DCCF83
:109F00001F8641E050E0BE01615F7F4FC8010E94A3
:109F10008B8AC12CDD24D394DE86CD8642E050E0CE
:109F2000BE01635F7F4FC8010E948B8ADE86CD86AB
:109F300042E050E0BE01635F7F4FC8010E948B8A00
:109F4000C8010E94638E892B09F46ECFE3E0AE2E28
:109F5000B12C230122E0420E511C0E94844E3B0191
:109F60004C01C8010E94BD8D18161906B4F00E945C
:109F7000844EDC01CB0186199709A809B909813AF9
:109F80009F40A105B105E0F40E94CA7F61E070E046
:109F900080E090E00E944A4EE4CFF7014281538175
:109FA00064817581808D918DA28DB38D481759077D
:109FB0006A077B0749F4848D958DC59729F409C0FC
:109FC000CC24CA94DC2C92C05EEFC52EDD24DA943A
:109FD0008DC0F70181A192A10C970CF49FC04CE0B9
:109FE00050E0BE016F5F7F4FC8010E94758D8B816D
:109FF0009C819827892798279A8B898B29813A8178
:10A00000322723273227F701468157812417350746
:10A0100009F07FC097FF7DC08F709270892B09F087
:10A02000E3C06F80788476246724762461147104F9
:10A0300009F4D5C0C12CD12C8D819E819827892708
:10A040009827C816D90608F46EC0812C912C41E0DF
:10A0500050E0BE016D5E7F4FC8010E94758D8B89F7
:10A06000982F907C09F091C0811185C042E050E0AA
:10A07000BE01615F7F4FC8010E94758D42E050E0D4
:10A08000BE01635F7F4FC8010E94758DC8010E94A9
:10A09000948DC8010E94948DC8010E94948DC801BE
:10A0A0000E94948D42E050E0BE016F5E7F4FC80178
:10A0B0000E94758D8F8598898115914009F06DC03A
:10A0C000CD84DE84DC24CD24DC2481E0C816D104D8
:10A0D00009F063C089899A898115944009F07AC092
:10A0E00044E050E0B201C8010E94758D0E94CA7F11
:10A0F00081E0A81AB10829F0FFEFCF16DF0609F4B6
:10A100002CCFC8010E942A8CC60173C08EEF9FEF2E
:10A1100070C04CEFC42EDD24DA94E8CF9DEFC92E39
:10A12000DD24DA94E3CF41E050E0BE01635F7F4F6E
:10A13000C8010E94758D8D85882351F08D859FEF14
:10A14000980F9D87882321F0C8010E94948DF6CF37
:10A150008D858111E8CFC8010E94948DC8010E94AD
:10A16000948DC8010E94948DC8010E94948DFFEFC8
:10A17000CF1ADF0A61CF8B899FEF980F9B8B8823C3
:10A1800041F0C8010E94948DF6CFC8010E94948DC1
:10A190001B8A8B8981115BCF69CFC12CD12C898916
:10A1A0009A89982789279827C816D90638F4C801AC
:10A1B0000E94948DFFEFCF1ADF0AF1CF2FEF821AA2
:10A1C000920A6814790409F042CF26EFC22EDD24EA
:10A1D000DA948CCF77EFC72EDD24DA9487CF3AEF6D
:10A1E000C32EDD24DA9482CF8BEFC82EDD24DA94DF
:10A1F0007DCF63960FB6F894DEBF0FBECDBFDF9163
:10A20000CF911F910F91FF90EF90DF90CF90BF9073
:10A21000AF909F908F907F906F905F904F90089538
:10A220001F920F920FB60F9211242F933F938F938B
:10A230009F93AF93BF938091040990910509A091DA
:10A240000609B09107093091030923E0230F2D3748
:10A2500020F40196A11DB11D05C026E8230F02962A
:10A26000A11DB11D20930309809304099093050952
:10A27000A0930609B09307098091080990910909F4
:10A28000A0910A09B0910B090196A11DB11D8093FF
:10A29000080990930909A0930A09B0930B09BF918B
:10A2A000AF919F918F913F912F910F900FBE0F9083
:10A2B0001F9018958F929F92AF92BF92EF92FF924C
:10A2C0000F931F93CF93DF93CDB7DEB7A1970FB650
:10A2D000F894DEBF0FBECDBF7C01FA01CB0119A2FD
:10A2E000223008F42AE08E010F5D1F4F822E912C40
:10A2F000A12CB12CBF01A50194010E9467BFF901F7
:10A30000CA01015011096A3014F4605D01C0695C32
:10A31000D8016C93232B242B252B61F7B801C7019F
:10A320000E9494A0A1960FB6F894DEBF0FBECDBFD9
:10A33000DF91CF911F910F91FF90EF90BF90AF9061
:10A340009F908F9008956AE975E00C9494A084E042
:10A3500090E00895DC011496ED91FC9115973097EB
:10A3600029F08081082E000C990B089580E090E080
:10A3700008950895DC011296ED91FC9113973097A2
:10A3800079F016968D919C9117978330910549F03D
:10A39000049719F421E030E006C0208530E003C0C6
:10A3A000089522E030E0C901089580911509909147
:10A3B0001609089560E073E186ED9BE00E945EA0BF
:10A3C00086ED9BE00E94A351109216091092150988
:10A3D00081E090E008954F925F926F927F928F920A
:10A3E0009F92AF92BF92CF92DF92EF92FF920F9324
:10A3F0001F93CF93DF93EC01EC81FD8183859485DE
:10A40000892B21F485859685892B89F180910F0907
:10A4100090911009892B59F5E881F9810484F5851B
:10A42000E02DCE0119954C0181E088169104F9F4D4
:10A43000EC81FD8145805680612C712C0E94844EF8
:10A440009B01AC01EC81FD816781708581859285DE
:10A45000AA24AA94BA2C6501830172010E94029376
:10A4600081111AC004C01092100910920F09EC81DA
:10A47000FD8185819681DF91CF911F910F91FF9092
:10A48000EF90DF90CF90BF90AF909F908F907F9094
:10A490006F905F904F900895EA81FB810190F08169
:10A4A000E02D008111816EE474E186ED9BE00E9455
:10A4B0005EA0B80186ED9BE00E94A9A086ED9BE01E
:10A4C0000E94A3519092100980920F09EC81FD81A6
:10A4D00041815281052E000C660B770B23818EE1A2
:10A4E00099E00E9446ADEC81FD8103811481618178
:10A4F00072814AE050E086ED9BE00E9415A06AE47C
:10A5000074E186ED9BE00E945EA0A80160E070E02F
:10A510002AE086ED9BE00E945A5186ED9BE00E9466
:10A52000A35160E070E08A819B810E9422AF8093FA
:10A53000060A8EE199E09093050A8093040A10922E
:10A54000110B1092130B1092120BEC81FD8163859D
:10A55000748542E050E0CE010E94B36BEC81FD8136
:10A560006585768543E050E0CE010E94B36B0C8197
:10A570001D8180E00E94EC92F801678370878187DB
:10A580009287EA81FB810190F081E02D00811181A9
:10A5900061E474E186ED9BE00E945EA0B80186ED67
:10A5A0009BE00E94A9A086ED9BE00E94A3510E941F
:10A5B000844E2B013C010E94844E9B01AC01AA24D5
:10A5C000AA94BA2C650112E3E12EF12C00E010E010
:10A5D000C301B2010E940293811145CF0E948F7D79
:10A5E000EACFCF93DF93EC016DE975E089E39BE05F
:10A5F0000E94C0778C819D810E947FB660E070E0F0
:10A600008A819B810E9467AE1D821C8281E090E05E
:10A61000DF91CF9108950C947FB60E94255B63EF84
:10A6200072E186ED9BE00E945EA086ED9BE00E94B9
:10A63000A35181E090E09093160980931509089545
:10A640008F929F92AF92BF92CF92DF92EF92FF9242
:10A650000F931F93CF93DF93EC010E94255B8C81B6
:10A660009D81892B59F481E190E00E94E7B5BC01FE
:10A670008A819B810E9467AE9D838C830C811D81A2
:10A680000115110559F460E074E18EE29BE00E942F
:10A690005EA08EE29BE00E94A351B7C180E00E94C1
:10A6A000EC92D80117966D937D938D939C931A9796
:10A6B0000C811D81CA80DB800115110509F42CC1B4
:10A6C000C114D10409F428C1F601E280F380E11439
:10A6D000F10409F421C1D70118968C918F7085304F
:10A6E00009F01AC1C7010E9425AA823008F414C1DA
:10A6F00061E0C7010E94A4A9FC0190859F7094307D
:10A7000029F4C184D284C114D10439F467EA73E115
:10A710008EE29BE00E945EA066C1B60180910D09A9
:10A7200090910E090E94EC5E7C01009761F46BE849
:10A7300073E18EE29BE00E945EA0B6018EE29BE098
:10A740000E94A9A050C16CEA75E00E94EC5E0097DF
:10A7500009F445C0FC0120852F70243009F03FC06A
:10A76000A184B284B50186ED9BE00E94A9A067E8B0
:10A7700073E186ED9BE00E945EA08FE3882E83E16B
:10A78000982EC12CD12CA114B104E9F0B401C5015B
:10A790000E94D1B7892B69F486E08C9DF0018D9DD4
:10A7A000F00D1124ED5BFC4E25913491922F832FF7
:10A7B00012C0FFEFCF1ADF0A86E0880E911CACE0D2
:10A7C000CA16D10401F762E273E186ED9BE00E94B4
:10A7D0005EA096E080E0F8019383848307C086E062
:10A7E00090E0D80114969C938E93139763EB75E0D9
:10A7F000C7010E94EC5EEC81FD810097A9F0DC01AD
:10A8000018962C9118972F70223071F419964D914B
:10A810005D916D917C911C97411551056105710504
:10A8200019F05283418304C080E895E292838183CA
:10A8300041815281052E000C660B770B23818EE13E
:10A8400099E00E9446AD68EB75E0C7010E94EC5E9E
:10A850006C010C811D81009779F1FC0180858F705E
:10A86000863051F56DEB75E0C6010E94EC5ED801B3
:10A870001C969C938E931B9762EC75E0C6010E9418
:10A88000EC5EF8019687858766EC75E0C6010E944C
:10A89000EC5E009749F0DC0119968D919C911A9716
:10A8A000F8019683858311C088EE93E0D80116964F
:10A8B0009C938E93159709C0F8011486138688EE31
:10A8C00093E096838583168615866CEC75E0C70148
:10A8D0000E94EC5ED80150969C938E931F97EA815C
:10A8E000FB810190F081E02D008111816AEE73E11E
:10A8F00083E29BE00E945EA0B80183E29BE00E949D
:10A90000A9A083E29BE00E94A351EC81FD8181E03C
:10A91000808381E090E07BC0F601A280B380C50116
:10A920000E9425AAE82ED50118968C918F70FF24DD
:10A93000F394853009F4F12C61EC73E18EE29BE035
:10A940000E945EA061E070E0012B11F460E070E015
:10A950004AE050E08EE29BE00E9415A06FEB73E1AD
:10A960008EE29BE00E945EA061E070E0CD2811F4D1
:10A9700060E070E04AE050E08EE29BE00E9415A0AB
:10A980006DEB73E18EE29BE00E945EA061E070E0FF
:10A99000AB2811F460E070E04AE050E08EE29BE00A
:10A9A0000E9415A06BEB73E18EE29BE00E945EA01B
:10A9B0006F2D70E04AE050E08EE29BE00E9415A00F
:10A9C00069EB73E18EE29BE00E945EA061E070E0C3
:10A9D000B1E0BE1510F460E070E04AE050E08EE2B5
:10A9E0009BE00E9415A08EE29BE00E94A35166EDC1
:10A9F00073E18EE29BE00E945EA08EE29BE00E94EB
:10AA0000A351EC81FD8182E0808380E090E0DF91C2
:10AA1000CF911F910F91FF90EF90DF90CF90BF905B
:10AA2000AF909F908F900895AF92BF92CF92DF9298
:10AA3000EF92FF920F931F93CF93DF93CDB7DEB7C3
:10AA400068970FB6F894DEBF0FBECDBF098B1A8B87
:10AA50002B8B3C8B4D8B5E8B6F8B788FDC01129632
:10AA60002D913C911397232B09F482C0CC2009F43B
:10AA70007FC06C01ED91FC91028CF38DE02D199556
:10AA80005C0167E173E186ED9BE00E945EA0CE0170
:10AA900041960E94F233A114B10451F460E0CE015A
:10AAA00041960E945236682FF601848195815DC0DF
:10AAB000F1E0AF16B10431F082E0A816B10421F044
:10AAC00081E003C085E001C084E019861A861B86F8
:10AAD0001C861D861E861F86188A8295807F9B8510
:10AAE0009F70892B8B871986EE24EA94FE2C0989A6
:10AAF0001A892B893C894D895E896F89788DCE01B1
:10AB000009960E942C786DE073E186ED9BE00E942F
:10AB10005EA0CE0109960E94F233A1E0AA16B1040C
:10AB200029F0B2E0AB16B10451F025C0B88863E05B
:10AB300070E0C6010E94D75E6B2D0E94216F6F8569
:10AB4000F601848195810E94216FBE8461E070E0EE
:10AB5000C6010E94D75E6B2D0E94216FBD8462E00A
:10AB600070E0C6010E94D75E6B2D0E94216F03C06A
:10AB700080E090E002C081E090E068960FB6F89423
:10AB8000DEBF0FBECDBFDF91CF911F910F91FF9020
:10AB9000EF90DF90CF90BF90AF9008950F931F93E9
:10ABA000CF93DF93C92FD62F082F192F17FF03C07C
:10ABB00011950195110961E0802F0E94014D6C2FC4
:10ABC000DD2351F06095661F6627661F802F0E9467
:10ABD000D24C63E972E108C0661F6627661F802FAA
:10ABE0000E94D24C6EE872E186ED9BE00E945EA06E
:10ABF00086ED9BE0DF91CF911F910F910C94A351B3
:10AC0000CF936130710541F164F4672B91F5909316
:10AC1000080A8093070A50930A0A4093090A81E0C0
:10AC200024C06230710571F06330710511F59093A5
:10AC3000080A8093070A552750930A0A4093090A85
:10AC400084E013C09093080A8093070A50930A0A7D
:10AC50004093090A83E009C09093080A8093070A89
:10AC600050930A0A4093090A82E00E948FAAC82FD3
:10AC700006C069E274E186ED9BE00E945EA0CC23F1
:10AC800089F064E174E18EE29BE00E945EA04AE0FC
:10AC900050E06C2F8EE29BE00E94BF9F8EE29BE013
:10ACA0000E94A35181E0C11180E0CF9108952F92BD
:10ACB0003F924F925F926F927F928F929F92AF924C
:10ACC000BF92CF92DF92EF92FF920F931F93CF9399
:10ACD000DF93CDB7DEB7C855D1090FB6F894DEBF04
:10ACE0000FBECDBF0E94844E9B01AC016091110943
:10ACF000709112098091130990911409AA24AA94C1
:10AD0000BA2C650110E3E12E15E7F12E00E010E00A
:10AD10000E940293882309F405C2E091FE08F09195
:10AD2000FF08309709F4FEC180913A0D8F5F809340
:10AD30003A0D2680378010E02114310409F44DC00B
:10AD4000F10180858F70853009F043C060E0C1015A
:10AD50000E94A4A9FC0181859285A385B4850597ED
:10AD6000A105B105B1F58DC020E030E048E152E425
:10AD7000C301B2010E94DCC118163CF4F1016081EC
:10AD800071818AED94E00E940A7267968EAD9FAD44
:10AD90006797892B09F44AC120E030E040E85FE37F
:10ADA00065966CAD7DAD8EAD9FAD65970E9410C070
:10ADB0009B01AC01C301B2010E947DC087FF2AC183
:10ADC00061E0C4010E94CE55CE0101960E9444B0BC
:10ADD00011E0F10122803380AFCF80913A0D815094
:10ADE00080933A0D0E94844E60931109709312096A
:10ADF00080931309909314090E94A9942B013C019C
:10AE00000E94844E6B017C010E9466A8882329F071
:10AE10008091390D882309F422C11123C9F00E94C1
:10AE2000A9946B017C0162EB72E186ED9BE00E94CC
:10AE30005EA02AE030E0B701A60186ED9BE00E940B
:10AE4000B29F6BE175E086ED9BE00E94A9A06AC10C
:10AE50000E94A9946B017C0160EB72E186ED9BE09E
:10AE60000E945EA02AE030E0B701A60186ED9BE0DB
:10AE70000E94B29F6EEA72E186ED9BE00E945EA0A6
:10AE800051C13A8229821B861A86CE0101960E9400
:10AE900053B0CE0101960E945BAE882309F4DAC05C
:10AEA00025961CAE1DAE1EAE1FAE259729961CAE74
:10AEB0001DAE1EAE1FAE299740E0BE016F5F7F4FF3
:10AEC000CE018F5B9F4F0E949D34CE0101960E9460
:10AED00007AF6B017C0168966FAF68976996DFAE2C
:10AEE000699760E070E0CE0101960E9422AF4C01AC
:10AEF000CE018F5B9F4F0E94153765966CAF7DAF7B
:10AF00008EAF9FAF6597CE0101960E9437B0182F84
:10AF1000B601DD0C880B990B0E942CC120E030E0BB
:10AF200048EC52E40E9482C02B013C01CE01019604
:10AF30000E94594567969FAF8EAF67976DEE72E19D
:10AF400086ED9BE00E945EA022E065964CAD5DAD73
:10AF50006EAD7FAD659786ED9BE00E942E7567EE26
:10AF600072E186ED9BE00E945EA022E0B301A201A7
:10AF700086ED9BE00E942E7561EE72E186ED9BE00E
:10AF80000E945EA0612F70E04AE050E086ED9BE0F9
:10AF90000E9415A0E114F10409F455C088E00E9454
:10AFA000EC929B01AC0144275527B70180E090E06B
:10AFB000AA24AA94BA2CC12CD12C11EAE12E17E0B4
:10AFC000F12E00E010E00E940293882309F4CCCE19
:10AFD000F101608171818EE29BE00E94A9A061ED88
:10AFE00072E18EE29BE00E945EA0F10160817181BE
:10AFF00080ED95E00E940A7280E090E0BC016896C6
:10B000004FAD689769965FAD6997CE0101960E9432
:10B01000A9AE0CC0A301920165966CAD7DAD8EAD5D
:10B020009FAD65970E947DC0181614F060E0C9CEF0
:10B0300062EC72E186ED9BE00E945EA086ED9BE0F3
:10B040000E94A351C1CE68EB72E186ED9BE00E94A5
:10B050005EA0BACECE0101960E9444B0BACE20E0E6
:10B0600030E041E050E060E4CE0101960E94B893E8
:10B0700040E450E067EA72E1CE0101960E94EAB72F
:10B0800068EA74E0CE0101960E946FC440E450E08B
:10B090006EE972E1CE0101960E94EAB7B301A20106
:10B0A000CE018F5B9F4F0E945D93BE016F5B7F4F10
:10B0B000CE0101960E9488A920E030E041E050E0F6
:10B0C00060E4CE0101960E94B89340E450E067EA44
:10B0D00072E1CE0101960E94EAB768EA74E0CE01FF
:10B0E00001960E946FC440E450E067E972E1CE012E
:10B0F00001960E94EAB7C701B60128EE33E040E0AE
:10B1000050E00E9467BFBA01A901CE018F5B9F4F3B
:10B110000E945D93BE016F5B7F4FCE0101960E943E
:10B1200088A97BCEC85ADF4F0FB6F894DEBF0FBE9A
:10B13000CDBFDF91CF911F910F91FF90EF90DF90E6
:10B14000CF90BF90AF909F908F907F906F905F90C7
:10B150004F903F902F900895FC0122813381232B43
:10B1600049F0868197818130910549F01CF0039761
:10B17000029718F080E090E0089582E090E0089552
:10B1800081E090E00895CF93DF93CDB7DEB760976D
:10B190000FB6F894DEBF0FBECDBF19821A821B8294
:10B1A0001C821D821E821F8218868B818F70806197
:10B1B0008B836FEF3E819F81888529817A815B81B6
:10B1C0004C814C873E87888B372F452F5C857E8549
:10B1D000892F988960960FB6F894DEBF0FBECDBF59
:10B1E000DF91CF9108958F929F92AF92BF92CF92AD
:10B1F000DF92EF92FF920F931F93CF93DF93E09133
:10B20000FE08F091FF08309709F469C0812EF02EF6
:10B21000932EC22EA52ED42EB72EE62EBC01CF0122
:10B220000E94EC5EEC01892B09F45CC088858F706C
:10B23000853009F057C060E0CE010E94A4A98C01BE
:10B2400061E0CE010E94A4A9FC01C185D285D8018C
:10B2500019962D913C911A972130310571F034F4F3
:10B26000232B09F03FC06F2DCE0118C022303105CD
:10B2700049F027303105A9F035C06F2DCE01039676
:10B280000E94216F6E2DCE010E94216F6D2DCE0187
:10B2900001960E94216F6C2DCE0102960E94216FB3
:10B2A00021C0892BF9F080858F708530D9F4C68153
:10B2B000D7812097B9F088858F70843061F40F2D85
:10B2C000182D2C2D392D4D2D5A2D6E2D7B2D898528
:10B2D0009A850E94F3580A80DB81C02DEACF80E076
:10B2E00090E002C081E090E0DF91CF911F910F913B
:10B2F000FF90EF90DF90CF90BF90AF909F908F9096
:10B300000895CF92DF92EF92FF920F931F93CF9306
:10B31000DF93E091F108F091F2083097C9F0908541
:10B320009F709530A9F469017A01EB01682FCF0174
:10B330000E94A4A9FC0190859F70943049F48185F6
:10B340009285009729F09601A701BE010E94F3584B
:10B35000DF91CF911F910F91FF90EF90DF90CF90F1
:10B360000895AF92BF92CF92DF92EF92FF920F9328
:10B370001F93CF93DF938091EE089091EF08892B74
:10B3800009F46DC0E1E0F0E0C0E0D0E0CC24C3946B
:10B39000D12CB6010C2E02C0660F771F0A94E2F77B
:10B3A00040911B0950911C097F0184E0E80EF11CBB
:10B3B000CF01B12C9C01A0910602B0910702A81701
:10B3C000B90720F42091060230910702A091B40D34
:10B3D000B091B50DA20FB31FAC90A091EE08B09143
:10B3E000EF089C0121503109A20FB31F0A2D10E074
:10B3F0002C9130E00217130729F0462B572BAC9203
:10B40000BB24B3940196E816F906A1F650931C09E3
:10B4100040931B09BB20E9F08091EE089091EF0862
:10B42000E80FF91F028110E0218130E0408150E0F7
:10B430003197608170E0CE010E94815980E00E94C6
:10B44000EC926093170970931809809319099093EF
:10B450001A092196F701C430D10509F09ACFDF917E
:10B46000CF911F910F91FF90EF90DF90CF90BF9001
:10B47000AF900895AF92BF92CF92EF92FF920F9349
:10B480001F93CF93DF93CDB7DEB728970FB6F8940D
:10B49000DEBF0FBECDBF5C0109831A832B833C83C3
:10B4A0004D835E836F83788761E774E186ED9BE06F
:10B4B0000E945EA0CE0101960E94F2336981611163
:10B4C00014C00B810F70013081F030F0023031F088
:10B4D000053021F010E06EC0CC24C394D501ED916D
:10B4E000FC91068CF78DE02D45C0F501828193819A
:10B4F0000E940CB019811130A9F0123009F047C038
:10B500001D821E821F821886D501ED91FC91068C4A
:10B51000F78DE02DCC24C39402E01A812B813C816D
:10B5200040E02DC0CE0101960E94B1A94997D4F404
:10B5300059C0873008F065C08150823010F486E62B
:10B540008D83D50112966D917C91139740E0CE01C9
:10B5500001960E94453460E07AE0F5018281938192
:10B560000E94703FD501ED91FC91068CF78DE02D86
:10B57000CC24C39409811A812B813C814D815E8149
:10B580006F817885C501199581E090E04EC064E631
:10B5900074E186ED9BE00E945EA04AE050E0612FDE
:10B5A00086ED9BE00E94BF9F86ED9BE00E94A35129
:10B5B00001E010E064E574E186ED9BE00E945EA08E
:10B5C0004AE050E0B80186ED9BE00E9415A086EDB0
:10B5D0009BE00E94A351CE0101960E94F23380E0CD
:10B5E00090E023C08B8182958F70863009F0A1CFC7
:10B5F0008CEF93E0A0E0B0E08D839E83AF83B887AB
:10B60000A0CF873049F480E090E0ACECB2E48D83C9
:10B610009E83AF83B88795CF8A50823008F091CF50
:10B6200086E690E0A0E0B0E0E7CF28960FB6F89469
:10B63000DEBF0FBECDBFDF91CF911F910F91FF9065
:10B64000EF90CF90BF90AF900895FC0182819381DD
:10B65000009719F062E00E940CB008950F931F93B9
:10B66000CF93DF93CDB7DEB728970FB6F894DEBF40
:10B670000FBECDBF19821A821B821C821D821E82C0
:10B680001F8218862B812F702B831982FC01028167
:10B690001381C8010E9437B0823071F0853061F0AB
:10B6A00040E0B801CE0101960E949D3460E0CE01D9
:10B6B00001960E94523602C080E090E028960FB6B4
:10B6C000F894DEBF0FBECDBFDF91CF911F910F91D8
:10B6D0000895CF92DF92EF92FF920F931F93CF9333
:10B6E000DF93CDB7DEB7C054D1090FB6F894DEBFF3
:10B6F0000FBECDBF8091FC089091FD08059789F1A0
:10B700006115710571F169017A018B0140E450E026
:10B71000CE0101960E94B3C46FE270E0CE010196A3
:10B720000E947AC4892B41F4980143E050E060E420
:10B73000CE0101960E94B89340E450E0B601CE01DC
:10B7400001960E9495C40E9466A8882351F08091BA
:10B75000FC089091FD08069721F48091390D88230B
:10B7600019F080E090E007C0B701CE0101960E9479
:10B7700088A981E090E0C05CDF4F0FB6F894DEBF8F
:10B780000FBECDBFDF91CF911F910F91FF90EF9032
:10B79000DF90CF900895CF92DF92EF92FF920F93B8
:10B7A0001F93CF93DF93CDB7DEB760970FB6F894B2
:10B7B000DEBF0FBECDBF7C016B01CA01B901AE0176
:10B7C0004F5F5F4F0E945294D701ED91FC91028828
:10B7D000F389E02D9801AE014F5F5F4FB601C701BD
:10B7E000199560960FB6F894DEBF0FBECDBFDF91FE
:10B7F000CF911F910F91FF90EF90DF90CF90089520
:10B80000CF92DF92EF92FF920F931F93CF93DF932C
:10B81000CDB7DEB760970FB6F894DEBF0FBECDBFD1
:10B820007C016B01BA01A901CE0101960E945D93D2
:10B83000D701ED91FC910288F389E02D9801AE01CA
:10B840004F5F5F4FB601C701199560960FB6F89428
:10B85000DEBF0FBECDBFDF91CF911F910F91FF9043
:10B86000EF90DF90CF900895AF92BF92CF92DF928A
:10B87000EF92FF920F931F93CF93DF93CDB7DEB775
:10B8800028970FB6F894DEBF0FBECDBF6C01162F00
:10B890005A01DC018D919C911197892B09F442C1C9
:10B8A0001496ED91FC911597309709F43BC1808176
:10B8B0006F3FB9F484FF34C14330510509F430C1FE
:10B8C000118112951F7068E874E186ED9BE00E947B
:10B8D0005EA04AE050E0612F86ED9BE00E94BF9F92
:10B8E00002C084FD1FC1D6011496ED91FC911597FD
:10B8F00001810F70101769F11396FC9066E874E1EE
:10B9000086ED9BE00E945EA04AE050E06F2D86ED40
:10B910009BE00E94BF9F64E874E186ED9BE00E947B
:10B920005EA04AE050E0602F86ED9BE00E94BF9F42
:10B9300061E874E186ED9BE00E945EA04AE050E081
:10B94000612F86ED9BE00E94BF9F86ED9BE00E94E9
:10B95000A351812F90E08D30910508F09CC0FC012F
:10B96000D6011496ED90FC9015978827E05FFE4F66
:10B970008F4F0C94DEBFF7019181292F2F70253056
:10B9800009F489C0D6018D919C91263048F422306B
:10B99000A9F46DED75E00E94EC5EF701608159C07D
:10B9A000273049F02A3051F463EE75E00E94EC5ED6
:10B9B000F70160816BC06CED75E055C06AEE75E013
:10B9C00038C06FEE75E0D6018D919C910E94EC5EBF
:10B9D000F7012081622F6170322F309530FB20F902
:10B9E00021C064EF75E0D6018D919C910E94EC5EC0
:10B9F000F701208121FB662760F931E0362730FB13
:10BA000021F910C06AEF75E0D6018D919C910E94DA
:10BA1000EC5EF701208122FB662760F931E03627D2
:10BA200030FB22F9208335C06AEE75E0D6018D9196
:10BA30009C910E94EC5E60E02CC060E076E002C069
:10BA400065E076E0F601808191810E94EC5ED7018D
:10BA50006C9161701EC06BE076E002C061E176E03F
:10BA6000F601808191810E94EC5ED7016C91669510
:10BA700061700FC068E176E002C06EE176E0F60129
:10BA8000808191810E94EC5ED7016C9162FB6627F8
:10BA900060F9009759F4D6011496ED91FC91159731
:10BAA0001F708181807F182B11833AC0D6011496B4
:10BAB000ED91FC911597B3E0AB16B10411F11F7035
:10BAC0002181207F122B118319821A821B821C82F2
:10BAD0001D821E821F8218860B810F700B831982B4
:10BAE000E12CFA801C8120E03E814F8158850E9424
:10BAF0004395D6011496ED91FC91159780818F7E28
:10BB00000EC081818F70982F9295907F892B8183B1
:10BB1000D6011496ED91FC91159780818061808308
:10BB200081E001C080E028960FB6F894DEBF0FBE1A
:10BB3000CDBFDF91CF911F910F91FF90EF90DF90DC
:10BB4000CF90BF90AF900895EF92FF920F931F9305
:10BB5000CF93DF93EC018B011D821C821A821B8222
:10BB6000E880F980E114F10409F464C08091290DA2
:10BB700090912A0D892B09F45DC0672B09F4870188
:10BB8000F80180858F708630D1F465E276E0C801D7
:10BB90000E94EC5E009719F0FC0181858A8366EAB9
:10BBA00074E0C8010E94EC5E009719F0FC018185E9
:10BBB00005C0F801808191810E94AAB78B8367E25A
:10BBC00076E0C7010E94EC5E009789F51A810B812F
:10BBD0006CE774E186ED9BE00E945EA04AE050E0D5
:10BBE000602F86ED9BE00E94BF9F6AE774E186EDBF
:10BBF0009BE00E945EA04AE050E0612F86ED9BE052
:10BC00000E94BF9F86ED9BE00E94A35120E030E0A0
:10BC1000A90167E276E0888199810E9450AA67E2D3
:10BC200076E0888199810E94EC5E009719F0099670
:10BC30009D838C83DF91CF911F910F91FF90EF90A7
:10BC400008954F925F926F927F92AF92BF92CF9280
:10BC5000DF92EF92FF920F931F93CF93DF93809128
:10BC60001B0990911C09C4E0D0E021E030E0AC0158
:10BC700042235323452B29F0A90140955095842355
:10BC80009523220F331F219791F790931C098093DE
:10BC90001B0940901709509018096090190970907D
:10BCA0001A09411451046104710409F471C00E941D
:10BCB000844E9B01AC01AA24AA94BA2C65011CE213
:10BCC000E12EFF24F39400E010E0C301B2010E94D2
:10BCD0000293882309F45CC0109217091092180986
:10BCE0001092190910921A09E12CF12CE091EE083A
:10BCF000F091EF08EC0FFD1F038110E0228130E08E
:10BD0000418150E0608170E0C7010E9481598FEF4E
:10BD1000E81AF80A249684E0E816F10439F7C1E03D
:10BD2000D0E080910602909107028C179D0728F4BD
:10BD3000809106029091070201C0CE012091B40DBE
:10BD40003091B50DF901E80FF91F4AE050E060812C
:10BD500089E39BE00E94BF9F6AE276E089E39BE073
:10BD60000E94A9A02196C131D105D9F689E39BE0B3
:10BD7000DF91CF911F910F91FF90EF90DF90CF90C7
:10BD8000BF90AF907F906F905F904F900C94A351B5
:10BD9000DF91CF911F910F91FF90EF90DF90CF90A7
:10BDA000BF90AF907F906F905F904F900895FC018F
:10BDB0006115710519F484819581089586819781B3
:10BDC000681779072CF084819581860F971F089555
:10BDD000828193810C9422AF0F931F93CF93DF93B3
:10BDE0008B01FC01C681D781209759F0B801888169
:10BDF00099810E945CC4892B21F00A80DB81C02DCF
:10BE0000F3CFCE01DF91CF911F910F9108956F92E3
:10BE10007F928F929F92AF92BF92CF92DF92EF92DA
:10BE2000FF920F931F93CF93DF93CDB7DEB7C85424
:10BE3000D1090FB6F894DEBF0FBECDBF3C014B0158
:10BE4000FC01E080F1806CE276E0C7010E94EC5ECC
:10BE50005C0161E376E0C7010E94EC5E6C01A11415
:10BE6000B10419F4892B09F4F9C06FEE75E0C7012C
:10BE70000E94EC5E8C016AEE75E0C7010E94EC5EE8
:10BE80007C01F301738062EA74E186ED9BE00E941D
:10BE90005EA04AE050E0672D86ED9BE00E94BF9FC8
:10BEA00060EA74E186ED9BE00E945EA04AE050E00B
:10BEB000B40186ED9BE00E9415A086ED9BE00E94F8
:10BEC000A351C114D104E1F1F60180858F70843053
:10BED000B9F56185728540E450E0CE0101960E947B
:10BEE000B3C40E9466A8882359F18091390D81114D
:10BEF00027C06FE270E0CE0101960E947AC4892BC0
:10BF000051F4F6012185328543E050E060E4CE0132
:10BF100001960E94B8938114910409F48DC0011513
:10BF2000110509F486C0F80180858F70843009F00E
:10BF300080C0F80161857285FB018081811189C013
:10BF4000A114B10409F48AC0F50180858F70843092
:10BF500009F084C061857285CE0101960E94F2B01D
:10BF6000CE0101960E945BAE882309F45DC089284A
:10BF7000F1F00115110529F0F80180858F708430EA
:10BF8000A1F025961CAE1DAE1EAE1FAE25972996BC
:10BF90001CAE1DAE1EAE1FAE299724962FAD249762
:10BFA0002F70E12CF12C01E01DC0F80131C0E1142B
:10BFB000F10429F0F70180858F70843041F12596D6
:10BFC0001CAE1DAE1EAE1FAE259729961CAE1DAE33
:10BFD0001EAE1FAE299724962FAD24972F70E12C0B
:10BFE000F12C02E023961FAD239725963FAD2597B0
:10BFF00040E027965FAD279728966FAD2897299642
:10C000007FAD2997CE0101960E94FD180DC0F70162
:10C0100061857285FB018081882331F040E050E02A
:10C02000CE0101960E944772CE0101960E9444B053
:10C0300015C066E376E00DC0E114F10429F0F701C4
:10C0400080858F70843019F069E376E002C0F701D3
:10C0500071CFCE0101960E9488A972CFC85BDF4FD5
:10C060000FB6F894DEBF0FBECDBFDF91CF911F9109
:10C070000F91FF90EF90DF90CF90BF90AF909F9087
:10C080008F907F906F9008952F923F924F925F9282
:10C090006F927F928F929F92AF92BF92CF92DF92D8
:10C0A000EF92FF920F931F93CF93DF93CDB7DEB73D
:10C0B000C555D1090FB6F894DEBF0FBECDBF4C01F8
:10C0C0003B01DC0112968C91803499F128F0823486
:10C0D00081F108F455C58058843008F051C5F40149
:10C0E00084819581892B09F44BC5A3016FEFC401AD
:10C0F0000E94345CD40112961C911297169511700F
:10C1000013960C9113978AEC800F803108F071C15F
:10C110006DE376E08D919C910E94EC5E7C0100972E
:10C1200009F467C1FC0180858F70853009F061C119
:10C1300023C16DE376E0D4018D919C910E94EC5E69
:10C140008C01F401838190911D0C981309C090918A
:10C150001E0C903429F480911F0C9091200C0BC080
:10C1600080931D0C90E490931E0C0E94064E9093B9
:10C17000200C80931F0C3C010115110509F4E7C048
:10C18000D80118962C912F70253009F0E0C0C80115
:10C190000E9425AA64968FAF6497843008F46BC020
:10C1A00063E0C8010E94A4A9FC01818592853AE060
:10C1B000D32ED89E9001D99E300D112463963FAFA7
:10C1C0002EAF639762E0C8010E94A4A9DC01199612
:10C1D0008D919C911A97D89E7001D99EF00C1124D4
:10C1E00057010F2C000CCC08DD0861E0C8010E944B
:10C1F000A4A966969FAF8EAF669760E0C8010E94C3
:10C20000A4A9FC012184328443845484C301072CF3
:10C21000000CAA0BBB0B9C01AD0122193309440988
:10C22000550963966EAD7FAD6397CB01770FAA0B6F
:10C23000BB0BBC01CD016A197B098C099D090E94C9
:10C2400057BF6696AEADBFAD669719962D913D91DD
:10C250004D915C911C9722193309440955090E949C
:10C2600089BFA20EB31EC41ED51E6496BFAD6497CF
:10C27000B53099F415C08AE0869D5001879DB00CB9
:10C2800011240B2C000CCC08DD08E12CF12CE0E093
:10C29000F8E26396FFAFEEAF639781E090E009C0EC
:10C2A00064E0C8010E94A4A9DC0119968D919C91BB
:10C2B0001A976396EEADFFAD6397AF01FF0F660B64
:10C2C000770B4A155B056C057D0534F45A016B014B
:10C2D00066246A9423E0722EA7010F2C000C660BD3
:10C2E000770BA416B506C606D70624F45A016B01CF
:10C2F000612C712C6496FFAD6497F23009F0DEC2B8
:10C300006301770CEE08FF0860E0C8010E94A4A951
:10C31000FC0181859285A385B485C816D906EA06F5
:10C32000FB060CF406C461E0C8010E94A4A9FC014C
:10C3300081859285A385B4858C159D05AE05BF05C5
:10C340000CF01EC4C12CD12C7601C394F5C32AE095
:10C35000289F5001299FB00C11240B2C000CCC08F5
:10C36000DD08E12CF12C20E038E263963FAF2EAFE0
:10C37000639781E090E0A2C280911D0C801309C0F8
:10C3800080911E0C803429F480911F0C9091200C18
:10C390000CC000931D0C80E480931E0C802F0E9423
:10C3A000064E9093200C80931F0C5C01990FCC08D3
:10C3B000DD0860E0C7010E94A4A9FC018185928587
:10C3C000A385B485A816B906CA06DB060CF43CC0E2
:10C3D00061E0C7010E94A4A955245394FC01818502
:10C3E0009285A385B4858A159B05AC05BD056CF5C2
:10C3F0002BC0202F30E0F901E85BFD4E8491F9015C
:10C40000E25DFA4E0491F901EC58FA4EF490FF20E7
:10C4100009F43DC281110E947C4CEF2DF0E0EE0F3B
:10C42000FF1FED54FB4EA591B491EC910E2331E02A
:10C4300020E009F430E0832F922F212F30E05524A3
:10C4400053942817390709F0512CD4011496ED9113
:10C45000FC9115978181E82FEF708E2F90E0FC0101
:10C460003197EC30F10508F08FC18827E35EFE4F6D
:10C470008F4F0C94DEBF0E94844E9B01AC01442779
:10C480005527D4011496ED91FC91159782819381E3
:10C49000BC0180E090E0AA24AA94BA2CC12CD12C33
:10C4A00018EEE12E13E0F12E00E010E00E9402935E
:10C4B000882309F469C1F4010081118160E076E00C
:10C4C000C8010E94EC5E892B09F0E4C165E076E0CA
:10C4D000C8010E94EC5E892B09F0DCC1E4C00E9417
:10C4E000844E9B01AC0144275527D4011496ED914D
:10C4F000FC91159782819381BC0180E090E0AA2491
:10C50000AA94BA2CC12CD12C1CE2E12EFF24F39466
:10C5100000E010E01AC00E94844E9B01AC01442749
:10C520005527D4011496ED91FC9115978281938142
:10C53000BC0180E090E0AA24AA94BA2CC12CD12C92
:10C5400016E9E12EF12C00E010E00E94029388230E
:10C5500009F41AC1A30164E0E5C00E94844E9B0166
:10C56000AC0144275527D4011496ED91FC91159701
:10C5700082819381BC0180E090E0AA24AA94BA2C25
:10C58000C12CD12C18EEE12E13E0F12E00E010E0CA
:10C590000E940293882309F4F7C0F40100811181FD
:10C5A0006BE076E0C8010E94EC5E892B09F075C152
:10C5B00061E176E0C8010E94EC5E892B09F06DC153
:10C5C00072C00E94844E9B01AC0144275527D401C0
:10C5D0001496ED91FC91159782819381BC0180E0C6
:10C5E00090E0AA24AA94BA2CC12CD12C1CE2E12EF2
:10C5F000FF24F39400E010E01AC00E94844E9B01D7
:10C60000AC0144275527D4011496ED91FC91159760
:10C6100082819381BC0180E090E0AA24AA94BA2C84
:10C62000C12CD12C16E9E12EF12C00E010E00E9483
:10C630000293882309F4A8C0A30169E073C00E9493
:10C64000844E9B01AC0144275527D4011496ED91EB
:10C65000FC91159782819381BC0180E090E0AA242F
:10C66000AA94BA2CC12CD12C18EEE12E13E0F12E95
:10C6700000E010E00E940293882309F485C0F401D1
:10C680000081118168E176E0C8010E94EC5E892B8F
:10C6900009F006C16EE176E0C8010E94EC5E892BCC
:10C6A00009F0FEC000C1A3016DE06BC00E94844E82
:10C6B0009B01AC0144275527D4011496ED91FC91C0
:10C6C000159782819381BC0180E090E0AA24AA940E
:10C6D000BA2CC12CD12C1CE2E12EFF24F39400E0F3
:10C6E00010E01AC00E94844E9B01AC0144275527DC
:10C6F000D4011496ED91FC91159782819381BC0130
:10C7000080E090E0AA24AA94BA2CC12CD12C16E97E
:10C71000E12EF12C00E010E00E9402938823A1F1A9
:10C72000A3016CE0C4010E94345CF4010481158112
:10C730000E94844ED80113967C936E93129724C066
:10C740000E94844E9B01AC0144275527D4011496C6
:10C75000ED91FC91159782819381BC0180E090E07E
:10C76000AA24AA94BA2CC12CD12C18E5E12E12E0EF
:10C77000F12E00E010E00E940293882329F0A3012B
:10C7800060E0C4010E94345CF40104811581D80189
:10C790008C9183FB992790F9951509F473C0982F14
:10C7A000907E39F0982F907E90528F71892B8C93C8
:10C7B000E7C10E94844EF80173836283D40112960C
:10C7C0008C91129780FF15C0552009F4D9C1149699
:10C7D000ED91FC9115978081886080831496ED918E
:10C7E000FC9115976081617070E0C4010E94075F41
:10C7F000C7C1652D70E0C4010E94075FD401149683
:10C80000ED91FC9115978181552099F08F708230C0
:10C8100069F028F481112DC0A30161E024C08530A6
:10C8200029F0873031F5A3016AE01DC0A30166E05D
:10C830001AC0E82FEF708E2F90E0FC013197ED3099
:10C84000F105B8F48827E75DFE4F8F4F0C94DEBFEB
:10C85000A30162E008C0A30165E005C0A30167E091
:10C8600002C0A30160E0C4010E94345C882309F483
:10C8700087C1D4011496ED91FC911597808150FAEF
:10C8800083F903C08F718066F801808379C180E0ED
:10C8900090E0D3CDA30163E074CFA30168E071CF32
:10C8A000A3016BE06ECF6AEF75E0C8010E94EC5EF9
:10C8B000892B09F0F8CEA30166E063CFD40114966A
:10C8C000ED91FC91159722813381A301421B530BFB
:10C8D0009A0157FF03C031952195310982179307BB
:10C8E0001CF480818F7112C04081842F82958695BF
:10C8F0008770282F30E0263031054CF48F5F982F59
:10C900009295990F907E842F8F71892B8083D4010B
:10C910001496ED91FC91159780818295869587708C
:10C9200090E00597BCF0C701FF0CAA0BBB0BA81643
:10C93000B906CA06DB0671F063962EAD3FAD63976C
:10C94000C901330FAA0BBB0BA816B906CA06DB0632
:10C9500009F016C1828193818615970509F410C1EB
:10C96000C601B5010E942CC120E030E040E251E454
:10C970000E9482C0D62EC72EB82EA92ED40113969F
:10C980001C916FEA74E186ED9BE00E945EA04AE094
:10C9900050E0612F86ED9BE00E94BF9F6DEA74E13D
:10C9A00086ED9BE00E945EA022E04D2D5C2D6B2D5C
:10C9B0007A2D86ED9BE00E942E7586ED9BE00E940D
:10C9C000A35169EB74E0F401808191810E94EC5ED7
:10C9D00019821A821B821C820B810F7000670B83E5
:10C9E0002D2D4D2D5C2D6B2D7A2D4D835E836F8308
:10C9F0007887E980FA801C813E814F8158856FEFEE
:10CA00000E944395D4010D911C916CE276E0C8011F
:10CA10000E94EC5E7C0161E376E0C8010E94EC5E5E
:10CA20008C01009799F1FC0180858F70843071F53D
:10CA30006185728540E450E0CE0101960E94B3C446
:10CA40006FE270E0CE0101960E947AC4892B61F4F6
:10CA5000D80119962D913C911A9743E050E060E47B
:10CA6000CE0101960E94B893AE014F5B5F4F6D2DD2
:10CA70007C2D8B2D9A2D0E9452940E9466A88823AB
:10CA800029F08091390D882309F472C0E114F10472
:10CA900009F447C0F70180858F70843009F041C0E8
:10CAA00061857285CE0101960E94F2B0CE01019699
:10CAB0000E945BAE882389F125961CAE1DAE1EAE8A
:10CAC0001FAE259724962FAD24972F7020672496AC
:10CAD0002FAF24974D2D8D2D9C2DAB2DBA2D299642
:10CAE0008CAF9DAFAEAFBFAF2997E12CF12C229652
:10CAF0000FAD229723961FAD239725963FAD25971F
:10CB000027965FAD279728966FAD289729967FAD1A
:10CB10002997CE0101960E94FD18CE0101960E9430
:10CB200044B0D4011496ED91FC9115977382628202
:10CB300027C0C12CD12C7601D4011496ED91FC9123
:10CB4000159782819381092E000CAA0BBB0B8C15C3
:10CB50009D05AE05BF05A1F0B601C4010E94075FA7
:10CB6000D4011496ED91FC911597D382C28208C02E
:10CB7000BE016F5B7F4FCE0101960E9488A986CFD0
:10CB800080E090E0CB5ADF4F0FB6F894DEBF0FBEC7
:10CB9000CDBFDF91CF911F910F91FF90EF90DF906C
:10CBA000CF90BF90AF909F908F907F906F905F904D
:10CBB0004F903F902F9008954F925F926F927F9287
:10CBC0008F929F92AF92BF92CF92DF92EF92FF929D
:10CBD0000F931F93CF93DF93CDB7DEB768970FB650
:10CBE000F894DEBF0FBECDBF6C018A015901DC0194
:10CBF00014968D919C911597DC011F968D919C91B7
:10CC00005097DC011696ED90FC9017972B01770F4B
:10CC100066087708E114F10409F464C1B2E0AB16C8
:10CC2000B10439F083E0A816B10449F465E476E074
:10CC300002C061E476E0C7010E94EC5EFC0130971F
:10CC400009F44AC181859285A385B485841595052B
:10CC5000A605B70509F040C168E476E0C7010E9467
:10CC6000EC5E5C016DE376E0C7010E94EC5ED601EC
:10CC70001296ED91FC91139762E0828193810E945C
:10CC8000A4A96C01003448F4F801FF27EE0FFF1F40
:10CC9000EC5FF54F0781108502C00FEF1FEF198A77
:10CCA0001A8A1B8A1C8A1D8A1E8A1F8A188E8B89E3
:10CCB0008F708B8B198AA114B10409F43DC0F50162
:10CCC00080858F708430C1F5818492849DECA92E7B
:10CCD00094E1B92E612C712C81149104D1F0B5012D
:10CCE000C4010E94D1B7892B51F485E0869DF001E3
:10CCF000879DF00D1124EF52FB4E64910CC0FFEFA5
:10CD00006F1A7F0A85E0A80EB11CA9E06A167104AB
:10CD100019F761E070E0B62E862F660F990BAA0B0B
:10CD2000BB0BFC013197E930F10590F58827EA5CEF
:10CD3000FE4F8F4F0C94DEBF8B898F70806A8B8B78
:10CD400020E030E00D8B1E8B2F8B388FBB24B394EB
:10CD50001FC08B898F70806A14C08B898F70806B25
:10CD600010C08B898F70806B8B8B11270BC08B89C8
:10CD70008F70806B8B8B102F002704C08B898F7076
:10CD800080668B8B20E030E00D8B1E8B2F8B388FD5
:10CD9000F701808091800FEF10E020E033E040E168
:10CDA00050E0BE016F5F7F4FCE0141960E943A3244
:10CDB0008C016CE075E186ED9BE00E945EA0B801FD
:10CDC00086ED9BE00E94A9A065E075E186ED9BE001
:10CDD0000E945EA06B2DBB0C770B4AE050E086ED05
:10CDE0009BE00E9415A063E075E186ED9BE00E9448
:10CDF0005EA0B40186ED9BE00E94A9A086ED9BE0B9
:10CE00000E94A351C114D10409F463C0D60118963D
:10CE10008C918F70863009F05CC0F701E080F18062
:10CE2000B701C6010E94EC5E6C01009709F451C085
:10CE300067E276E00E94EC5E8C010097E9F0DC018D
:10CE400019968D909D90AD90BC901C976989662332
:10CE500021F070E080E090E004C0CE0141960E9495
:10CE6000533786169706A806B90699F1F801618727
:10CE700072878387948721C06AEF74E186ED9BE017
:10CE80000E945EA0B70186ED9BE00E94A9A086EDFE
:10CE90009BE00E94A3512989222321F030E040E049
:10CEA00050E006C0CE0141960E9453379B01AC0171
:10CEB00067E276E0C6010E9450AAE988FA880B89E9
:10CEC0001C892D893E894F89588D6FEFC6010E94BC
:10CED000439581E090E008C0D7011296ED90FC9058
:10CEE000139798CE80E090E068960FB6F894DEBF76
:10CEF0000FBECDBFDF91CF911F910F91FF90EF90AB
:10CF0000DF90CF90BF90AF909F908F907F906F9069
:10CF10005F904F9008952F923F924F925F926F9241
:10CF20007F928F929F92AF92BF92CF92DF92EF92B9
:10CF3000FF920F931F93CF93DF9300D000D0CDB714
:10CF4000DEB78C010E9453B72FEC37E040E050E091
:10CF50000E9489BFDC01CB010196A11DB11DF80122
:10CF600084839583A683B78380839183A283B383CD
:10CF70005801F3E4AF0EB11CC5010E942A8C64E491
:10CF800070E0C5010E94368E882309F436C10E94E4
:10CF9000844E2B013C01812C912CC8018E5B9F4F4C
:10CFA0009E838D8348EEC42E43E0D42EE12CF12CD9
:10CFB00052E0252EAD81BE818C91833009F404C1ED
:10CFC000811120C0F80184819581A681B7810196E5
:10CFD000A11DB11D84839583A683B7830E94844ECF
:10CFE0006419750986099709A70196010E9467BF10
:10CFF000A90161E0C8010E946C9B81E0AD81BE8106
:10D000008C93CAC08430F9F4F80184819581A6819B
:10D01000B7810196A11DB11D84839583A683B78333
:10D020000E94844E6419750986099709A701960123
:10D030000E9467BFA90163E0C8010E946C9BAD819B
:10D04000BE812C92A9C0813059F5F80142AD53AD93
:10D0500064AD75AD9E012F5F3F4FC8010E94749C67
:10D06000382EF2E08F1392C089819A81AB81BC8106
:10D07000F80184839583A683B7830E94844E641944
:10D08000750986099709A70196010E9467BFA90142
:10D0900063E0C8010E946C9BAD81BE813C927CC064
:10D0A000823009F079C0F80142AD53AD64AD75AD81
:10D0B0009E012F5F3F4FC8010E94749C382EF5E0FF
:10D0C0008F135DC0E3E0AD81BE81EC93F80182A1D6
:10D0D00093A1A4A1B5A1892B8A2B8B2B41F484E8C1
:10D0E00093E0A0E0B0E082A393A3A4A3B5A3F801CA
:10D0F00086A197A1A0A5B1A5892B8A2B8B2B61F4C2
:10D1000082A193A1A4A1B5A1B695A795979587955E
:10D1100086A397A3A0A7B1A7F80182A593A5A4A56C
:10D12000B5A5892B8A2B8B2BA9F482A193A1A4A14D
:10D13000B5A1AC01BD0123E076956795579547955C
:10D140002A95D1F7841B950BA60BB70B82A793A743
:10D15000A4A7B5A7F80186A197A1A0A5B1A586A708
:10D1600097A7A0ABB1AB82A593A5A4A5B5A582ABAB
:10D1700093ABA4ABB5AB88248394912C0DC0F6E09F
:10D180008F1304C0AD81BE811C9206C0BFEF3B125D
:10D1900003C0ED81FE811082F1E08F16910409F445
:10D1A00009CF0E94844EDC01CB0184199509A609A0
:10D1B000B709F80126A937A940AD51AD281739079D
:10D1C0004A075B0708F0F6CEC5010E942A8CF801D9
:10D1D00084819581A681B7810196A11DB11D8483AB
:10D1E0009583A683B7830E94844EF801FE966083E0
:10D1F000718382839383C40102C080E090E026960D
:10D200000FB6F894DEBF0FBECDBFDF91CF911F9157
:10D210000F91FF90EF90DF90CF90BF90AF909F90D5
:10D220008F907F906F905F904F903F902F900895D8
:10D230000F931F93CF93DF93EC010091E3091091BB
:10D24000E409B8010E941BB8209709F440C0099670
:10D2500008171907E0F10E9466A88823C1F18091A0
:10D26000E9099091EA09019611F481E090E0909328
:10D27000EA098093E909E091E109F091E2098091DE
:10D28000EA098583E091E109F091E2098091E909D9
:10D2900086836091E1097091E20947E050E0CE0198
:10D2A0000E949DA8E091E109F091E209E80FF91FC1
:10D2B0001082AC01445051096091E1097091E2097A
:10D2C00082E8DF91CF911F910F910C94BDA880E06F
:10D2D000DF91CF911F910F9108951F93CF93DF930B
:10D2E0001F921F92CDB7DEB76CE271E080E090E054
:10D2F0000E944A4E1FB7F8948091D00C811127C02C
:10D30000E9EAF5E18491E3E6F5E19491E82FF0E0B4
:10D31000EE0FFF1FEC5EFA4EA591B491EC91E9235C
:10D3200021F461E085E30E94D24C61E085E30E9434
:10D33000014D8CB580618CBD8CB580648CBD61E085
:10D3400084E30E94014D61E083E30E94014D8091DE
:10D35000D00C8F5F8093D00C1FBF249ACE01019612
:10D360000E9493A789819A810E94E36C67E080E024
:10D3700090E00E94253F65E58BE190E00E94253F0B
:10D3800065E58AE190E00E94253F0E94E26C80E022
:10D3900090E49093050E8093040E80E090E69093C5
:10D3A0000D0E80930C0E80E098E49093070E80930E
:10D3B000060E80E098E690930F0E80930E0E80E0AC
:10D3C00090E59093090E8093080E80E090E790938B
:10D3D000110E8093100E80E098E590930B0E8093D1
:10D3E0000A0E80E098E79093130E8093120E0F9030
:10D3F0000F90DF91CF911F910895AF92BF92CF927E
:10D40000DF92EF92FF920F931F93CF93DF931F92C0
:10D410001F92CDB7DEB75C018B016A0179010E94D2
:10D420006D69CE0101960E9493A789819A810E941D
:10D43000E36C46E050E06AEC7CE089E090E00E941A
:10D44000F63EC50102960E94CD6CC60102960E946E
:10D45000DB6CC70102960E94D46C0E94E26CF8015A
:10D4600082819381A481B5818093C9099093CA096F
:10D47000A093CB09B093CC090F900F90DF91CF917F
:10D480001F910F91FF90EF90DF90CF90BF90AF90E2
:10D490000895CF92DF92EF92FF92CF93DF93CDB7B3
:10D4A000DEB768970FB6F894DEBF0FBECDBFFA01A6
:10D4B0002EEB33E03A8329835FEF5B835C835D83EC
:10D4C0001E8238872F83C280D380E480F580C9868E
:10D4D000DA86EB86FC863E872D87FB0142815381ED
:10D4E000648175814F87588B698B7A8B3C8B2B8B32
:10D4F000FC0182819381A481B5818D8B9E8BAF8B42
:10D50000B88F9E012F5F3F4FAE01495F5F4FBE0155
:10D51000635F7F4FCE0143960E94FD6968960FB608
:10D52000F894DEBF0FBECDBFDF91CF91FF90EF909B
:10D53000DF90CF9008950F931F93CF93DF93CDB7D4
:10D54000DEB768970FB6F894DEBF0FBECDBFFB0104
:10D55000DC0112964D915D916D917C9115974D8BEB
:10D560005E8B6F8B788F8EEB93E09A83898321E0BB
:10D57000288F0D891E892F89388D0B831C832D835D
:10D580003E8398878F8302811381248135810987A7
:10D590001A872B873C879E878D874F87588B698B8F
:10D5A0007A8BAE014F5F5F4FBE01695F7F4FCE0147
:10D5B0000D960E94496A68960FB6F894DEBF0FBEBA
:10D5C000CDBFDF91CF911F910F910895CF93DF933E
:10D5D000CDB7DEB762970FB6F894DEBF0FBECDBFF2
:10D5E000FC0182819381A481B5818F87988BA98B5F
:10D5F000BA8B2EEB33E03A83298341E04A8B4F8587
:10D60000588969897A894B835C836D837E833887E7
:10D610002F8389879A87AB87BC87BE016F5F7F4F57
:10D62000CE0107960E949B6A62960FB6F894DEBF01
:10D630000FBECDBFDF91CF910895CF92DF92EF92D1
:10D64000FF920F931F93CF93DF936C01EB017B014C
:10D6500082E0E80EF11C00E010E0C601800F911F8F
:10D660000E9441BFF70181937F010F5F1F4F04307C
:10D67000110599F78A81882361F08F3F61F48B81CE
:10D680008F3F49F48C818F3F31F481E09D819F3F32
:10D6900019F480E001C081E090E0DF91CF911F910B
:10D6A0000F91FF90EF90DF90CF900895EF92FF924F
:10D6B0000F931F93CF93DF937C018B010E5F1F4F5E
:10D6C000C0E0D0E0F80161918F01C7018C0F9D1F70
:10D6D0000E9449BF2196C430D105A1F7DF91CF91B7
:10D6E0001F910F91FF90EF900895FC01DC018D9147
:10D6F0008111FDCF40E050E020E030E08AE09191E0
:10D70000992301F1243031055CF59E3271F44F3FCD
:10D71000510509F02CF5DB01A20FB31F12964C93B3
:10D720002F5F3F4F40E050E0EACF849FD001859FBC
:10D73000B00D1124492F990F550B405351094A0F31
:10D740005B1FDDCF4F3F510509F054F42430310504
:10D750003CF4FB01E20FF31F428381E090E0089567
:10D7600080E090E008954F925F926F927F928F9247
:10D770009F92AF92BF92CF92DF92EF92FF920F9360
:10D780001F93CF93DF936115710509F45DC08A0182
:10D79000FB016C01C681D781209709F455C08885AB
:10D7A0008295807F8595859585958595823019F040
:10D7B0008530A9F045C089849A84AB84BC8441E05B
:10D7C00050E0B801C4010E9400568823C9F19801B5
:10D7D00040E050E0B401C6010E94DC6531C0CE01DA
:10D7E0000E9425AA823061F560E0CE010E94A4A9C2
:10D7F000FC014184528463847484720161E0CE012F
:10D800000E94A4A9FC01A184B2844201A50144198B
:10D8100055094F5F5F4FB801C2010E94005688232F
:10D8200079F0AE14BF0464F0A701481959099801B2
:10D83000B701C6010E94DC65FFEFEF1AFF0AF1CFC6
:10D840000A80DB81C02DA8CFDF91CF911F910F916E
:10D85000FF90EF90DF90CF90BF90AF909F908F9010
:10D860007F906F905F904F900895CF93DF931F92BA
:10D87000CDB7DEB76983DC01ED91FC910280F381C5
:10D88000E02D41E050E0BE016F5F7F4F19950F9092
:10D89000DF91CF910895DC01ED91FC91068CF78D1D
:10D8A000E02D199591E089270895862F089581E04C
:10D8B00086270895CF93DF931F92CDB7DEB7898374
:10D8C0002091D20C3981E091D30CF091D40C822FAD
:10D8D00090E080959095F8940080082200824BE0BB
:10D8E00000C05DE000005A95E9F700800822089426
:10D8F000379508F4022A00824A9599F778940F9098
:10D90000DF91CF9108950F931F93CF93DF931F92D1
:10D91000CDB7DEB78C01DC01ED91FC910084F1857F
:10D92000E02D1995892B51F0BE016F5F7F4FF801F3
:10D9300084850E94A58C898190E002C08FEF9FEFC3
:10D940000F90DF91CF911F910F910895FC01848575
:10D950000C94F68CCF93DF931F92CDB7DEB741E0E6
:10D9600050E0BE016F5F7F4FFC0184850E94F68C02
:10D97000181619061CF4898190E002C08FEF9FEF02
:10D980000F90DF91CF910895FC018485843011F0D0
:10D990000C94FC8A80E090E0089544E050E0BC01E3
:10D9A0008FE090E00C94F63E44E050E0BC0185E04E
:10D9B00090E00C94F63E44E050E0BC0181E090E041
:10D9C0000C94F63E08958CBD9DBD08956F927F9294
:10D9D0008F929F92AF92BF92CF92DF92EF92FF927F
:10D9E0001F93CF93DF931F921F92CDB7DEB75C01D9
:10D9F0003B016A01FC011485143041F481E090E0A0
:10DA0000F5019383828380E090E05BC07A0141302E
:10DA1000584018F0E12C88E0F82ECE0101960E94C3
:10DA200093A789819A810E94E36C812F0E94509B69
:10DA30004C0163E070E0812F0E94878C873111F0E8
:10DA40008C3121F48E149F0440F302C0E12CF12CA0
:10DA5000CE0101960E9493A789819A810E94E36C6E
:10DA60009701A30160E070E0812F0E94EB9A60E2D1
:10DA700070E0812F0E9498A762E070E0812F0E94E1
:10DA8000878C84FD14C063E070E0812F0E94878C36
:10DA9000811104C0812F0E94BB8BB0CFCE010196B3
:10DAA0000E9493A789819A810E94E36CE5CF40E1AF
:10DAB00062E070E0812F0E94B18BEF2809F49ECFC5
:10DAC000C6010F900F90DF91CF911F91FF90EF90C3
:10DAD000DF90CF90BF90AF909F908F907F906F908E
:10DAE00008958F929F92AF92BF92DF92EF92FF9232
:10DAF0000F931F93CF93DF931F921F92CDB7DEB783
:10DB0000FC012485243009F082C05A018B017C017C
:10DB1000D12C8D2D0E94178E811103C0F701D48660
:10DB200007C08B7F8831D1F3D394F4E0DF12F1CFBB
:10DB3000F7018485843009F46AC020910302309192
:10DB400004022F5F3F4F11F420E030EC30930402C9
:10DB500020930302409103025091040220E061E00F
:10DB60000E94DE8BF80182818F3F51F483818F3FC9
:10DB700099F484818F3F81F485818F3F69F444C09B
:10DB800081110AC0F8018381811106C0848181114D
:10DB900003C085818823C1F1A114B104A9F1F70163
:10DBA000D484CE0101960E9493A789819A810E9414
:10DBB000E36CB8016E5F7F4F8D2D0E94BE8EB50164
:10DBC0008D2D0E94AD8E64E070E08D2D0E9498A78F
:10DBD0000E94844E4B015C01F4E98F0EF1E19F1E1F
:10DBE000A11CB11CC7010E9413A8873141F161E05B
:10DBF00070E080E090E00E944A4E0E94CA7FC70118
:10DC00000E9413A8811106C084E0F701848780E098
:10DC100090E01DC00E94844E86169706A806B9069D
:10DC200008F7F70184850E94BB8B84E0F7018487A5
:10DC300065EC76E189E39BE00E9482A0E8CF6AEB85
:10DC400076E189E39BE00E9482A081E090E00F9062
:10DC50000F90DF91CF911F910F91FF90EF90DF9088
:10DC6000BF90AF909F908F90089578941F920F92DD
:10DC70000FB60F9211240BB60F92CF92DF92EF9254
:10DC8000FF920F931F932F933F934F935F936F9345
:10DC90007F938F939F93AF93BF93CF93DF93EF9334
:10DCA000FF93809170008E7F809370000FE310E0EF
:10DCB0008BE1E82EF12C9BE2C92ED12CC091D50C22
:10DCC000D091D60C2097F9F40332110508F43BC02B
:10DCD00003521109E091D30CF091D40C9081209162
:10DCE000D20C822F8095982390839BE0D7011197C7
:10DCF000F1F79150D9F78081822B8083C60101977B
:10DD0000F1F780E00DC00B301105E8F00B50110960
:10DD1000E091D70CF091D80CEC0FFD1F319780816A
:10DD20000E945A6C2196D093D60CC093D50C80914A
:10DD30000102909102028C179D0708F0BFCF10924C
:10DD4000D60C1092D50C8091700081608093700089
:10DD5000FF91EF91DF91CF91BF91AF919F918F9103
:10DD60007F916F915F914F913F912F911F910F91F3
:10DD7000FF90EF90DF90CF900F900BBE0F900FBEF3
:10DD80000F901F90189581E08093D10C8091000234
:10DD9000282F30E0F901EC58FA4EE491F0E0EE0F54
:10DDA000FF1FE25DFD4E459154915093D40C40937A
:10DDB000D30CF901E25DFA4EE491E093D20C61E0FC
:10DDC0000E94014D83E08093B100E0E7F0E08081A4
:10DDD000816080830895CF93DF931816190644F06D
:10DDE000809170008E7F809370001092D10C19C0CA
:10DDF000EC018091D70C9091D80C0E947FB6CE0197
:10DE0000C130D24014F080E092E0909302028093FF
:10DE100001020E94E7B59093D80C8093D70C892B10
:10DE200029F4109202021092010208C08091D10CD4
:10DE3000811104C0DF91CF910C94C36EDF91CF911B
:10DE40000895FF920F931F93CF93DF938C01F62ECB
:10DE50008091D10C811102C00E94C36EE80121970C
:10DE6000C11582E0D80798F48091010290910202D6
:10DE70008017910718F4C8010E94EB6E8091D70CAF
:10DE80009091D80C009719F0C80FD91FF882DF9134
:10DE9000CF911F910F91FF900895DC0180E06150B8
:10DEA00040F09D91E82FE927F0E0E654FA4E849186
:10DEB000F6CF0895AF92BF92CF92DF92EF92FF928A
:10DEC0001F93CF93DF93EC010E94844E6B017C0182
:10DED00028EEC20E23E0D21EE11CF11C8BE4A82E1A
:10DEE000B12C0E94844E6C157D058E059F0598F41B
:10DEF00060EFCE010E943D90CE010E949390182FBA
:10DF000080FF11C0EF85F889309709F01995C50198
:10DF10000197F1F7E6CF81E08A836DE476E089E34B
:10DF20009BE00E94C077812FDF91CF911F91FF90DE
:10DF3000EF90DF90CF90BF90AF9008950F931F9315
:10DF4000CF93DF93EC01162F042F0E945A6F00230A
:10DF500019F0CE010E947691CE010E94319065EABF
:10DF60008FEC99E00E94FF8F612F8FEC99E00E9467
:10DF7000FF8FCE01DF91CF911F910F910C942E90C6
:10DF8000EF92FF920F931F93CF93DF938C017B014E
:10DF900040E065E50E949E6FE70188E0E80EF11C15
:10DFA000699140E0C8010E949E6FCE15DF05C1F760
:10DFB000DF91CF911F910F91FF90EF9008951F93E4
:10DFC000CF93DF93EC01162F0E945A6FCE010E946F
:10DFD000319062ED8FEC99E00E94FF8F612F70E02D
:10DFE0006095709584E0660F771F8A95E1F7612B45
:10DFF0008FEC99E00E94FF8FCE010E942E90CE01FF
:10E000000E949390181711F084E08A83DF91CF91DA
:10E010001F9108951F93CF93DF93EC010E945A6FD5
:10E0200080FD31C0CE010E946B9160E0CE010E9464
:10E03000DF6FCE010E945A6FCE010E94319064EBD7
:10E040008FEC99E00E94FF8FCE010E942E90CE01AE
:10E050000E945A6F182F82FF03C082E08A8304C097
:10E060008A81823009F41A828881882341F0CE01A6
:10E070000E946B91682F6160CE010E94DF6F11FBDF
:10E08000882780F901C080E0DF91CF911F9108952A
:10E09000CF92DF92EF92FF920F931F93CF93DF9374
:10E0A0007C01EB018A01FC01858196810E940A7046
:10E0B0008823C9F1BE01F701858196810E94C06F56
:10E0C00040E06EEBF701858196810E949E6FE8012A
:10E0D0006801F9E0CF0ED11CF70105811681C80156
:10E0E0000E945A6FC8010E94319066E98FEC99E056
:10E0F0000E94FF8FC8010E942E90C8010E945A6F93
:10E1000061EEC8010E943D90C8010E9493908993DE
:10E11000CC16DD0609F7F701858196810E940A7009
:10E1200091E0813009F090E0892FDF91CF911F912C
:10E130000F91FF90EF90DF90CF900895CF93DF93F2
:10E14000EA010E944870882339F068E0CE010E94FD
:10E150004D6F91E02885281390E0892FDF91CF91B2
:10E160000895CF93DF93CDB7DEB729970FB6F89414
:10E17000DEBF0FBECDBFAE014F5F5F4F0E949E70EE
:10E18000882389F08D818F3361F020F48F3159F429
:10E1900089E00CC08F3519F08F3739F004C08BE05F
:10E1A00005C08AE003C080E001C08CE029960FB66C
:10E1B000F894DEBF0FBECDBFDF91CF9108956F926F
:10E1C0007F928F929F92AF92BF92CF92DF92EF9207
:10E1D000FF920F931F93CF93DF93FC0124852111AE
:10E1E0009EC0872E762EEC010E940A70811108C015
:10E1F00068E576E089E39BE00E94C0778FEF90C0EE
:10E20000CE010E945A6F40E060EFCE010E949E6FE7
:10E21000C12CD12C66246A94EE24E394F12C0C2DAD
:10E2200006950695069510E08C2D8770570101C064
:10E23000AA0C8A95EAF78B85082E000C990BC81654
:10E24000D90634F4FE01E00FF11F93809A2006C036
:10E2500099249394C816D90609F0912CCE010E94F6
:10E260005A6FCE010E94319068E78FEC99E00E94CE
:10E27000FF8F911002C060E001C060E88FEC99E070
:10E280000E94FF8FCE010E942E90CE010E945A6FF5
:10E29000282F2074982F907885FF11C02223A9F091
:10E2A00042E050E0682F89E39BE00E94BF9F64E654
:10E2B00076E089E39BE00E94C0778EEF31C02111A8
:10E2C00004C0911104C06C2C08C0992331F0FE01E8
:10E2D000E00FF11F83818A2907C0FE01E00FF11FC3
:10E2E0008A2D8095938189238383FFEFCF1ADF0ADC
:10E2F00080E4C816D10409F092CF6B86EFEF6E125E
:10E3000002C081E08C87DE011396E72DF82D2B9655
:10E310008D918193CA17DB07D9F781E001C080E0B6
:10E32000DF91CF911F910F91FF90EF90DF90CF90F1
:10E33000BF90AF909F908F907F906F900895AF9215
:10E34000BF92CF92DF92EF92FF920F931F93CF93E2
:10E35000DF93CDB7DEB7AF970FB6F894DEBF0FBE31
:10E36000CDBF7C015B016A010EEB13E01A830983C8
:10E370001B821C821D821E82CE0109960E942C8B5C
:10E380001BA70AA71CA61DA61EA61FA68091C90929
:10E390009091CA09A091CB09B091CC098EA39FA3FB
:10E3A000A8A7B9A78B839C83AD83BE8318861F82E1
:10E3B000AE01465D5F4FB501CE0101960E94904EC1
:10E3C00081309105B1F4D701ED91FC910684F78578
:10E3D000E02D1DA30CA38CA59DA5AEA5BFA58EA366
:10E3E0009FA3A8A7B9A7A601BE016C5D7F4FC70177
:10E3F0001995AF960FB6F894DEBF0FBECDBFDF9173
:10E40000CF911F910F91FF90EF90DF90CF90BF9031
:10E41000AF9008950F931F93CF93DF938C01EB017F
:10E42000209741F06091E3097091E409CE010E94C8
:10E430001BB802C080E090E020E0AC01BE01C80142
:10E44000DF91CF911F910F910C9426A9FC0192812D
:10E45000892F82958F7019F0823021F016C09F703D
:10E46000906292839B016E3681E078072CF477FFEF
:10E4700005C020E030E002C02DE631E02683878130
:10E4800030FB80F9878381E0089580E008956F92E2
:10E490007F928F929F92AF92BF92CF92DF92EF9234
:10E4A000FF920F931F93CF93DF93CDB7DEB7EA9719
:10E4B0000FB6F894DEBF0FBECDBF78AF6FAB5AAFCB
:10E4C00049AF672B09F4B3C2FA01309719F02081E4
:10E4D000211109C0FC012385222329F09C01255F1D
:10E4E0003F4F3AAF29AF6C01E9ADFAAD309721F457
:10E4F000F601A588B6880AC080818823C9F3CE01B9
:10E50000C9960E9425AE5C01892B91F300E010E0D2
:10E51000EFA8F8AC4701800E911EF401808188239A
:10E5200051F0082E000C990B0E941BC4F40180834B
:10E530000F5F1F4FEDCFE114F10441F1F70180812E
:10E54000882321F18D3229F190ED980F9A3008F14E
:10E55000853211F18B3719F1833221F12CED822EA6
:10E5600026E1922E01E010E0C4010E94E1B7AC0167
:10E57000B401C7010E94FAB7892BB1F00F5F1F4F9A
:10E58000F9E08F0E911C0931110571F70FEF1FEFA4
:10E590000BC000E010E008C008E010E005C00EEF7E
:10E5A0001FEF02C007E110E064EB77E186ED9BE02E
:10E5B0000E945EA04AE050E0B80186ED9BE00E9418
:10E5C00015A086ED9BE00E94A35119A61AA61BA6D2
:10E5D0001CA61DA61EA61FA618AA8BA58F708BA70A
:10E5E00009A785E0A816B10451F096E0A916B10478
:10E5F00059F0A114B10469F0772473940BC0772407
:10E60000739408E110E006C07724739407E110E0EA
:10E6100001C0712C6A2C6A2DCE0189960E94343576
:10E6200029873A874B875C876D877E878F87988B92
:10E630000A3011058CF40830110524F50E3FEFEF78
:10E640001E070CF4E6C10F3FFFEF1F0709F00CF4A3
:10E65000EEC1012B71F1DDC10731110509F497C13C
:10E660000831110509F0D5C160E0CE0189960E94FC
:10E670005C35298B3A8B4B8B5C8B6D8B7E8B8F8BB8
:10E68000988F17C0CE01C7960E94C5942BA52F70F6
:10E69000206A2BA7092E000CAA0BBB0B482F8DA7B5
:10E6A0009EA7AFA7B8ABE9ACFAAC09A51AA53CA5E3
:10E6B000B7C119821A821B821C828B818F7080667F
:10E6C0008B831982EFA9F8AD309709F460C080817F
:10E6D000882309F45CC08FA898ACF401808188235A
:10E6E00059F08D3249F080538A3030F0FFEF8F1AA5
:10E6F0009F0A98AE8FAAEFCFC4010E94AAB78C01DF
:10E700006EE270E0C4010E947AC4009769F0FC01D7
:10E71000818180334CF08A3354F4E82E880FFF084F
:10E72000F0E3EF1AF10806C0E12CF12C03C099E0E8
:10E73000E92EF12C6CE270E0C4010E947AC40097CB
:10E7400019F418AE1FAA03C0019698AF8FABE1145D
:10E75000F104A1F02AE0209FC001219F900D112417
:10E76000101611061CF0F194E194F1088C010E0DC5
:10E770001F1D012E000C220B330B0CC0012E000CB0
:10E78000220B330B8B818F70806A8B8303C000E078
:10E7900010E0980189819A81AB81BC8189A39AA3F9
:10E7A000ABA3BCA30DA31EA32FA338A7662DCE0138
:10E7B00081960E94343529833A834B835C836D8331
:10E7C0007E838F839887FBA0F2948FE0F8224E011E
:10E7D00081E3880E911C00E010E08FA998AD892B91
:10E7E00071F00330110559F00F5F1F4FCE01C7962E
:10E7F0000E94C594F401819391934F01EECFFAE00A
:10E80000AF16B10489F08BE0A816B10411F199E0BC
:10E81000A916B10419F5CE0181960E945337CE0195
:10E8200089960E942672F5C0CE0181960E945337C8
:10E830008BA5982F92959F7019F0923021F0E9C026
:10E840008F7080628BA7653610F064E670E06EA76B
:10E85000E0C0CE0181960E94533794C081E090E0E1
:10E86000F11002C080E090E0800F911F823091058E
:10E8700001F11CF4019741F0CCC08330910549F1BE
:10E88000049709F452C0C5C0772051F088E0FE011A
:10E89000B196DE01999601900D928A95E1F7B9C083
:10E8A000CE0181960E945337CE0189960E94803511
:10E8B000B0C019A9CE0181960E9453378BA58F70E5
:10E8C00080638BA76FA788A970FB80F988AB1EA710
:10E8D000A0C01BA5E9A808A9FBA8CE0181967720B6
:10E8E00061F00E9453371F7010621BA76FA770FB67
:10E8F00000F908ABEEA6FDA68CC00E9453371F702E
:10E9000010621BA76FA770FB00F908ABEEA62F2DB6
:10E9100030E0AFEFB0E00E94BBBF24E630E040E063
:10E9200050E00E9489BF2DA774C01BA5E9A808A9C3
:10E93000FBA8CE018196772061F00E9453371F70AB
:10E9400010621BA76FA770FB00F908ABEEA6FDA62F
:10E9500017C00E9453371F7010621BA76FA770FB70
:10E9600000F908ABEEA62F2D30E0AFEFB0E00E942B
:10E97000BBBF24E630E040E050E00E9489BF2DA7F5
:10E980006DA97EA9CE0189960E94F47742C060E00D
:10E99000CE0189960E945C3529A33AA34BA35CA3C0
:10E9A0006DA37EA38FA398A7FE0131967F0100E09F
:10E9B00010E08FA998AD892B71F004301105E9F0B2
:10E9C0000F5F1F4FCE01C7960E94C594F701819338
:10E9D00091937F01EECF0330110521F00430110532
:10E9E000C1F40BC09D812B8139818BA58F70806410
:10E9F0008BA73FA72EA79DA70CC09F812D813B8190
:10EA000049818BA58F7080658BA74FA73EA72DA747
:10EA100098ABE9ACFAAC09A51AA52BA53CA54DA568
:10EA20005EA56FA578A9C6010E94FD1802C080E00E
:10EA300090E0EA960FB6F894DEBF0FBECDBFDF912F
:10EA4000CF911F910F91FF90EF90DF90CF90BF90EB
:10EA5000AF909F908F907F906F9008957F928F924C
:10EA60009F92AF92BF92CF92DF92EF92FF920F935D
:10EA70001F93CF93DF938C016A017B01722E9A0161
:10EA8000AB01C701B6010E94A9C2882319F06EE646
:10EA900076E027C046015701E894B7F82FEF3FEF23
:10EAA0004FE75FE7C501B4010E94A9C281110DC003
:10EAB0002FEF3FEF4FE75FE7C501B4010E947DC034
:10EAC00018161CF462E776E00CC02FEF3FEF4FE71B
:10EAD0005FE4C701B6010E94DCC1181694F466E732
:10EAE00076E0C801DF91CF911F910F91FF90EF90D9
:10EAF000DF90CF90BF90AF909F908F907F900C94BD
:10EB000094A02FEF3FEF4FE75FECC701B6010E94E3
:10EB10007DC087FDE4CF20E030E0A901C701B60148
:10EB20000E947DC087FF0AC06DE2C8010E94C69F97
:10EB3000EC01F7FAF094F7F8F09402C0C0E0D0E0EE
:10EB4000B12C60E070E080E09FE37B1441F020E0B6
:10EB500030E040E251E40E9482C0B394F6CFA701B6
:10EB600096010E9411C06B017C010E94FBC04B0109
:10EB70005C012AE0AB01BC01C8010E945A51C80FD8
:10EB8000D91F7720C1F1C501B4010E942AC19B01A0
:10EB9000AC01C701B6010E9410C06B017C016EE29E
:10EBA000C8010E94C69FC80FD91F20E030E040E294
:10EBB00051E4C701B6010E94E1C14B015C010E9412
:10EBC000FBC06B01E12CF12C2AE0B701A601C801C2
:10EBD0000E945A51C80FD91FC701B6010E942AC10D
:10EBE0009B01AC01C501B4010E9410C06B017C0106
:10EBF0007A947110DACFCE01DF91CF911F910F91EE
:10EC0000FF90EF90DF90CF90BF90AF909F908F904C
:10EC10007F9008950F931F93CF93DF93FC0181851D
:10EC200092850097C9F08B01EF01DC01ED91FC9119
:10EC30000484F585E02D1995892B71F089859A85D5
:10EC4000DC01ED91FC910480F581E02DB801DF91AC
:10EC5000CF911F910F91199480E090E0DF91CF91B7
:10EC60001F910F910895EF92FF920F931F93CF93EF
:10EC7000DF93CDB7DEB728970FB6F894DEBF0FBE8F
:10EC8000CDBF19821A821B821C821D821E821F82A6
:10EC900018862B812F70E12CF12C02E01A813C8127
:10ECA00040E05E816F8178850E94FD1828960FB63E
:10ECB000F894DEBF0FBECDBFDF91CF911F910F91B2
:10ECC000FF90EF9008950F931F93CF93DF93EC0184
:10ECD000209731F10A811B8188858295807F8595F7
:10ECE00085958595859583FD06C08E819F810097CA
:10ECF00011F00E94637688858F70843031F48985A5
:10ED00009A85009711F00E947FB6888199810097BB
:10ED100011F00E947FB6CE010E947FB6E801D8CFE5
:10ED2000DF91CF911F910F9108958F929F92AF9293
:10ED3000BF92EF92FF920F931F93CF93DF938C01BB
:10ED40007B0149015A010E94D63DEC01892B09F152
:10ED50008885807F8360888789869A86AB86BC8613
:10ED600088819981009711F00E947FB6C7010E94A7
:10ED700023C499838883BE01C801DF91CF911F917D
:10ED80000F91FF90EF90BF90AF909F908F900C9459
:10ED900033AADF91CF911F910F91FF90EF90BF9019
:10EDA000AF909F908F9008958F929F92AF92BF9255
:10EDB000CF92DF92EF92FF920F931F93CF93DF9347
:10EDC0001091280D113208F0C2C0082FD091270DE4
:10EDD0000E94254E6B017C01C091FF0CCC2311F1E8
:10EDE0008091010D9091020DA091030DB091040D41
:10EDF000892B8A2B8B2B81F30E94254E8090010D4D
:10EE00009090020DA090030DB090040DDC01CB0199
:10EE10008C199D09AE09BF0988169906AA06BB067A
:10EE2000D8F681C082E08093FF0C0093FE0C8FEF38
:10EE30008093FD0C1092FC0C1093FB0CA7E0BDE03E
:10EE4000EBEDFCE080E0181721F09D9191938F5F2E
:10EE5000FACF1092DA0C9091DA0C8D2F880F892B53
:10EE60008093DA0C8091D90C813089F51092D90CFD
:10EE70000E94254E6B017C018091DA0C8093BB00CF
:10EE80008091010D9091020DA091030DB091040DA0
:10EE9000892B8A2B8B2BA9F00E94254E0091010D06
:10EEA0001091020D2091030D3091040DDC01CB0176
:10EEB0008C199D09AE09BF09081719072A073B07D6
:10EEC00090F18091BC0083FDD7CF85EC01C085EE29
:10EED0008093BC000E94254E6B017C018091FF0C49
:10EEE000823039F58091010D9091020DA091030DB2
:10EEF000B091040D892B8A2B8B2B81F30E94254E18
:10EF00000091010D1091020D2091030D3091040D1F
:10EF1000DC01CB018C199D09AE09BF09081719073F
:10EF20002A073B07D8F68091000D0E947290C5E039
:10EF300013C08091FD0C8F3F79F08091FD0C8032E1
:10EF400041F08091FD0C803331F0C4E005C0C1E098
:10EF500003C0C2E001C0C3E01092060D1092280D5C
:10EF60001092050D8C2FDF91CF911F910F91FF9083
:10EF7000EF90DF90CF90BF90AF909F908F900895CB
:10EF80000F931F93CF93DF93EC010E9494A08C0109
:10EF9000CE010E94A351800F911FDF91CF911F914D
:10EFA0000F910895FC01A7812A2F2E7FD1F0828135
:10EFB00082958F7081508330A0F4A695B0E01197B0
:10EFC0002BE531E00E94F5BF24E630E040E050E060
:10EFD0000E9489BFDA01C90187569F4FAF4FBF4FCB
:10EFE00008958FEF9FEF0895CF93DF93EC018A810F
:10EFF000982F92959F7019F0943050F503C08F7040
:10F0000080628A83CB01770FAA0BBB0B9C01AD01F9
:10F010002959310941095109A4E6B0E00E94A8BF6D
:10F020002BE531E040E050E00E9489BF25363105F4
:10F030002CF437FF05C020E030E002C024E630E0C9
:10F040002F5F220F8F818170282B2F8381E001C0D9
:10F0500080E0DF91CF9108952F923F924F925F927F
:10F060006F927F928F929F92AF92BF92CF92DF92D8
:10F07000EF92FF920F931F93CF93DF93CDB7DEB73D
:10F08000A4970FB6F894DEBF0FBECDBF6C01098BFD
:10F090001A8B2B8B3C8B4D8B5E8B6F8B788F2DE07F
:10F0A000E216F10430F4F701EA53FC4F4081498F36
:10F0B00001C0198ECE0141960E94D27797FD04C0FF
:10F0C000BC01C6010E94F4770B89802F8F70D60196
:10F0D00012969C911297907FF92EF82A1296FC9224
:10F0E000F294FFE0FF228F2D90E08C30910508F024
:10F0F00004C4FC018827E15CFE4F8F4F0C94DEBFF7
:10F1000002950F70802F90E0FC013197EB30F105F4
:10F1100008F072C08827E55BFE4F8F4F0C94DEBF6E
:10F12000888DF60187838F89D60116968C93169762
:10F130008E8915968C9315978D8914968C931497B8
:10F140000295007F12968C9112978F70082B129661
:10F150000C93D3C38F89988DF6018683878190FBAA
:10F1600080F987838E898583C8C38D899E89AF89FD
:10F17000B88DB7FD0BC08F3F9105A105B105B1F06A
:10F18000ACF08FEF90E0A0E0B0E010C080E00EC0E7
:10F190008F89988DF6018683878190FB80F987831C
:10F1A0008E8985838D898483A8C38D89D601149621
:10F1B0008C93A3C38D889E88AF88B88C20E030E004
:10F1C000A901C501B4010E947DC087FD0FC020E0E8
:10F1D00030E04FE753E4C501B4010E94DCC11816CA
:10F1E0003CF0C501B4010E94FBC003C060E001C057
:10F1F0006FEFF601648381C363E578E186ED9BE000
:10F200000E945EA04AE050E0602F86ED9BE00E94E5
:10F21000BF9F60E578E162C38D899E89AF89B88D13
:10F22000F60184839583A683B783007F82818F70E4
:10F23000082B028362C360E0CE0141960E945236E1
:10F24000D60114968C93149779C002950F70802F75
:10F2500090E0FC013197EB30F10508F077C088278A
:10F26000EA5AFE4F8F4F0C94DEBF6D897E898F89DD
:10F27000988D0E942CC120E030E040E251E40E94D1
:10F2800082C00BC06D8970E080E090E010C06D8995
:10F290007E898F89988D0E942CC1F60164837583C5
:10F2A000868397832AC36D897E898F89988D0E9472
:10F2B0002AC1D60114966D937D938D939C931797D5
:10F2C0001CC30295007FF60182818F70082B028398
:10F2D0008D899E89AF89B88D84839583A683B783F2
:10F2E0000CC30295007FD60112968C9112978F70F5
:10F2F000082B12960C938D899E89AF89B88DF601E3
:10F3000084839583A683B783F8C260E0C6010E9418
:10F310005236D60114968C9314978F89988D169631
:10F320008C93169717968C91179790FB80F91796E8
:10F330008C9317978E8915968C93159712968C91AE
:10F3400012978F70806212968C93D7C26EE378E129
:10F3500086ED9BE00E945EA04AE050E0602F86EDC3
:10F360009BE00E94BF9F6BE378E1B8C211E001C04F
:10F3700010E002950F70802F90E0FC013197EB3088
:10F38000F10508F09CC28827EF59FE4F8F4F0C946F
:10F39000DEBF8D899E89AF89B88DF6018483958300
:10F3A000A683B7830295007F82818F70082B02832A
:10F3B00088E0B4C20630C9F030F4013059F00330AF
:10F3C00039F52FEF26C00730D9F00A50023000F58A
:10F3D0002D891FC02D8930E0A4E6B0E00E94BBBF9C
:10F3E0002FEF30E040E050E008C06D897E898F89C2
:10F3F000988D2AE030E040E050E00E9489BF09C0CB
:10F400006D897E898F89988D0E94F4C0262F01C056
:10F4100020E084E68F8B888D8E7F888F1E8A8B8973
:10F420008F7080628B8B2D8B2E8930E0AFEFB0E038
:10F430000E94BBBFE4E68E2E912CA12CB12CA5011D
:10F4400094010E9489BF29013A011901FD89FA8FAF
:10F45000EF2EF12C112309F479C1088D069510E0E7
:10F460000150110908F084C040E8441651040CF022
:10F470004AC08FE790E0841995098E9DD0018F9D39
:10F48000B00D9E9DB00D11242FEF30E00E94F5BF0E
:10F4900021E83EE740E050E00E9489BFD601179680
:10F4A0002C93D2012EEF31E00E94F5BF5FE7852E4D
:10F4B000912CA12CB12CA50194010E9489BFD701E8
:10F4C0000E94A8BF2FEF30E040E050E00E9489BFCB
:10F4D00079018A01D2012BE930E00E94F5BFA50134
:10F4E00094010E9489BFDA01C9018C599F4FAF4F27
:10F4F000BF4F1C01FFEFEF16F10419F114F1EE24D8
:10F50000EA94F12C1EC0C201550CAA0BBB0B9C0146
:10F51000AD012058310941095109ABE9B0E00E9421
:10F52000A8BF2FE730E040E050E00E9489BFDA0139
:10F53000C9018C599F4FAF4FBF4F1C01D601179681
:10F540001C926EE278E186ED9BE00E945EA04AE0AC
:10F5500050E0B10186ED9BE00E9415A060E278E1E9
:10F5600086ED9BE00E945EA04AE050E0B701E6C055
:10F570009801AAEBBFEF0E94EDBFA50194010E9484
:10F5800089BFDA01C9018C599F4FAF4FBF4F8B8F95
:10F590009C8FAD8FBE8F26E430E0D8010E94F5BF6E
:10F5A000A50194010E9489BF49015A019EE1890E7B
:10F5B000911CA11CB11CC201052C000CAA0BBB0B99
:10F5C0008F8F98A3A9A3BAA390E8491651040CF011
:10F5D00058C08FE790E0841995098E9DD0018F9DCA
:10F5E000B00D9E9DB00D1124A50194010E94B3BFE2
:10F5F0009B01AC01AFEFB0E00E94A8BF24E63AE661
:10F6000040E050E00E9489BFD60117962C932F8DC1
:10F6100038A149A15AA18B8D9C8DAD8DBE8D280F2F
:10F62000391F4A1F5B1FAEEFB1E00E94A8BF23EE57
:10F6300030E040E050E00E9489BF3CA32BA39A8DAC
:10F64000A92FB0E00E94A8BF2FEF30E040E050E0CB
:10F650000E9489BF79018A01D2012FEF30E00E9418
:10F66000F5BF2FE730E040E050E00E9489BF19016C
:10F67000AFEFEA16F10401F1FCF0EE24EA94F12C6C
:10F680001BC02F8D38A149A15AA120583109410929
:10F690005109ABE9B0E00E94A8BF2FE730E040E09D
:10F6A00050E00E9489BFDA01C9018C599F4FAF4FCA
:10F6B000BF4F1C01F60117826AE178E186ED9BE0FD
:10F6C0000E945EA02AE030E04B8D5C8D6D8D7E8DBA
:10F6D00086ED9BE00E94CD9F64E178E186ED9BE0A2
:10F6E0000E945EA02AE030E0B501A40186ED9BE017
:10F6F0000E94CD9F6CE078E186ED9BE00E945EA0C9
:10F700004AE050E0B10186ED9BE00E9415A064E064
:10F7100078E186ED9BE00E945EA04AE050E0B701F0
:10F7200086ED9BE00E9415A06BEF77E186ED9BE0F4
:10F730000E945EA04AE050E06BA17CA186ED9BE0B8
:10F740000E9415A086ED9BE00E94A351E4E7F5E13D
:10F75000E491F0E0EE0FFF1FE25DFD4E8591949184
:10F76000EEE2F5E1E4912F89388D3170AFEFBFEF14
:10F770000E94BBBF2DE631E040E050E00E9489BF0F
:10F7800044275527AAEFB5E00E94A8BFDC01CB01B2
:10F790009058AF4FBF4FCD01BB2797FDB095AB2F12
:10F7A0008E3FF1E09F0760F48F3F910518F4682FBA
:10F7B00080E029C06EEF962F981B80E06FEF24C089
:10F7C0008C3F43E0940760F48D3FE2E09E0718F41D
:10F7D0008E5F6FEF03C06CEF681B8FEF90E014C07B
:10F7E0008A3FF5E09F0769F08B3F44E0940728F4D7
:10F7F00094E0980F8FEF60E007C06AEF681B862FD8
:10F8000001C080E060E09FEFAFEFEA1AFA0AF10171
:10F81000FF2731962094312C9E9FA0019F9F500D71
:10F820001124452F5527420D531D6E9F90016F9F48
:10F83000300D1124232F3327220D331D8E9FB0014D
:10F840008F9F700D1124872F9927280E391ED701FD
:10F850000E94F5BF2B013C014424662477249101CA
:10F860000E94F5BFBB27A92F982F872F5301420174
:10F87000882A992AAA2ABB2A9A01D7010E94F5BF91
:10F88000DC01CB018827AA27BB27BA2FA92F982FE5
:10F89000882788299929AA29BB29F601A683958357
:10F8A000848364EF77E186ED9BE00E945EA0C60151
:10F8B0000E94F23360E080E00E94014D1EC062EEC3
:10F8C00077E186ED9BE00E945EA04AE050E0602F69
:10F8D00086ED9BE00E94BF9F6FED77E186ED9BE098
:10F8E0000E945EA04AE050E06F2D86ED9BE00E94F2
:10F8F000BF9F86ED9BE00E94A351F98DFF2361F02D
:10F900006F2FC6010E94C93529833A834B835C83DC
:10F910006D837E838F83988788E0F601DE011996D8
:10F9200001900D928A95E1F729853A854B855C8592
:10F930006D857E858F859889A4960FB6F894DEBF75
:10F940000FBECDBFDF91CF911F910F91FF90EF9030
:10F95000DF90CF90BF90AF909F908F907F906F90EF
:10F960005F904F903F902F9008956F927F928F926B
:10F970009F92AF92BF92CF92DF92EF92FF920F933E
:10F980001F93CF93DF93CDB7DEB72C970FB6F894C4
:10F99000DEBF0FBECDBF4C01762E672E6A01590126
:10F9A00081E090E09093100980930F0926E240E8EF
:10F9B00055E260E070E08EE199E00E9446AD709201
:10F9C000060A8EE199E09093050A8093040A10924A
:10F9D000110B1092130B1092120B0115110541F02F
:10F9E0000130110539F4FE2CEE24EE24EA9402C015
:10F9F000FF24FA94C701A0E0B0E089839A83AB8327
:10FA0000BC8380E190E09E838D83A60160E070E07E
:10FA10004F83588769877A879C878B874AE050E0B5
:10FA2000672D762D86ED9BE00E9415A06CED77E1A9
:10FA300086ED9BE00E945EA0BE01695F7F4F86ED70
:10FA40009BE00E9478B18C0168ED77E10E945EA096
:10FA50004AE050E0B501C8010E9415A065ED77E1CC
:10FA6000C8010E945EA0BE016F5F7F4FC8010E9467
:10FA700078B10E94A351A114B10491F082E0A816BC
:10FA8000B10409F5D0928C0AC0928B0A10928E0AAA
:10FA900010928D0AF092900AE0928F0A86E010C0D0
:10FAA000D0928C0AC0928B0AE11003C080E090E0F3
:10FAB00002C080E09FEF90938E0A80938D0A85E0CC
:10FAC0000E948FAA07C06DEB77E186ED9BE00E9454
:10FAD0005EA080E01092100910920F09882331F087
:10FAE000C4010E94944280E090E002C081E090E076
:10FAF0002C960FB6F894DEBF0FBECDBFDF91CF912D
:10FB00001F910F91FF90EF90DF90CF90BF90AF903B
:10FB10009F908F907F906F900895A89508950E9470
:10FB20004CA3A8950E94DB0E039724F00E947E98B8
:10FB30000E94D9230C94215E60E08DE00C94D24C9D
:10FB400061E08DE00C94D24CCF92DF92EF92FF9265
:10FB50000F931F93CF93DF936C01EB01099000206B
:10FB6000E9F72197C61BD70BC032D10514F0CFE1BE
:10FB7000D0E08B01E12CF12CEC16FD0664F4F801C9
:10FB800061918F01C7018C0D9D1D0E9449BFFFEF40
:10FB9000EF1AFF0AF1CF60E0C6018C0F9D1FDF91C5
:10FBA000CF911F910F91FF90EF90DF90CF900C9429
:10FBB00049BFCF93DF931F92CDB7DEB71982892B50
:10FBC00021F0FB016281738103C0BE016F5F7F4F33
:10FBD00086E390E00E94A47D6AE079E183E29BE005
:10FBE0000E945EA00F90DF91CF910895CF93DF9395
:10FBF000C0E0D0E060E0CE010E9449BF2196CD3444
:10FC0000D105C1F76CE486E490E00E9449BF68E446
:10FC100087E490E00E9449BF63E488E490E00E949A
:10FC200049BF66E489E490E00E9449BF6AEF78E149
:10FC300083E29BE0DF91CF910C945EA0EF92FF9264
:10FC40000F931F93CF93DF931F92CDB7DEB78B0136
:10FC5000CE0101969F938F938FEC9CE09F938F939F
:10FC60008EEC9CE09F938F938DEC9CE09F938F9301
:10FC70008CEC9CE09F938F938BEC9CE09F938F93F5
:10FC80008AEC9CE09F938F938AE796E09F938F93F3
:10FC9000FB0183818F9382818F930E9439C50FB6B8
:10FCA000F894DEBF0FBECDBF06977CF4F801028149
:10FCB00013816CE179E18EE29BE00E945EA0B801C5
:10FCC0008EE29BE00E94A9A019C00E94E7318AEC55
:10FCD000E82E8CE0F82E00E010E0F70161917F0142
:10FCE000C8010E9449BF0F5F1F4F06301105A9F7D9
:10FCF0006EE279E183E29BE00E945EA00F90DF91CB
:10FD0000CF911F910F91FF90EF900895EF92FF9286
:10FD10000F931F93CF93DF93CDB7DEB72C970FB61A
:10FD2000F894DEBF0FBECDBF8C017B018EEB93E05C
:10FD30009A8389831B821C821D821E8298878F83EF
:10FD400019861A861B861C86053011055CF0BE01DB
:10FD5000695F7F4FF701808591850E94756B892BC4
:10FD600009F052C0BE016F5F7F4F82E190E00E94B8
:10FD7000566B043011050CF44FC0BE01695F7F4F14
:10FD8000F701868197810E94756B892B09F444C025
:10FD9000BE01695F7F4F8EE090E00E94566BBE010E
:10FDA000695F7F4FF701848195810E94756B892B74
:10FDB000F1F1BE01695F7F4F8AE090E00E94566BCF
:10FDC000BE01695F7F4FF701828193810E94756B4D
:10FDD000892BC1F1BE01695F7F4F86E090E00E94F0
:10FDE000566B63EE78E183E29BE00E945EA02C9666
:10FDF0000FB6F894DEBF0FBECDBFDF91CF911F913C
:10FE00000F91FF90EF900895BE01695F7F4F82E1EF
:10FE100090E00E94566BB1CFBE016F5F7F4F8EE0C6
:10FE200090E00E94566B033011050CF0B8CFBE0174
:10FE30006F5F7F4F8AE090E00E94566B02301105A1
:10FE40000CF0BECFBE016F5F7F4F86E090E00E9456
:10FE5000566B0130110529F6BE016F5F7F4F86E0BA
:10FE600090E00E94566B6AEE78E183E29BE00E948C
:10FE70005EA0B7CFCF93DF93CDB7DEB72C970FB689
:10FE8000F894DEBF0FBECDBF1C821B821E821D8276
:10FE90008FEF9FEF98878F8387ED93E09A83898315
:10FEA0008CE490E09A8789871C861B8669EC78E150
:10FEB00083E29BE00E945EA06091290D70912A0D63
:10FEC000CE0101960E94D63B6FEFCE0101960E94B3
:10FED000B73A69EB78E183E29BE00E945EA02C9642
:10FEE0000FB6F894DEBF0FBECDBFDF91CF9108955E
:10FEF000CF93DF93CDB7DEB769970FB6F894DEBF27
:10FF00000FBECDBF8FE290E09A838983FE013396C6
:10FF100087E1DF011D928A95E9F764EA78E183E2DF
:10FF20009BE00E945EA0AE014E5F5F4F66E08AECF0
:10FF30009CE00E9418951E866EE876E0CE01019640
:10FF40000E946FC4BE016F5F7F4F86ED9BE00E94F1
:10FF5000A9A0CE0101960E9418691E8666E976E086
:10FF6000CE0101960E946FC4BE016F5F7F4F86ED88
:10FF70009BE00E94A9A060EA76E0CE0101960E9473
:10FF80000A7269960FB6F894DEBF0FBECDBFDF913F
:10FF9000CF9108958091390D8F5F8093390DA89589
:10FFA0000E94D9238091390D81508093390D089595
:10FFB00068EC7BE183E29BE00E945EA065EB7BE165
:10FFC00083E29BE00E945EA067EA7BE183E29BE024
:10FFD0000E945EA06FE97BE183E29BE00E945EA04D
:10FFE00083E29BE00E94A35162E97BE183E29BE014
:10FFF0000E945EA062E87BE183E29BE00E945EA03B
:020000021000EC
:1000000066E77BE183E29BE00E945EA06FE57BE117
:1000100083E29BE00E945EA06BE47BE183E29BE0D5
:100020000E945EA066E37BE183E29BE00E945EA00B
:1000300067E27BE183E29BE00E945EA068E17BE1F6
:1000400083E29BE00E945EA060E17BE183E29BE0B3
:100050000E945EA06FEF7AE183E29BE00E945EA0C7
:1000600064EF7AE183E29BE00E945EA06AEE7AE1AF
:1000700083E29BE00E945EA062EE7AE183E29BE075
:100080000E945EA066ED7AE183E29BE00E945EA0A2
:100090006CEB7AE183E29BE00E945EA06DE97AE17D
:1000A00083E29BE00E945EA068E87AE183E29BE045
:1000B0000E945EA06BE77AE183E29BE00E945EA073
:1000C0006DE67AE183E29BE00E945EA061E67AE160
:1000D00083E29BE00E945EA069E57AE183E29BE017
:1000E0000E945EA06EE47AE183E29BE00E945EA043
:1000F00061E47AE183E29BE00E945EA069E37AE139
:1001000083E29BE00E945EA06EE27AE183E29BE0E4
:100110000E945EA083E29BE00C94A351AF92BF9239
:10012000CF92DF92EF92FF920F931F93CF93DF93C3
:100130006C017B018A010E9441BF81508E3FA0F477
:100140005701C0E0D0E001501109C017D1077CF47D
:10015000C6018C0F9D1F0E9441BFF50181935F0175
:10016000882329F02196F1CF80E090E005C0CE0DE4
:10017000DF1D188281E090E0DF91CF911F910F91F8
:10018000FF90EF90DF90CF90BF90AF9008958823BD
:1001900019F067E379E102C069E379E183E29BE06A
:1001A0000C945EA0CF93DF93CDB7DEB72C970FB63C
:1001B000F894DEBF0FBECDBF69E878E183E29BE033
:1001C0000E945EA083E29BE00E94A3518CE490E039
:1001D0000E9441BF8B37D1F51C821B821E821D827B
:1001E0008FEF9FEF98878F8387ED93E09A838983C2
:1001F0008CE490E09A8789871C861B860E947A3857
:10020000CE0101960E9472A790932A0D8093290D2A
:10021000892B49F46CE678E18EE29BE00E945EA0B7
:100220008EE29BE01BC065E678E183E29BE00E94E2
:100230005EA083E29BE00E94A3510E94F14680E110
:100240009CE00E94388C81E090E00CC068E778E187
:1002500083E29BE00E945EA083E29BE00E94A351A8
:1002600080E090E02C960FB6F894DEBF0FBECDBFB5
:10027000DF91CF910895AF92BF92CF92DF92EF922C
:10028000FF920F931F93CF93DF93CDB7DEB7C05884
:10029000D1090FB6F894DEBF0FBECDBF8E010F5B44
:1002A0001F4FD8011D921C92FE01ED5BFF4F2EE106
:1002B000DF011D922A95E9F70297CCF0FB016281DC
:1002C00073814FE150E0C8010E94B3C4B80186E1D8
:1002D00090E00E94A47DB80183E29BE00E94A9A067
:1002E00067E27AE183E29BE00E945EA01BC040E2ED
:1002F00050E0B80186E190E00E948E80892BB1F435
:1003000040E250E06BE17AE1C8010E9408B86DEF6D
:1003100079E183E29BE00E945EA0B80183E29BE06A
:100320000E94A9A083E29BE00E94A3518091CF0C80
:100330001F928F938091CE0C1F928F938091CD0C42
:100340001F928F938091CC0C1F928F938091CB0C36
:100350001F928F938091CA0C1F928F9382EA96E02E
:100360009F938F931F9280E48F93CE0101966C012F
:100370009F938F930E94CDC469EE79E183E29BE065
:100380000E945EA0B80183E29BE00E94A9A0B60192
:1003900083E29BE00E94A9A083E29BE00E94A3511C
:1003A0007E0191E6E90EF11CD70113961C921E9274
:1003B000129788EE93E0A0E0B0E0F7018483958384
:1003C000A683B78384E0848788E993E09183808360
:1003D00016870587108A178680E590E0928B818BBF
:1003E000158A62E47BE389E09EE30E9491B88C0168
:1003F0000FB6F894DEBF0FBECDBF892BE1F183E0CD
:1004000090E00E94E7B5D8011D969C938E931C97AF
:10041000FC01F182E0821282C7010E94D18A882306
:1004200019F0C7010E94388CD7011F966D917C91FD
:1004300050975196AD90BC9052976115710569F037
:10044000CE0189589F4F0E94ABA0A501BE016958FB
:100450007F4FC7010E94716D07C0F70165857685E2
:10046000A501C7010E949F71181619060CF478C0E7
:10047000C8010E94E23D00E010E0F701E388F48843
:100480000115110509F463C0F8ECEF16F10409F049
:100490004CC06DED79E183E29BE00E945EA0EB969B
:1004A0001FAE1EAEEB97ED961FAE1EAEED978FEF13
:1004B0009FEFEF969FAF8EAFEF978DEE93E0E996AB
:1004C0009FAF8EAFE997C158DF4F19830883CF578D
:1004D000D040F8940E947A38CE0189589F4F0E94EC
:1004E00072A790932A0D8093290D7894C8010E94D9
:1004F000E23D8091290D90912A0D892B29F466EC1B
:1005000079E18EE29BE027C06BEB79E183E29BE02F
:100510000E945EA00E94F14664EB79E183E29BE0D9
:100520000E945EA084E090E0BBC06CE979E18EE2BD
:100530009BE00E945EA04AE050E0B7018EE29BE0A3
:100540000E9415A08EE29BE00E94A35106C069E8BC
:1005500079E186ED9BE00E945EA08EE090E0A0C075
:10056000D7011D96BC901D971E96AC90DF92CF923E
:1005700085E899E19F938F931F930F930E941AB977
:10058000DF92CF9280E899E19F938F931F930F930F
:100590000E941AB9D8011C96ED91FC911D9781E03B
:1005A0008283DF92CF928DE799E19F938F931F9380
:1005B0000F930E941AB9D8011C96ED91FC911D97DA
:1005C0001282AF92BF9287E499E19F938F931F931A
:1005D0000F930E941AB982E899E19F938F931F931A
:1005E0000F930E941AB9F701148A138AD8011C9636
:1005F000ED91FC911D97A080B1800FB6F894DEBFFD
:100600000FBECDBF83E3C82ED12CD501ED91FC9157
:100610000084F185E02DC501199541975CF4B1E0A6
:10062000CB1AD10839F064E170E080E090E00E94DC
:100630004A4EEBCF6E01F7E7CF0ED11CDF92CF927F
:100640008BE399E19F938F931F930F930E9437B988
:100650000F900F900F900F900F900F90019709F04F
:100660000CCFF60180819181D70154969C938E9393
:100670005397D12C80E08A3039F4BAE0DB1609F4C4
:10068000FCCE9AE0D92E03C08D3009F0D82EC801D7
:100690000E94DCB88F3F79F7C8010E94E23DEDCEA1
:1006A000C058DF4F0FB6F894DEBF0FBECDBFDF914D
:1006B000CF911F910F91FF90EF90DF90CF90BF905F
:1006C000AF9008950E943B819093FD088093FC08B1
:1006D00080E19CE00C94388C089585E090E00895CA
:1006E000DC011496ED91FC911597309719F08289F1
:1006F0009389089580E090E0089508950C947FB662
:100700000C947FB68F929F92AF92BF92DF92EF923E
:10071000FF920F931F93CF93DF93CDB7DEB7289748
:100720000FB6F894DEBF0FBECDBF09831A832B83AB
:100730003C834D835E836F837887DC011496ED9153
:10074000FC9115973097A9F120813181232B89F1F4
:100750008C01ED91FC910484F585E02D19957C01C7
:10076000019739F58B81982F9F70A92EB12CD980D4
:10077000DD20C9F1A114B104F9F0913001F19130FB
:1007800008F445C0923009F442C09C3009F462C0BC
:1007900064E87CE186ED9BE00E945EA04AE050E0C8
:1007A000B50186ED9BE00E9415A086ED9BE00E94BE
:1007B000A351E12CF12C63C0AA24A394B12C8FEF98
:1007C0008D0D823090F46D2DF801828193810E940D
:1007D0000CB060E071E0D80112968D919C91139756
:1007E0000E94703F4CC0913051F664E97CE186ED87
:1007F0009BE00E945EA04AE050E06D2D86ED9BE0FC
:100800000E94BF9F86ED9BE00E94A351C1CF807FD5
:1008100081F2CE0101960E9415374B015C01D8018F
:100820001496ED91FC91159762877387848795875D
:1008300061EA7CE186ED9BE00E945EA022E0B501CA
:10084000A40186ED9BE00E942E7586ED9BE00E9440
:10085000A35115C0807F09F4ACCFCE0101960E9450
:1008600015374B015C01D8011496ED91FC91159759
:1008700066837783808791876BEA7CE1DBCFC70152
:1008800028960FB6F894DEBF0FBECDBFDF91CF9193
:100890001F910F91FF90EF90DF90BF90AF909F90CE
:1008A0008F900895FC01828193810E9437B021E0EE
:1008B00030E0823011F420E030E0C90108952F9239
:1008C0003F924F925F926F927F928F929F92AF92E0
:1008D000BF92CF92DF92EF92FF920F931F93CF932D
:1008E000DF93CDB7DEB769970FB6F894DEBF0FBEC2
:1008F000CDBFDC011496ED91FC911597309709F46A
:100900007AC120813181232B09F475C19C878B87A3
:10091000ED91FC910484F585E02D1995019709F07E
:100920006AC1EB85FC8582819381009709F463C1DC
:100930000E9437B0823009F45EC1AB85BC85149645
:10094000ED91FC91159700811181F80182AD88230A
:1009500009F451C10E94844E698B7A8B8B8B9C8BDE
:10096000F80182A193A1A4A1B5A149895A896B89F3
:100970007C89481B590B6A0B7B0B86A597A5A0A900
:10098000B1A9481759076A077B0708F434C1048CDA
:10099000F58DE02D80819181A281B3818D879E8725
:1009A000AF87B88BD8019096ED91FC9191972D85EA
:1009B0003E854F85588960817181828193810E9433
:1009C00010C04B015C01F80122A533A544A555A533
:1009D0006D857E858F8598890E9410C06B017C0192
:1009E000D80150962D913D914D915C915397C50141
:1009F000B4010E94E1C1F80126A137A140A551A58B
:100A00000E9411C02B013C01D80196966D937D93F5
:100A10008D939C939997DB96BC91BD8BB11116C0B9
:100A2000F8012485358546855785C701B6010E94A2
:100A3000E1C19B01AC01C301B2010E9410C0D80109
:100A400096966D937D938D939C939997F80146A00C
:100A500057A060A471A4F6A9F987D801D796BC91D4
:100A6000BA87F80130AC21AC29853B2F432D522D9C
:100A7000C301B2010E94DCC118162CF489859A8545
:100A8000A32DB22D17C0D801D2968D919D910D90B6
:100A9000BC91A02D8E8B9F8BA88FB98F9C01AD012F
:100AA000C301B2010E947DC087FF09C08E899F8962
:100AB000A88DB98DF80186A397A3A0A7B1A7FD893A
:100AC000FF2371F0D8011C962D913D914D915C91C1
:100AD0001F97C501B4010E94E1C14B015C0103C035
:100AE000812C912C5401F801248935894689578934
:100AF000C701B6010E94E1C19B01AC01D8019696E5
:100B00006D917D918D919C9199970E9410C0A50146
:100B100094010E9411C06B017C019B01AC016985AD
:100B20007A85832D922D0E947DC087FD18C0F80123
:100B3000F2A9F987D801D396BC91BA87F80134A8F5
:100B400025A829853B2F432D522DB601C7010E94B0
:100B50007DC087FD04C0C986DA863E2C2F2CD801C3
:100B60005E96ED91FC915F9789859A85A32DB22DB4
:100B700080839183A283B3838D859E85AF85B88959
:100B8000F80182A793A7A4A7B5A789899A89AB89F9
:100B9000BC8982A393A3A4A3B5A3AB85BC851296FD
:100BA000ED91FC91139761E0828193810E94A4A949
:100BB000AB85BC851496ED91FC9115973281B3817C
:100BC000A481E58119821A821B821C820B810F701D
:100BD0000067232F432F5B2F6A2F7E2F4D835E8369
:100BE0006F837887E980FA801C813E814F81588528
:100BF0006FEF0E94439581E090E069960FB6F894FC
:100C0000DEBF0FBECDBFDF91CF911F910F91FF903F
:100C1000EF90DF90CF90BF90AF909F908F907F909C
:100C20006F905F904F903F902F900895CF93DF93F8
:100C3000EC0161ED76E089E39BE00E94C077EC81F6
:100C4000FD81309721F0808191810E947FB68C8157
:100C50009D810E947FB660E070E08A819B810E9446
:100C600067AE1D821C8281E090E0DF91CF910895F4
:100C70002F923F924F925F926F927F928F929F92AC
:100C8000AF92BF92CF92DF92EF92FF920F931F939A
:100C9000CF93DF93CDB7DEB72E970FB6F894DEBFB4
:100CA0000FBECDBF1C010E94255BD10114968D9112
:100CB0009C911597892B79F484E190E00E94E7B527
:100CC000BC01F101828193810E9467AED10115962A
:100CD0009C938E931497F1010480F581E02DFA879F
:100CE000E987EF2B59F461E77CE18EE29BE00E94FB
:100CF0005EA08EE29BE00E94A351E8C2A985BA855E
:100D00001D921C92F1010280F381E02DFE87ED8798
:100D100002811381EF2B09F460C20115110509F45A
:100D20005CC2D80118968C918F70853009F055C23D
:100D3000C8010E9425AA882309F44FC260E0C801B7
:100D40000E94A4A98C01FC0180858F70853039F048
:100D500068E17CE18EE29BE00E945EA0A0C2C80137
:100D60000E9425AA823031F148F4813009F06BC02D
:100D7000C12CD12C7601460157013BC0863008F0CA
:100D800062C062E0C8010E94A4A9FC0190859F7026
:100D9000933029F4C184D284E384F4840EC0923069
:100DA00049F461857285838594850E942CC16B010D
:100DB0007C0103C0C12CD12C760161E0C8010E94E6
:100DC000A4A9FC0190859F70933029F481849284BA
:100DD000A384B4840EC0923049F461857285838502
:100DE00094850E942CC14B015C0103C0812C912C85
:100DF000540160E0C8010E94A4A9FC0190859F7085
:100E0000933029F441845284638474840AC09230FC
:100E100021F561857285838594850E942CC12B0103
:100E20003C0120E030E0A901C301B2010E947DC075
:100E300087FF19C077FA709477F87094E1E0F0E0DA
:100E4000FC87EB8712C01C861B86C12CD12C760137
:100E5000460157012601370108C01C861B86412C1C
:100E6000512C320102C01C861B86AD85BE851496AE
:100E7000ED91FC91159780858295807F859585956C
:100E800085958595823039F0833091F481859285FE
:100E9000A385B48511C061857285838594850E9480
:100EA0002CC1E985FA8562877387848795870AC094
:100EB00080E090E0A0EAB1E4E985FA858287938733
:100EC000A487B5878CE390E00E94E7B58C01898503
:100ED0009A850296D8015F969C938E935E9789853A
:100EE0009A8506965D969C938E935C9789859A85E4
:100EF0000A9691969C938E939097DA961C92F8019D
:100F000012AA13AA14AA15AA80E090E0AFE7B3E4EE
:100F100086AB97ABA0AFB1AF84E690E0A0E0B0E0C5
:100F200086A797A7A0ABB1AB8B859C85918F808F4F
:100F300020E030E0A901C301B2010E947DC087FD1D
:100F40007DC020E030E0A901C501B4010E947DC050
:100F500087FD74C020E030E0A901C701B6010E94FE
:100F60007DC087FD6BC081E090E0D8015B969C93CB
:100F70008E935A97DB968C93DB97F80140825182CF
:100F80006282738214968D929D92AD92BC92179755
:100F9000C086D186E286F3861C964D925D926D9254
:100FA0007C921F972DEC3CEC4CEC5DE3C501B40149
:100FB0000E94E1C14B015C01F801608B718B828B57
:100FC000938B2DEC3CEC4CEC5DE3C701B6010E9429
:100FD00082C06B017C01D80154966D937D938D93F3
:100FE0009C935797EB85FC85319741F5A3019201BE
:100FF00060E070E0CB010E9410C0D8011C966D9398
:101000007D938D939C931F97A501940160E070E000
:10101000CB010E9410C0F801608B718B828B938B87
:10102000A701960160E070E0CB010E9410C0D801DA
:1010300054966D937D938D939C9357970E94844E05
:10104000F80186A497A4A0A8B1A8DC01CB01881957
:101050009909AA09BB0982A393A3A4A3B5A3D101AB
:101060001496ED91FC9115971183008301151105DC
:1010700009F419C1F80182AD81113BC0068CF78DCE
:10108000E02DC080D180E280F380D8019696CD9289
:10109000DD92ED92FC9299975C96ED91FC915D97B3
:1010A00080819181A281B381F80182A793A7A4A72F
:1010B000B5A746A857A860AC71ACA3019201C701BF
:1010C000B6010E94DCC118166CF0F80142A853A8C2
:1010D00064A875A8A3019201C701B6010E947DC052
:1010E00087FF07C0D80196964D925D926D927C92D3
:1010F000999781E0F80182AFC501B4010E942AC12D
:101100009B01AC0160E070E48CE995E40E9482C030
:101110006B017C019B01AC01D80150966D917D91D2
:101120008D919C9153970E94E1C1F801608B718B66
:10113000828B938BA701960164897589868997892B
:101140000E9482C0D80154966D937D938D939C9399
:10115000579788E893E1A0E0B0E0F80186A797A749
:10116000A0ABB1ABD1011296ED91FC911397019018
:10117000F081E02D008111816DE47CE183E29BE050
:101180000E945EA0B80183E29BE00E94A9A083E2D6
:101190009BE00E94A351F1018281938119821A82FE
:1011A0001B821C821D821E821F8218862B812F703B
:1011B000E12CF12C01E01A813C8140E05E816F81DD
:1011C00078850E94FD18D1011496ED91FC91159738
:1011D00081E090E0938B828B7BC0C8010E9425AA9E
:1011E000E82ED80118968C918F70FF24F3948530E7
:1011F00009F4F12C69E37CE18EE29BE00E945EA0A1
:101200004AE050E061E070E08EE29BE00E9415A0B1
:1012100067E37CE18EE29BE00E945EA061E070E00B
:10122000ED85FE85EF2B11F460E070E04AE050E0C0
:101230008EE29BE00E9415A065E37CE18EE29BE0DC
:101240000E945EA061E070E0012B11F460E070E0AC
:101250004AE050E08EE29BE00E9415A063E37CE14F
:101260008EE29BE00E945EA06F2D70E04AE050E0AD
:101270008EE29BE00E9415A061E37CE18EE29BE0A0
:101280000E945EA061E070E0F1E0FE1510F460E005
:1012900070E04AE050E08EE29BE00E9415A08EE2F2
:1012A0009BE00E94A35160E67CE18EE29BE00E94FD
:1012B0005EA08EE29BE00E94A351D1011496ED91B5
:1012C000FC91159782E090E0938B828B80E090E018
:1012D0002E960FB6F894DEBF0FBECDBFDF91CF9133
:1012E0001F910F91FF90EF90DF90CF90BF90AF9044
:1012F0009F908F907F906F905F904F903F902F9036
:1013000008958F929F92AF92BF92CF92DF92EF9209
:10131000FF920F931F93CF93DF93CDB7DEB728973C
:101320000FB6F894DEBF0FBECDBF09831A83122F0C
:101330002B833C834D835E836F837887B7011F7057
:10134000C12ED12CDC011496ED90FC9015976115FF
:10135000710569F0FB018081882349F0D7011F9650
:101360008D919C9150970E94EC5E892B51F5D7018D
:101370001F96ED91FC915097E680F780812E912C7D
:10138000A12CB12CE114F104E1F06DED76E0C70180
:101390000E94EC5EFC0190859F70923049F481853B
:1013A0009285A385B48588159905AA05BB0549F0E2
:1013B00060EE76E0C7010E94EC5EF701E280F38008
:1013C000E1CFF980FF20A1F1C114D10419F011304F
:1013D00089F503C0CC24C394D12C8FEF8F0D8230BC
:1013E00020F16AEF7BE186ED9BE00E945EA04AE07F
:1013F00050E06F2D86ED9BE00E94BF9F86ED9BE045
:101400000E94A3516AEE7BE186ED9BE00E945EA004
:101410004AE050E0B60186ED9BE00E9415A086ED03
:101420009BE00E94A35180E001C081E090E014C0E5
:101430001130B9F2113068F467E07CE186ED9BE091
:101440000E945EA02B81207F81E090E029F480E063
:1014500003C01230B9F3D6CF28960FB6F894DEBF8A
:101460000FBECDBFDF91CF911F910F91FF90EF90F5
:10147000DF90CF90BF90AF909F908F900895089588
:10148000CF93DF931F92CDB7DEB76983DC01ED9177
:10149000FC910280F381E02D41E050E0BE016F5FDE
:1014A0007F4F19950F90DF91CF910895FC01818DA9
:1014B000928D0895FC018489958908952EEB33E07F
:1014C000FC0131832083FB01408951896289738942
:1014D000FC0142835383648375830895DC01ED919D
:1014E000FC91048CF58DE02D199480E00895FC01A9
:1014F0009485FB018485981303C081E0943009F43E
:1015000080E0089521E0FC018485843009F420E026
:10151000822F089508958F929F92AF92BF92DF928B
:10152000EF92FF920F931F93CF93DF931F921F921F
:10153000CDB7DEB77C014B018A01FC01A688B788D4
:10154000D08CCE0101960E9493A789819A810E9436
:10155000E36C8D2D0E94509B8017910720F48D2DF8
:101560000E94509B8C019801A401B5018D2D0E9411
:10157000EB9A0E94E26CF70186899789800F911F90
:10158000978B868BC8010F900F90DF91CF911F91A1
:101590000F91FF90EF90DF90BF90AF909F908F9052
:1015A0000895CF93DF93FC0124852430D1F0EC0122
:1015B0000E9413A8843181F0882371F0883161F092
:1015C0008C3161F4E881F9810084F185E02DCE0150
:1015D000199521E0892B19F420E001C021E0822F28
:1015E00001C080E0DF91CF9108958EBD00000DB461
:1015F00007FEFDCF8EB50895DF92EF92FF920F9315
:101600001F93CF93DF931F921F92CDB7DEB7D82ED3
:10161000CE0101960E9493A789819A810E94E36C72
:10162000E12CF12C8D2D0E94403F8C01892B21F063
:101630008D2D0E94403F7C010E151F0599F70E94D9
:10164000E26CC8010F900F90DF91CF911F910F9125
:10165000FF90EF90DF900895FC011382128288EED4
:1016600093E0A0E0B0E084839583A683B7838DE404
:1016700094E0918380838EEB93E097878687108A2E
:10168000118A128A138A84E0808F0895AF92BF92E4
:10169000CF92DF92EF92FF920F931F93CF93DF933E
:1016A000CDB7DEB7AF970FB6F894DEBF0FBECDBF94
:1016B0007C015B016A010EEB13E01A8309831B8234
:1016C0001C821D821E82CE0109960E942C8B1BA7B4
:1016D0000AA71CA61DA61EA61FA68091C909909147
:1016E000CA09A091CB09B091CC098EA39FA3A8A74A
:1016F000B9A78B839C83AD83BE8318861F82AE01FE
:10170000465D5F4FB501CE0101960E94904E81303B
:101710009105B1F4D701ED91FC910488F589E02D94
:101720001DA30CA38CA59DA5AEA5BFA58EA39FA3AD
:10173000A8A7B9A7A601BE016C5D7F4FC701199587
:10174000AF960FB6F894DEBF0FBECDBFDF91CF913D
:101750001F910F91FF90EF90DF90CF90BF90AF90CF
:1017600008959B0190E00496982F8827642F820F9C
:10177000931F0C94253F1F93CF93DF931F921F92CB
:10178000CDB7DEB7182FCE0101960E9493A78981AD
:101790009A810E94E36C60E170E0812F0E9498A71B
:1017A0004FEF62E070E0812F0E94B18B0E94E26CEB
:1017B0000F900F90DF91CF911F910895DF92EF92DC
:1017C000FF920F931F93CF93DF931F921F92CDB77A
:1017D000DEB7182FD62E7A01022F0E94BB8BCE01C6
:1017E00001960E9493A789819A810E94E36C4D2DF6
:1017F000402B60E070E0812F0E94B18BE114F10476
:1018000059F4E090330DF090340D8FEFE81AF80A98
:10181000F092340DE092330D4F2D64E070E0812F93
:101820000E94B18B4E2D65E070E0812F0E94B18B3C
:1018300061E070E0812F0E9498A70E94E26C81E035
:101840000F900F90DF91CF911F910F91FF90EF902C
:10185000DF900895CF93DF93FC01808D843029F0D1
:10186000EF010E94BB8B84E0888FDF91CF910895B8
:10187000CF92DF92EF92FF920F931F93CF93DF935C
:101880001F921F92CDB7DEB7FC01F484F4E0FF167F
:1018900099F18C01CE0101960E9493A789819A81CA
:1018A0000E94E36C68E070E08F2D0E9498A70E9470
:1018B000E26C0E94844E6B017C01C8010E9413A857
:1018C0008823B9F062E370E080E090E00E944A4E25
:1018D0000E94844EDC01CB018C199D09AE09BF0921
:1018E000883E9340A105B10540F3F80184850E942C
:1018F000BB8B84E0F80184870F900F90DF91CF912C
:101900001F910F91FF90EF90DF90CF900895CF93AC
:10191000DF9390E00496982F8827EC01C60FD71F1D
:101920000E94C43E8FE00E94F58A8D2F0E94F58AA6
:101930008C2F0E94F58A80E00E94F58AC82F0E94B1
:10194000C23E8C2FDF91CF910895CF92DF92FF920C
:101950000F931F93CF93DF931F921F92CDB7DEB7E4
:10196000F82E6B01CE0101960E9493A789819A817E
:101970000E94E36C68E270E08F2D0E94878C082F34
:1019800010E069E270E08F2D0E94878C702F66272F
:10199000682B21E030E0A6018F2D0E94A39A0E94BF
:1019A000E26C81E090E00F900F90DF91CF911F915A
:1019B0000F91FF90DF90CF900895CF93DF931F9208
:1019C000CDB7DEB7FC01218D328D232B49F0BE014E
:1019D0006F5F7F4F808D0E94A58C898190E002C04F
:1019E0008FEF9FEF0F90DF91CF9108958F929F928D
:1019F000BF92CF92DF92EF92FF920F931F93CF93FC
:101A0000DF931F921F92CDB7DEB7B82E6B017A011C
:101A1000CE0101960E9493A789819A810E94E36C6E
:101A2000812C912C8B2D0E94403F8C01892B21F021
:101A30008B2D0E94403F4C010815190599F701159F
:101A4000110599F463E070E08B2D0E94878C84313E
:101A5000D9F18823C9F101E010E08C3111F400E0E4
:101A600010E01195019511092FC0E016F1060CF454
:101A700087011016110644F568E270E08B2D0E9474
:101A8000878CE82EF12C69E270E08B2D0E94878C08
:101A9000FE2CEE24E82A9801A601B7018B2D0E94A6
:101AA000A39AE00EF11E4F2D68E270E08B2D0E948C
:101AB000B18B4E2D69E270E08B2D0E94B18B60E4FA
:101AC00070E08B2D0E9498A70E94E26CC8010F90D5
:101AD0000F90DF91CF911F910F91FF90EF90DF90CA
:101AE000CF90BF909F908F900895CF93DF93FC018C
:101AF000218D328D2115310519F48FEF9FEF11C023
:101B0000EC014217530708F0A901888D0E94F68C5A
:101B10001816190694F7298D3A8D281B390B3A8F20
:101B2000298FDF91CF9108950F931F93CF93DF9368
:101B30001F92CDB7DEB7FC01218D328D232B61F0D2
:101B40008C0141E050E0BE016F5F7F4F808D0E94AD
:101B5000F68C181619061CF08FEF9FEF08C0F801DD
:101B6000818D928D0197928F818F898190E00F9066
:101B7000DF91CF911F910F9108950F931F93CF93F2
:101B8000DF93CDB7DEB728970FB6F894DEBF0FBE50
:101B9000CDBF8C01D80159968D919C915A97892B74
:101BA00041F0ED91FC910284F385E02DC801199577
:101BB000F1CFF801808D0E94FC8A1816190654F5A1
:101BC00048E050E0BE016F5F7F4FD80158968C917E
:101BD0000E94F68C18161906FCF4D801509684E081
:101BE000FE01319601900D928A95E1F78D8190E08A
:101BF000982F88272E81820F911DF801958B848B59
:101C00008F8190E0982F88272885820F911D928FD1
